:020000040000FA
:040000006FD00400B9
:101000006F009044000000000000000090200020CD
:10101000A4220020A9BDF9F55C23002000000000F7
:10102000000000005C230020902000200000000051
:101030000000000090200020000000009020002010
:101040000000000090200020902000209020002030
:101050009020002090200020B82B0020902000201D
:10106000000000009020002090200020EC230020B1
:1010700090200020C22300209020002090200020FB
:101080009020002090200020902000209020002020
:101090009020002001A04111B7170040985F3AC688
:1010A000945F3247E39CE6FE3245410182800111A4
:1010B00013078008F337078093F787083EC20100C3
:1010C0000100B7170040930570052380B70413068D
:1010D00080FA2380C7040100010083C6B70493F699
:1010E000F60DA385D704238007049246F3A6068055
:1010F0000100010093760502D5CEF336078093F602
:10110000860836C4010001002380B7042380C70489
:1011100001000100B70614007D89558D88C70100C4
:1011200001000100010023800704A246F3A6068007
:101130000100010073370780137787083AC6010062
:1011400001002380B7042380C704010001000100CF
:1011500001003727004093061005A303D7802380A2
:101160000704B247F3A70780010001009307800836
:10117000F3B7078093F787083ECE01000100B71749
:101180000040130770052380E704130780FA2380CB
:10119000E7040100010003C7B70413670708A3852C
:1011A000E70423800704F247F3A70780010001004A
:1011B0000561828093760504BDC6F336078093F6F9
:1011C000860836C8010001002380B7042380C704C5
:1011D00001000100B7061400938606047D89558D31
:1011E00088C7010001000100010023800704C246F6
:1011F000F3A6068001000100733707801377870884
:101200003ACA010001002380B7042380C70401000B
:1012100001003727004093062005A303D7802380D1
:101220000704D24781B773370780137787083ACC12
:10123000010001002380B7042380C70401000100DE
:1012400098471367070C98C723800704E24719BF24
:101250000111814601468145114506CE6D24930753
:101260008008F3B7078093F787083EC601000100A6
:10127000B7170040130770052380E704130780FAAF
:101280002380E7040100010003C767041367170008
:101290002383E70423800704B247F3A707800100F4
:1012A0000100F2400561828041118146014681457D
:1012B0001145912C13078008F337078093F78708AF
:1012C0003EC401000100B7170040130670052380DB
:1012D000C704930680FA2380D70401000100FD555E
:1012E0002396B70223800704A245F3A505800100D9
:1012F000010073370780137787083AC601000100A1
:101300002380C7042380D7040100010003C76704BA
:10131000136717002383E70423800704B247F3A76A
:1013200007800100010001A0BD473305F50201005F
:101330007D1575FD8280411122C426C206C6AA848D
:10134000014463179400B2402244924441018280D8
:1013500005041305803E4204C13F4180DDB7000013
:101360009305000273A04580824573901534924026
:101370002242B2424243D2436244F2440255925561
:101380002256B2564257D2576258F25806499649E9
:10139000264AB64A464BD64B664CF64C065D965DE1
:1013A000265EB65E465FD65F09617300203041114C
:1013B000B7170040985F3AC6945F3247E39CE6FE59
:1013C000324541018280B71700401307000323888C
:1013D000E7028547171700002326F7F47300203033
:1013E000411122C406C6370400201C408297F5BF75
:1013F00037370040834747009146BD8B6389D7004C
:1014000099466394D700834757407300203097165E
:10141000000083C6F6F39387160017160000A30991
:10142000F6F203478700973700009387E75CB6978B
:101430002380E700B7E70400BC4F0946894517152C
:1014400000000345C5E98297C9B723030480154707
:101450002303E48001002302A48082808307648048
:10146000E3CE07FE23030480828083076480E3CEFB
:1014700007FE03454480828083076480E3CE07FE35
:101480002302A4808280411126C44AC24EC006C6EF
:101490001377F50BAD47AA892E8995446306F700AB
:1014A00019456537653F8D444E854537FD59FD1417
:1014B00063983401B240A2441249824941018280BA
:1014C000135509011375F50F453F2209CDB70111D9
:1014D00026CC06CEB704080051371545BD37713705
:1014E00069372AC6A53F32459377150089EB136506
:1014F00015001375F50FF240E24405618280FD147A
:10150000E9FC0145CDBF397126DC4ADA4ED852D606
:1015100056D45AD25ED006DE62CE66CCB7E700E083
:101520007D5783AA070022C603AA470023A0E71815
:1015300023A2E718B7170040130770052380E704BC
:10154000130780FA2380E70483C74704930B75FFD2
:10155000B684E20793FBFB0F8546AA892E8B32895E
:1015600037240040E187015763FA76016308D5000C
:101570008946130700026313D5000157D98F93F7EB
:10158000F70FB71C00402382FC0411472303E480BB
:101590001305F00F5D3D094CD135636D7C11B70526
:1015A0000700DA9537870700795563F2E504B387BA
:1015B0009500636EF702370B0800A94733EB65010E
:1015C0006399F90689E48144513D26850DA0DA85A9
:1015D0000945553D05090345F9FFFD14050B693D16
:1015E00081C49377FB0FFDF7DD3569FD7D55B71796
:1015F0000040130770052380E704130780FA238057
:10160000E70403C74704418B2382E704F250B7E79E
:1016100000E023A0571123A24711E254324452594B
:10162000C259325AA25A125B825B724CE24C21615F
:101630008280A5476395F90685691309F00FB30603
:101640009900B3742B01B6941349F9FFB374990050
:10165000856B33796901416B9387F9FFB3F72701F4
:1016600099E363FC340193D94900C147E3E637FFAE
:1016700099BF0569C1697D19D9B71305800D6388C4
:101680006901130500026384790113051008CA85F6
:10169000DD3B353D21DD4E99B3843441D9B7DA8540
:1016A0002D45D533CA94E30099F205097D3BA30F7C
:1016B000A9FED5BF9387F9FF93F7F70F6361FC0C81
:1016C00083C71C0413073008631FF704370708009B
:1016D000636BEB04B3079B00B706100063F5D704F8
:1016E000334BEB0089476393F9068980D549E38C36
:1016F00004ECDA850945413B11090327C9FF9147ED
:101700002320E48003076480E34E07FE2303348133
:10171000FD17EDFBFD14110B81C49377FB0FE9FF5F
:101720007D3371F5E1B5B717004003C75704B7071C
:1017300008001377070219E3B78707007955E378A4
:10174000FBEA33079B00E3FFE7F855B58547E382E3
:10175000F9F2DA852D45053B9389F4FFE38504E62C
:10176000293393F7390091EB83260480032709007E
:1017700093074900E39AE6E43E89CE84F1BFB5477A
:101780006396F9001305900BC93135BDB1471305B8
:10179000B00AE38BF9FE99476391F904B705080095
:1017A000B365BB002D45C53181448D4BA1497539C9
:1017B00063967401832704802320F9008504E3984D
:1017C00034FF8327048013172B016355070023126E
:1017D000F900D5BB2322F900FDB39D476399F902B7
:1017E00081451305B0044531BD442320090023225F
:1017F0000900FD599D3993F77400CA9703C7070084
:10180000FD14398D2380A700E39634FF6DBBA147FB
:101810006392F9046D398144630D0B008D47930485
:10182000C0036308FB009304000563048B01930469
:1018300040041375C507E30895D81945393139397E
:101840000545213126850D3909453D314931E31CD6
:1018500005D669BB91476399F90013056006F53613
:10186000F53E130590090DB7E38F09D4F154A9BBD8
:10187000BD660147173600001306C644938606A6C8
:1018800085458347060093F7F70F91C382800507CC
:10189000E3F9E6FE973700002386B742DDB77D16F1
:1018A0006206618693178601E18763D407000145CC
:1018B0008280931726003307F500AE9718439C43A8
:1018C00063E7E7007D16E37FF7FC7D5582800545E1
:1018D0008280FD15E205E18513978501618793F705
:1018E000F50F63480700FD15139725002A97584305
:1018F00065D7138517006205618582803308B502BC
:101900001C4283A80600B335B502C29733B5070160
:10191000AE98469585486367B5006394A50063E378
:10192000070181480C43C6950CC388C21CC2828043
:1019300081471397870161876343B70082801397BC
:1019400027002A97232007008507E5B7814701472D
:1019500093968701E18663C5B60013351700828030
:1019600093962700AA9694428507558FD5B793D7AB
:1019700055408A07AA979C4305453315B5007D8DD0
:10198000828017F3FFDFE702C33B2A84993705C53E
:10199000931725003E940327C4FF814711EB7D1563
:1019A00016053E954205418517F3FFDF6700A33B0F
:1019B00005838507E5B70145C5BF814713978701B3
:1019C00061876343C700828013972700B386E500D1
:1019D00094422A97850714C3D5B77D16620661869F
:1019E000014793178601E18763D507001335170078
:1019F000828093172600B306F500AE9794429C436D
:101A00007D16B58F5D8FF1BF8A05AA950147636387
:101A1000B500828083A6C5FFF11593D71600D98F34
:101A20009CC11397F601E5B72A8301480147014598
:101A30006343D7008280B387050183A80700B307FB
:101A400006019C43C697AA976384F80033B5170133
:101A50000507B3080301620723A0F8006187110896
:101A6000C1BF2A8301478147014563C3D7008280F4
:101A70003388E50083280800330EE600032E0E00AD
:101A80003388A8403308C8416384080133B508018E
:101A90008507B308E300E20723A00801E1871107E7
:101AA000E9B717F3FFDFE702C3290111B286B28459
:101AB0002E86AA850A8575372A84A6850A857935F2
:101AC00033348000060413351500018D056117F3CA
:101AD000FFDF6700432917F3FFDFE702032441110B
:101AE000AA89AE8A328BB68402C202C402C60144FD
:101AF000131C8401135C8C4163499C02939B14006A
:101B0000FD1B0549138CF4FFF15C33048901620469
:101B10006184634D740592478E04CE9423AEF4FE27
:101B2000410117F3FFDF6700C32213192400B30B31
:101B30002B01014A93172A00D69783A50B008843EF
:101B40007800340050005D3B050A93178A01E18755
:101B5000F11BE351FCFE92474E9905042320F90046
:101B6000A2473EC2B24702C63EC459B7131A890102
:101B7000135A8A41131D240093178A01E18763CF0A
:101B8000970092470A044E941CC0A2470509137996
:101B9000F90F3EC2B24702C63EC485BFB3079A03DF
:101BA00013152A0056950841780034005000050AA4
:101BB000EA97DA978C439933C1B70000197106C2CE
:101BC00012C416C61AC81ECA22CC26CE2AD02ED2BD
:101BD00032D436D63AD83EDA42DC46DECAC0CEC26D
:101BE000D2C4D6C6DAC8DECAE2CCE6CEEAD0EED29D
:101BF000F2D4F6D6FAD8FEDA97050000938505727E
:101C00008841E700050092402242B2424243D2435B
:101C10006244F244025592552256B2564257D25768
:101C20006258F25806499649264AB64A464BD64B60
:101C3000664CF64C065D965D265EB65E465FD65FE8
:101C40000961730020300000972100209381813BBF
:101C500017510020130101BB17F5FFFF1305C53A0B
:101C6000970500209385053A171600201306C6FD38
:101C700063FAC5008322050023A0550011059105D4
:101C8000E3EAC5FE17A501001305055097150020CE
:101C90009385C5FB171600201306C66563FAC500B9
:101CA0008322050023A0550011059105E3EAC5FE36
:101CB0001715002013050564974500209385854C72
:101CC0006377B500232005001105E36DB5FEFD42E5
:101CD000739002BC8D4273904280B72200009382C1
:101CE000828873900230970200209382A23193E29F
:101CF00032007390523097420000938262F17390E9
:101D000012346FC0E42F73002030397101436EC666
:101D100019A0397141536AC866CA62CC5ECE19A057
:101D2000397101535AD056D252D44ED64AD826DAF7
:101D300022DC06DE33016140828241114AC026C2A4
:101D400022C406C68282B24D4101024D924C224C01
:101D5000B24B4101024B924A224AB2494101024927
:101D600092442244B240410182803D432A876373FA
:101D7000C3029377F700BDEFADE5937606FF3D8A8A
:101D8000BA960CC34CC30CC74CC74107E36BD7FED4
:101D900011E28280B306C3408A069702000096963D
:101DA0006780A6002307B700A306B7002306B70085
:101DB000A305B7002305B700A304B7002304B700A9
:101DC000A303B7002303B700A302B7002302B700A1
:101DD000A301B7002301B700A300B7002300B70099
:101DE000828093F5F50F93968500D58D9396050126
:101DF000D58D61B79396270097020000969686824C
:101E0000E78086FA9680C1171D8F3E96E374C3F86B
:101E1000A5B73367B500FD530D8B79E7B7877F7F93
:101E20009387F7F710419441B372F6003363F600DD
:101E3000BE92B3E262006397720C6318D6065041FB
:101E4000D441B372F6003363F600BE92B3E262008F
:101E50006398720A631BD60410459445B372F6006A
:101E60003363F600BE92B3E262006391720A631EAE
:101E7000D6025045D445B372F6003363F600BE92E5
:101E8000B3E26200639A72086311D6021049944962
:101E9000B372F6003363F600BE92B3E2620063935E
:101EA00072085105D105E30FD6F613170601939773
:101EB0000601631CF7001357060193D7060133058B
:101EC000F7409375F50F91E982804183C183330513
:101ED000F7409375F50F91E182801377F70F93F731
:101EE000F70F3305F74082800346050083C60500DF
:101EF000050585056313D60065FA3305D640828053
:101F000011059105E312D6FE014582802105A10548
:101F1000E31CD6FC014582803105B105E316D6FCF1
:101F2000014582804105C105E310D6FC0145828050
:101F3000B717004003C777051377E70FA38BE704B4
:101F4000130700F8A38DE7043D47238CE70413072C
:101F50005003A38CE70403C7A7051377D70F238D7E
:101F6000E7048280B717004003C7E7020D894111DB
:101F70001377C70F498F93068008F3B6068093F650
:101F8000860836C601000100930670052380D70439
:101F9000930680FA2380D704010001002387E7021B
:101FA00023800704B247F3A7078001000100410125
:101FB000828041112A83014E930E407E130F001937
:101FC000930F400663E56E12930800191303400651
:101FD000B3781503854E0D4FA14F337365020D89FC
:101FE0001335150063EFBE121308F6FF7946729899
:101FF0004208135808013307C70213D61700BE075B
:1020000032976146B3F6C60213068070B386C602E5
:102010003697A166F58F42075D8FB716004083C7DC
:10202000F60293F70708A303F1000346710083C784
:10203000F60293F70708E394C7FE83477100B716CB
:10204000004093F7F70F6388071293078008F3B7F0
:10205000078093F787083EC401000100B7170040CE
:10206000930670052380D704930680FA2380D70453
:102070000100010023AA070383C6170393E606089D
:10208000A388D70223800704A247F3A70780010093
:1020900001001166B71700407D16D45BC85F9385B9
:1020A0004703A98EF18EF5FA93068008F3B60680F1
:1020B00093F6860836C6010001009306700523805A
:1020C000D704930680FA2380D7040100010098C149
:1020D00003C7170313670704A388E70223800704D5
:1020E000B247F3A7078001000100410182807D1300
:1020F0003368E3039308E016630E08003368F303C4
:102100009308D016630808009378330093B818003A
:102110009388D81633081E01131E0801135E0E01A2
:1021200055B56393E50305486386080001486303DA
:1021300003002A8871087298FD15131E0801C20554
:10214000135E0E01C18179BD13F8150063F4BF0061
:102150007908D5B713381800E5BF83C7F60293F79F
:102160000708A303F1000346710083C7F60293F743
:102170000708E394C7FE8347710093F7F70FF1DF79
:10218000E9B531714AD966CB06DF22DD26DB4ED7B1
:1021900052D556D35AD15ECF62CD6AC96EC7AA8CCA
:1021A00002D8EF00901C2A8993078008F3B70780B4
:1021B00093F787083EDA01000100B71700401307C4
:1021C00070052380E704130780FA2380E7040100E9
:1021D000010003C7F7021377770FA387E70203C74E
:1021E000F70213678700A387E70223800704D2570B
:1021F000F3A70780010001000545AD33130780C137
:102200003347E902116A93070AE893065002BD6951
:10221000930BA004814A014B1304800893047005BA
:102220007D1AB347F9023307D7023EC0FD873ECC83
:10223000938709A69309803E3347F7023AC27D8708
:102240003AC4334739038549B399990193D9394041
:10225000B306D702B30B7703B3C6F602B3CBFB02C8
:1022600036C6FD8636C893D6FB4136CEB7460F003C
:10227000938606243349D9028566938606FAB39677
:102280009601B389E902130760553309D902930611
:102290000010B389E9023349D902B3C9F902931690
:1022A000390036CA37190040FD8636D0930D09042F
:1022B00093D7F9413ED2F336048093F6860836DC94
:1022C00001000100930770052380FD00930680FA4A
:1022D0002380DD00010001008346390593F6860F57
:1022E000A309D9048346390593E61600A309D90446
:1022F00023800D00E256F3A6068001000100130CB6
:1023000080FA116DF336048093F6860836DE0100FC
:102310000100930770052380FD0023808D010100DB
:10232000010083463905216693E60602A309D90414
:1023300083560905B3E6A6012318D9048356090577
:10234000D18E2318D90423800D00F256F3A60680FF
:10235000010001008346390593F60602638A0618D8
:1023600003463905218A6DDE0818EF001004733624
:10237000048013768608B2C20100010023809D000C
:1023800023808D0101000100B717004003C6370507
:102390001376F60DA389C70403C637051366060234
:1023A000A389C704835609052166B3E6A60123184D
:1023B000D90483560905D18E2318D90423800D0032
:1023C0009646F3A60680010001008346390593F680
:1023D00006026386061483463905A18AEDFE97003E
:1023E0000020E78040CBAA8636D497000020E78003
:1023F00080CAA256E30AD5FE835609054255B3E6C4
:10240000A6012318D904C12783463905A18AEDDE28
:10241000035609058346290582473376CA00B30669
:10242000DA0293D5F641B296B388F640E24733B864
:10243000C6002E983308F840A247B3B616013308F9
:10244000D84063C70701631DF800924763FA17017C
:10245000C247634DF80E63950701B24763E8F80E73
:10246000894663E7660FF2469315180013D3F80107
:102470005E8613951800B365B30042D646D4EF606C
:10248000E1363258050B137BFB0F634700016312E3
:102490000838A258638F083613081500B336A80011
:1024A000B69513D6F5013298B336C800AE961358D8
:1024B0001800FE06B3E6060173360480137686081C
:1024C000B2C60100010023809D0023808D01010020
:1024D00001000356C902B296C206C1822316D90270
:1024E00023800D00B646F3A606800100010019BD49
:1024F000F336048093F68608B6C0010001002380FD
:102500009D0023808D01010001008346390593E67B
:102510000602A309D90423800D00864605BDF336C3
:10252000048093F68608B6C40100010023809D0054
:1025300023808D01010001008346390593E60602E0
:10254000A309D90423800D00A646A5BDE30D0BF019
:10255000F336048093F68608B6C80100010093069E
:1025600080FA23809D002380DD0001000100834666
:10257000390593F5FC0F93F6860FA309D90483461A
:102580003905CD8EA309D90423800D00C646F3A6D4
:10259000068001000100130580FA03463905930601
:1025A00039051D8A631496297336048013768608CC
:1025B000B2CC01000100130680FA23809D00238025
:1025C000CD000100010003C606001376F60D23803E
:1025D000C60003C60600136606022380C6008356A3
:1025E00009051166D18E2318D90483560905216681
:1025F000D18E2318D90423800D00E646F3A6068069
:1026000001000100130680FA8346390593F606029D
:102610006388062483463905130C3905A18AFDDA3F
:1026200008186123F336048093F68608B6D00100BB
:102630000100930680FA23809D002380DD000100C5
:10264000010083460C00116693F6F60D2300DC00B2
:1026500083460C0093E606022300DC00835609053E
:10266000D18E2318D904835609052166D18E2318EB
:10267000D90423800D008656F3A6068001000100D0
:10268000130680FA8346390593F606026385062011
:1026900083463905A18AEDFE97000020E780A09FC0
:1026A0002A8C97000020E780009FE30C85FF83566B
:1026B000090511664255D18E2318D9042923834672
:1026C000390513063905A18AFDDAF336048093F63D
:1026D0008608B6D401000100930680FA23809D008D
:1026E0002380DD00010001008346060093F6F60D0D
:1026F0002300D60023800D00A656F3A60680010015
:1027000001008356090503462905D247B376DA004E
:102710003306CA021305800C9355F6413696330DE5
:10272000F6408257333CD6002E9C3336A601330C3C
:10273000FC40330CCC403308850392564E86B335AB
:10274000A5033305A503C295EF60410A63468001E6
:10275000631E0C16630C0D16130615003335A60008
:102760002E959356F5013696B335D600AA959396D5
:10277000F50105828585D18E6346B000639D051AFB
:10278000638B061A0356C90215823305D600333609
:10279000C500B2956348B000639105241306F00F9D
:1027A000637DA622894663F3561593078008F3B725
:1027B000078093F78708BED6010001003717004055
:1027C000930770052300F704930780FA2300F704AA
:1027D000010001008356C70289678117D58FC207A0
:1027E000C1832316F70223000704B657F3A7078017
:1027F00001000100FA506A54DA544A59BA592A5A67
:102800009A5A0A5BFA4B6A4CDA4C4A4DBA4D296126
:1028100082801308F5FF3335A800FD152E95135659
:10282000F5013298B336C800AA9651B1F336048048
:1028300093F68608B6CA0100010023809D0023801C
:10284000AD000100010083463905CD8EA309D904EE
:1028500023800D00D646F3A606800100010035BB9B
:10286000F336048093F68608B6CE0100010023807B
:102870009D002380CD00010001008346390593E6C9
:102880000602A309D90423800D00F646F3A60680AC
:102890000100010095BBF336048093F68608B6D29A
:1028A0000100010023809D002380CD000100010074
:1028B0008346390593E60602A309D90423800D0057
:1028C0009656F3A60680010001006DBB9306F5FF46
:1028D00033B5A600FD152E959355F501AE96B3B50B
:1028E000B600AA951396F501858269B5F336048082
:1028F00093F68608B6D801000100930680FA23807B
:102900009D002380DD00010001008356C902056699
:10291000011693F6F60FD18EC206C1822316D90294
:1029200023800D00C656F3A6068001000100850A2B
:1029300093FAFA0F49B233E6B60045C20356C9020C
:102940003305D0403338A000B305B040B38505410E
:1029500015826345B000D1E16371A608894663F032
:10296000560593078008F3B7078093F78708BEDA08
:1029700001000100B7170040130770052380E7042A
:10298000130780FA2380E7040100010003D7C70280
:102990007D8B2396E70223800704D65781BDF3364B
:1029A000048093F68608B6DC01000100930680FAE5
:1029B00023809D002380DD00010001008356C902B1
:1029C0000566011693F6F60FD18EC206C182231654
:1029D000D90223800D00E656B9B793078008F3B7F4
:1029E000078093F78708BEDE01000100371700401B
:1029F000930770052300F704930780FA2300F70478
:102A0000010001000356C70293975600B297C20710
:102A1000C1832316F70223000704F657C1BB914771
:102A200063EEB702178701001307C7AC8A05BA9592
:102A30009C41BA978287B717004003A7470B1345FD
:102A4000F5FF698F23AAE70A03A7070B698F23A85D
:102A5000E70A03A7070A798D23A0A70A8280B71780
:102A6000004083A6470B1347F5FFF98E23AAD70A28
:102A700083A6070B558D23A8A70A83A6070A758F7F
:102A800023A0E70A8280B717004003A7470B498FAE
:102A900023AAE70A03A7070B1345F5FF45BFB7179E
:102AA000004083A6470B1347F5FF758F23AAE70A5B
:102AB00003A7070A598D4DB7B717004003A7470B67
:102AC000498FEDB7914763EEB702178701001307EF
:102AD000A7A38A05BA959C41BA978287B717004089
:102AE00003A7470D1345F5FF698F23AAE70C03A73A
:102AF000070D698F23A8E70C03A7070C798D23A086
:102B0000A70C8280B717004083A6470D1347F5FF37
:102B1000F98E23AAD70C83A6070D558D23A8A70CE1
:102B200083A6070C758F23A0E70C8280B71700409F
:102B300003A7470D498F23AAE70C03A7070D1345E9
:102B4000F5FF45BFB717004083A6470D1347F5FFB4
:102B5000758F23AAE70C03A7070C598D4DB7B7173C
:102B6000004003A7470D498FEDB7B71700408847CE
:102B7000420541819377050491EB9377F501375531
:102B8000E801130505803345F50282809377050C33
:102B9000130700046397E7009377F50137459C1C02
:102BA000CDB72165130505D0828037E700E01C43CF
:102BB0005443A183E206D58F1CC1FD572320F7188B
:102BC0002322F718828013178500B7E700E023A0BF
:102BD000E710618123A2A7108280B7F700E0884741
:102BE000CC478280814737370040A14663C4C70085
:102BF000328582800345B740E38EA6FE3385F5001B
:102C00000345050085072304A740CDB7970700209B
:102C10009387476A9C43173700201307A7563E95B2
:102C2000636EE500174700201307C79D6368A70080
:102C3000170700202320A7683E858280FD57EDBF3F
:102C4000411122C406C62A840D372947B307E5027D
:102C5000B2408D83B3D7870222449507B3D7E702EA
:102C600037370040C207C1832316F7004101828035
:102C7000716541111305052006C6D937B7370040E5
:102C8000130770F82381E7000D47A381E7001307BE
:102C90000004A380E70005472387E700B240410115
:102CA000828037370040834727001A0593F7F703E0
:102CB000C98F93F7F70F2301F7008280B7370040E1
:102CC00003C7170019C9D98DA380B70003C7070030
:102CD000136787002380E700828093C5F5FFF98D95
:102CE000A380B7008280B73700402147B736004045
:102CF00091E1828003C6B700E30CC7FE05050346D9
:102D0000F5FFFD15C2052384C600C181D5B7411169
:102D100022C406C62A84913D2947B307E502B24082
:102D20008D83B3D7870222449507B3D7E70237379D
:102D30000040C207C1832316F740410182807165BC
:102D400041111305052006C6D937B73700401307D0
:102D500070F82381E7400D47A381E7401307000483
:102D6000A380E74005472387E740B24041018280C6
:102D7000CC41411106C6328503C6150083C5050046
:102D800022064D8E42068D654186138875A2630C1E
:102D90000611634BC804138845A26300060D634AFD
:102DA000C800938535A26301B60823900600294622
:102DB0004DA0138855A26305060D938565A2E31601
:102DC000B6FE8D451D4663E6E5081146198E63F390
:102DD000C7003E86B7E704002390C600FC479795DE
:102DE0000100938565349DA0138895A263030611A5
:102DF000634E060D1388A5A263000613938505A5EF
:102E0000E315B6FA99451D4663E5E504198E63F3AB
:102E1000C7003E86B7E704002390C600FC4797052D
:102E200000209385A5491DA09D451D4663E3E5024D
:102E30002146198E63F3C7003E86B7E70400FC47BE
:102E40002390C600970500209385C54ABA958297BE
:102E50000146B240328541018280AD451D46E3EA1C
:102E6000E5FE3146198E63F3C7003E86B7E70400DE
:102E70002390C600FC47977501009385E56BF9B771
:102E8000B1451D46E3E7E5FC3546198E63F3C700FF
:102E90003E86B7E704002390C600FC479775010003
:102EA0009385856A65B78D451D46E3E4E5FA1146CD
:102EB000198E63F3C7003E86B7E704002390C6006F
:102EC000FC47979501009385E52649B78D451D463A
:102ED000E3E1E5F81146198E63F3C7003E86B7E7D4
:102EE00004002390C600FC47979501009385452672
:102EF000B1BFA5451D46E3EEE5F42946198E63F3FF
:102F0000C7003E86B7E704002390C600FC479775CC
:102F100001009385A5611DBFB5451D46E3EBE5F2B4
:102F20003946198E63F3C7003E86B7E70400239045
:102F3000C600FC47977501009385455E01BFB7E762
:102F4000040003A3071397060020938626D9414661
:102F5000A54517050020130565CF02832D4559EFC0
:102F600003C5050009476317E50803A8450041119B
:102F700006C6034718003285034608002207416849
:102F8000518F930828FE6308170363E9E8000518CA
:102F9000630307052390060029451DA8130648FE74
:102FA000630BC7021518E31707FF15463E87637BBF
:102FB000F602154705A83E8691C30546B7E704000B
:102FC000FC472390C6004206CC45418282970145CA
:102FD000B240410182801306700F3E876374F60091
:102FE0001307700FB7E704002390E600FC471316A1
:102FF0000701D9BF23900600054582808280416782
:1030000079176304E504411122C406C685472A8462
:10301000639FF500B7E7040022852244B24003A372
:103020008713970500209385A52D410102838947C9
:103030006399F500B7E7040083A7070B85458297DE
:1030400071D9B2402244410182808280797122D4B8
:1030500052CC2E842A8A97750100938525511775C5
:1030600001001305655206D63AC626D24AD0B68468
:1030700032894ECEEF50D142A68517750100130557
:10308000A551EF50F1412945EF50D14583478400C8
:1030900093F70702E1E78349040089470545324772
:1030A0006396F908544083C7160083C60600A2073A
:1030B000D58FC166138616FE638CC7028D16638F8B
:1030C000D7068D669386269029456391D706B7E784
:1030D0000400A285225403A34714B250F249A686E5
:1030E0004A86925402595285624A85474561028355
:1030F0002D450DEF9307700F354563E99702B7E74C
:103100000400FC4748441306700FCA858297814922
:10311000970700209387871F9C43014581CB9C43E1
:1031200091C74E852686CA8582970145B2502254A2
:1031300092540259F249624A456182802D457DF7D9
:103140009307700F3545E3E397FEB7E70400FC47AC
:1031500048441306700FCA8582975DBF2145F9B7B1
:10316000411122C437E404008327841326C2AA84B1
:10317000416506C697050020938585187D158297C1
:103180008327C40A170500001305A5E785888297E1
:1031900095C0032304132244B240924497060020B2
:1031A000938686C54146C545170500201305C5B35E
:1031B00041010283B2402244924401454101828090
:1031C00019C59707002023A3A71401458280454510
:1031D00082801147636AA70A977601009386C637F3
:1031E0000A0536951841411106C63697AE87B28555
:1031F00002871307700F6145639DE700B7E704007E
:10320000FC471306700F170500201305E51682977B
:103210000145B2404101828005476145E39BE7FEDD
:10322000B7E70400FC470546170500201305050D08
:10323000F9BF1307700F6145E39DE7FCB7E7040092
:10324000FC471306700F1705002013056522C1B750
:103250001307700F6145E39EE7FAB7E70400FC47E8
:103260001306700F17050020130505304DB71547DD
:103270006145E390E7FAB7E70400FC4715461705F8
:1032800000201305250861B709458280411126C237
:10329000B7E4040083A7C41322C44AC006C62E8420
:1032A000970500209385C5052A898297058905C55C
:1032B00097070020938747A383D7A70BA28503A373
:1032C000440D2310F4002244B24092444A8502493E
:1032D000014641010283B2402244924402494945D9
:1032E000410182809707002023840702970700206E
:1032F00023A20702B717004003A7070CB706C0FFB9
:10330000FD16758F23A0E70C03A7070DB706400035
:10331000558F23A8E70C03A7070C3D9B23A0E70CC0
:1033200003A7070D1367070123A8E70C8280B717CF
:10333000004003A5470C83A7470C5981134515008E
:10334000C18B058999E3136525009707002083C782
:1033500027FC6380A70297070020238BA7FA11C9D7
:1033600097070020938707FB03A30700630303006D
:103370000283828011456FE0DFE0411193962500C2
:10338000AA852D4506C697F0FF1FE780C017B240FB
:10339000014541018280011122CC06CE3714004044
:1033A00026CA4AC84EC652C483447405034AB405AB
:1033B0008349840503499405EFE09FB78347A4053B
:1033C00093F4F40F137AFA0F93E71700230DF40424
:1033D00093F9F90F1379F90FB717004003C7A70541
:1033E000058B6DFF03D5C705A38D4705238C3705D6
:1033F000A38C2705A38B9704F2406244D244424930
:10340000B249224A0561828041119397050122C485
:1034100006C626C2C1872E8463DC0700B7E4040019
:10342000FC54829719C1BC5482972165218D3DA01F
:1034300093F7150013C5150095E393F7250085C78D
:10344000FD35B7E70400BC4F1306000A8945170590
:1034500000200345A5EC829713452400B240224486
:103460009244410182809397250163D50702B7E416
:10347000040083A7C41E8297F53DBC4C37F60200BA
:10348000130606E0896517050020034525E98297A4
:10349000096569BF939715010145E3D107FC1775CD
:1034A000010013052516EF507114B7E70400BC4F57
:1034B00013060064916517050020034525E68297F1
:1034C0001165ADB72D71232A9110FD74E98C232C61
:1034D000811023282111232631112A84AE893289B3
:1034E000930600100A86A6852D45232E111097F00D
:1034F000FF1FE780400113154401B7E70400FC47B4
:1035000051810A0513962900CA850A958297A685D6
:1035100085660146254597F0FF1FE780C0FE0A86B5
:10352000A68593060010294597F0FF1FE780A0FDB0
:103530008320C11103248111832441110329011126
:103540008329C11015618280B7F7070003C70701FF
:10355000411106C622C426C24AC0A547631AF70015
:103560009537B2402244924402490145410182808C
:1035700013942500AA843289A286AA85014625458E
:1035800097F0FF1FE78020F8A2864A86A685294586
:1035900097F0FF1FE78020F7E9B71D71A2CC37E451
:1035A00004005C5C485886CE4946977501009385B7
:1035B000E500829701E91775010013056501EF50D9
:1035C000F10201A0B7F600E0795798CAFD57DCCAAE
:1035D0000567B7E700E023A0E7101306F00290C2EA
:1035E00023A0E71801000100370700201847130641
:1035F000000481459706002023A0E6D24157A38A04
:10360000E7403C440808829797170020938787DE9D
:103610003EC8856713870760231AE1001D673ACC0F
:1036200037070105130707103ACE9387B7D313075F
:10363000B00F2310E1022312F102054797F7FFFFB5
:103640009387E7592301E1023ED8170700001307CB
:1036500007D397070000938747D4B7F50700BAC28E
:103660003EDC17070000130767EE970700009387FB
:10367000A7D081463000E1051945BAC43EDE97F077
:10368000FF1FE78040E818088147994630003E96C2
:103690000346060085070507A30BC700E398D7FE7E
:1036A000C24791C70357410185676373F70001A0C3
:1036B000B7E7040083A7470A08088297AA8501C9CB
:1036C00017750100130505F2EF50815D01A0F6406A
:1036D000664425618280411126C2B7E4040083A7B5
:1036E000040806C622C417050000130525D28297D8
:1036F00017040020130484C22300A4003128DD36FF
:1037000003450400224403A38405B24092441306F7
:103710000032896541010283797106D622D41307EC
:103720008008F337078093F787083EC20100010045
:10373000B7170040930570052380B704130680FA7D
:103740002380C7040100010083C6F70293F6A60F89
:10375000A387D702238007049246F3A606800100C0
:10376000010073370780137787083AC4010001000E
:103770002380B7042380C7040100010003C7F702B8
:1037800013672700A387E70223800704A247F3A754
:103790000780010001000545EFE0CFFCE13E014755
:1037A00081468147054685451305407EEFE07F80D1
:1037B00037E404003C446800514681458297B707CE
:1037C000C0A83EC8B787E803938707D03ECA97F7DB
:1037D000FF1F9387C7BD3EC67C5868008297B250D2
:1037E00022544561828041119775010093854551AE
:1037F00017750100130545D906C6EF50614A1775C4
:1038000001001305656AEF50A149B2402945410105
:103810006F50414D4111977501009385A54F177564
:103820000100130565D606C6EF50814717750100E4
:1038300013054566EF50C146B240294541016F501E
:10384000614A411122C406C6834705002A849DC3EC
:10385000977501009385C551177501001305C5D2F1
:10386000EF5001444C401775010013052578EF50C7
:1038700021431DA058411DE7977501009385454FD1
:1038800017750100130545D0EF50814117750100F0
:1038900013054577EF50C1402244B240294541010C
:1038A0006F504144A1679386D7036311D702977580
:1038B00001009385E54B177501001305E5CCEF502A
:1038C000213E177501001305E574E9B7ED079775FB
:1038D00001009385E549177501001305E5CA6319D1
:1038E000F700EF50E13B177501001305E5735DB775
:1038F000EF50013B4C40177501001305E57485BF7F
:103900004111977501009385254217750100130534
:10391000A5C706C6EF50C138B240294541016F50D6
:10392000613C797122D426D24AD02E842A898145DD
:10393000B2844800714606D6EFE02FC397F7FF1F09
:103940009387076BDC4783D70700231421012313D8
:10395000F100EF20F0029547A305F1009307401F07
:103960003EC6FD572305A100230AF100EF20901366
:103970002686A2854800EF209003B250225492542C
:10398000025945618280970700202392079C970780
:103990000020238D079AB7E70400BC47411106C6F3
:1039A000414681451385413D8297EF109067EF10A6
:1039B00010450145EF30801503C7C1259307F00A74
:1039C000631BF7009307F00889451385C125239EE3
:1039D000F124EF300040EF30E04F8145370504001F
:1039E0009707002023A0079697070020239A0794A3
:1039F000970700202387079497070020239F0792AB
:103A000097070020239A079297070020239907928F
:103A100097070020239A0792EF2000380145EF30E6
:103A20000042977501009385A532177501001305B3
:103A3000A5B5EF50E1261775010013052567EF5076
:103A40002126B240294541016F50C129411122C4AC
:103A500006C626C293F715002E84638D070C814697
:103A600017F6FF1F13064656854517050020035518
:103A7000658CEF80B00A05C5977501009385052E0A
:103A800017750100130545B0EF508121177501002E
:103A9000130585CFEF50C1202945EF50A12497751C
:103AA00001009385A52B177501001305E5ADEF50B7
:103AB000211F17750100130565CEEF50611E2945C2
:103AC000EF50412217F5FF1F130585525C4505474E
:103AD0002390E700EFF0E01A977501009385052821
:103AE00017750100130545AAEF50811B17750100DA
:103AF000130505CCEF50C11A2945EF50A11E9307BD
:103B000010F8238EF1249707002083D76782A38EB5
:103B1000F1241385C125A1839145238FF124A38F1F
:103B20000124EF30002B13451400B240224492448C
:103B30004101828093F72500D1CB1707002003575E
:103B4000278051C397F6FF1F9386C67F94429777CD
:103B500001009387A75717F6FF1F0346867E81450E
:103B60001385413DEF40D008AA8431CD97750100FF
:103B70009385852517750100130505A1EF504112A6
:103B8000A68517750100130525C4EF50611129455D
:103B9000EF50411597F7FF1F2394077A930710F80A
:103BA000238EF12497F7FF1F83D78778A38EF12404
:103BB000A183238FF12491458D471385C125A38FC0
:103BC000F124EF3000211345240085B793F7450019
:103BD000B1CF977501009385251F17750100130557
:103BE000A59AEF50E10B177501001305A5BFEF5023
:103BF000210B2945EF50010F930720F8238EF12464
:103C000097F7FF1F83D76773A38EF124A183238FB8
:103C1000F1248547A38FF124EF20C0681385C125C7
:103C20009145EF30001B1345440001B793F7850021
:103C30008DCF977501009385251917750100130520
:103C4000A594EF50E105177501001305E5BAEF5093
:103C500021052945EF50010997F7FF1F2392076EB1
:103C6000EF40F00513458400C9B593F70501A5C3DE
:103C7000854517F5FF1F0355456CEF00B14F97754C
:103C8000010093856514177501001305E58FEF504A
:103C9000210117750100130565B7EF506100294533
:103CA000EF504104930730F8238EF12497F7FF1F5C
:103CB00083D7A768A38EF1241385C125A1838D45E1
:103CC000238FF124EF30E01013450401B9BD93F7C1
:103CD0000502B5C3977501009385050F177501009F
:103CE0001305858AEF40D17B17750100130545B494
:103CF000EF40117B2945EF40F17E930740F8238E7A
:103D0000F12497F7FF1F83D72763A38EF124A183A4
:103D1000238FF1248547A38FF12497F7FF1F239D5D
:103D20000760EF2020581385C1259145EF30600AC8
:103D300013450402DDBB93F70504CDC79775010059
:103D4000938585081775010013050584EF405175AB
:103D500017750100130545AFEF4091742945EF40F9
:103D6000717883C7C1251307700A6388E7041307B6
:103D7000800A6386E7061307600A6397E7029307E2
:103D800060F8238EF12497F7FF1F83D7475BA38E3C
:103D9000F124A183238FF1248547A383F126B14524
:103DA0001385C125EF30E002EF20C04F1345040416
:103DB00097F7FF1F239507588DBB930770F8238E45
:103DC000F12497F7FF1F83D78757A38EF124A18390
:103DD000238FF1248547A380F1269945D1B7930716
:103DE00080F8F1BF93F705080145E38007D4977584
:103DF0000100938565FD176501001305E578EF4027
:103E0000316A177501001305A5A5EF4071692945B1
:103E1000EF40516D9307A0F8238EF12497F7FF1F11
:103E200083D78752A38EF124A183238FF124854762
:103E3000A38FF12497F7FF1F23980750EF208046A8
:103E40001385C1259145EF20D07813450408F1B9B9
:103E5000411122C4977501009385C5F22A84176524
:103E600001001305657206C6EF4091634C4017755B
:103E7000010013052515EF40B1622945EF40916619
:103E8000034704009307F00F6319F70297750100C9
:103E9000938545EF176501001305056FEF405160ED
:103EA0004C40177501001305E512EF40715F224485
:103EB000B240294541016F40F162B24022444101C4
:103EC000828085CD411122C4176501001305C56BA1
:103ED0002E84977501009385E5E506C6EF40515C99
:103EE000A285177501001305251AEF40715B224466
:103EF000B240294541016F40F15E8280411122C4E8
:103F000026C22E84AA8497750100938565E3176500
:103F100001001305656706C6EF409158177501004B
:103F200013054517EF40D1572945EF40B15B977511
:103F300001009385E5E097F7FF1F239D973E1765E6
:103F4000010013056564854497F7FF1F2392873EA0
:103F500097F7FF1F239F973C97F7FF1F2399873EF3
:103F6000EF40115497F5FF1F83D5653E177501008B
:103F70001305C512EF40D1522945EF40B15697F7CE
:103F8000FF1F2385973CEF1080672285EF201038B4
:103F90000545EF20D06A97F7FF1F93876705DC4739
:103FA00003D70700C167FD176312F7022244B7E782
:103FB0000400B240924403A3870517F5FF1F034591
:103FC00065361306000A854541010283B24022444A
:103FD000924441018280011122CC37E404005C5CF0
:103FE00006CE26CA354697750100938525ED1775CF
:103FF000010013056579829701E917650100130532
:10400000255DEF40B15E01A097F7FF1F93874765DD
:104010003EC4B7F507008567938707C0814617F64A
:10402000FF1F13066630E10519453EC697E0FF1FE6
:10403000E780604D7C44194697F5FF1F9385C52E98
:10404000138581368297340017F6FF1F1306C62D9D
:104050009775010093850531177501001305053229
:10406000EF408011AA8415C9977501009385C5D4C6
:104070001765010013054551EF409142A68517755C
:1040800001001305A5E4EF40B1412945EF409145FA
:10409000F2406244D24405618280EFA06028177527
:1040A00001001305A5D9EF30C02CEF70A016EF006A
:1040B000313517F5FF1F130565F0EF001122177555
:1040C00001001305A5D8EF007135AA84EF30700701
:1040D000EFC0805AEF20D154EF409023EF30B0660C
:1040E000EFE0703797750100938505CD17650100E6
:1040F0001305854989C8EF40B13AA68517750100B7
:10410000130505DF49B7EF40B139177501001305F5
:1041100065E0EF40F1382945EF40D13CEFE0101A5F
:10412000EFB040446305050E854537050400EF10E8
:10413000B04697750100938525C8176501001305E2
:10414000A544EF40F13517750100130525DEEF405A
:1041500031352945EF40113997F7FF1F938787D9EC
:1041600083D7070017F7FF1F2313F71E854717F79D
:10417000FF1F230DF71CEF10C065EF10404817F527
:10418000FF1F0355C51CEF20701897F7FF1F83C74B
:10419000D71BB9EFA303010083274417130671004F
:1041A0008545130550308297977501009385C5C0EA
:1041B000176501001305453DEF40912E177501006D
:1041C000130505D9EF40D12D2945EF40B131977541
:1041D0000100938565BE176501001305E53AEF40C0
:1041E000312C177501001305A5DCEF40712B71BD53
:1041F00097750100938545BC176501001305C53807
:10420000EF40112A17750100130505D865BF977592
:104210000100938565BA176501001305E536EF4087
:10422000312817750100130565E8EF40712729450E
:10423000EF40512B0145EF20904051BF411122C466
:1042400037E404008327041A06C68297EF20D014AF
:104250008327040817F5FFFF1305857F829797F7DB
:10426000FF1F2381A70C17F5FF1F130565D8EF204B
:1042700040302244B2404101B9BB411122C49146B1
:104280002A84138601349D652D4506C697E0FF1FDD
:10429000E7806027B7F7070003C70701A547631347
:1042A000F70001A09306001001469D65254597E0A3
:1042B000FF1FE7804025238081342244B24091468D
:1042C000138601349D652945410117E3FF1F6700EF
:1042D0008323B7E704001171FC47CED79389C1252A
:1042E000A2DDCAD986DFA6DB2E8432892E86AA8576
:1042F0004E85829783C70900130780029387E707DB
:1043000093F7F70F636AF774176701001307C72F56
:104310008A07BA979C43BA9782878D4797750100A1
:104320009385C5AB1765010013050526630BF400E3
:10433000EF4011171765010013050569EF4051168D
:10434000FDA2EF40F1151765010013056569EF4007
:1043500031152945EF401119930720F8114693852F
:10436000C1254A85238EF124A38F0124EFF06FDB52
:104370002A840DC597750100938545A61765010030
:1043800013058520EF40D111A285176501001305A3
:10439000E568EF40F1102945EF40D1149775010011
:1043A0009385C5A3176501001305051EEF40510F46
:1043B000176501001305C567EF40910E2945EF40D1
:1043C00071124165930730FA05469385C1257D1525
:1043D000238EF124EFF0EFD42A840DC597750100E8
:1043E0009385C59F176501001305051AEF40510B12
:1043F000A2851765010013056562EF40710A294522
:10440000EF40510EB7E70400BC4F0566130606C81F
:10441000A14517F5FF1F0345E5F08297FE506E5446
:10442000DE544E59BE591161828091476301F402F6
:10443000977501009385859A176501001305C514CA
:10444000EF401106176501001305C561C5BDB7E74B
:104450000400FC4F914517F5FF1F0345A5EC82971B
:104460009775010093858597176501001305C511A0
:10447000EF4011031765010013058560EF405102FD
:104480002945EF403106EF10F0619145E1A28547E3
:104490006301F40297750100938545941765010047
:1044A0001305850EEF40C17F176501001305C55E3A
:1044B00071B597F7FF1F239227E9B7E70400056658
:1044C000BC4F130606C8C145A9B78D476301F40266
:1044D0009775010093858590176501001305C50A3E
:1044E000EF40017C176501001305C55C81BD930792
:1044F00040F811469385C1254A85238EF124A38F68
:104500000124EFF00FC22A84E30A05F09775010039
:104510009385C58C1765010013050507EF404178A9
:10452000A285176501001305654FEF4061772945A6
:10453000EF40417BE5B59147E31CF4F8B7E7040091
:10454000FC4F9305000217F5FF1F0345A5DD829779
:104550009775010093858588176501001305C502CD
:10456000EF400174176501001305455601BF8947E7
:1045700063E1870297750100938545861765010001
:1045800013058500EF40C1711765010013054555FE
:1045900075B383C4E12583C7D12597750100938541
:1045A000E583A20417650100130505FEDD8CEF40CD
:1045B000216FA285176501001305C553EF40416EB9
:1045C000C2042945EF400172C1849305D4FF93963C
:1045D0000401C1824A8693F5F50F1385F125EF108A
:1045E000207FE35D90E2930750F8238EF12483C788
:1045F000390022869385C12585074A85A38FF1243A
:10460000EFF02FB22A84E30B05E097650100938554
:10461000E57C17650100130525F7EF406168A28569
:1046200017750100130545A509B7894763E187029E
:10463000976501009385857A176501001305C5F418
:10464000EF400166176501001305854CC5B9EF10F1
:104650007045A2851385C125EF20A077C1B38D4792
:104660006301F402976501009385457717650100A2
:10467000130585F1EF40C162176501001305054B75
:1046800075B9B76602000146B7750200054597E0A7
:10469000FF1FE78040E7930760F8238EF124A38F84
:1046A00001249307002623A0F126E57793870721AD
:1046B0002392F1263146A383A1269385C1254A85FD
:1046C00023830126EFF0EFA52A84E30905D497653B
:1046D00001009385A570176501001305E5EAEF4019
:1046E000215CA285176501001305C5453DBDB14795
:1046F0006301F402976501009385456E176501001B
:10470000130585E8EF40C1591765010013054545BC
:1047100035B1B7E70400FC4F9305000417F5FF1F00
:10472000034545C08297EF10F037B14525B7914753
:1047300063E18702976501009385456A176501006B
:10474000130585E4EF40C1551765010013050543C6
:10475000F5B683C4012683C7F125A204DD8C8E043F
:10476000B77702006D14BE942286A68517650100F6
:1047700013050542EF40C152B7E70400FC4722860B
:10478000938511262800829793160401C182300078
:10479000A685094597E0FF1FE780E0D62A8419C562
:1047A0001765010013058540EF404164930770F8D9
:1047B00019469385C1254A85238EF124A38081263D
:1047C000EFF02F962A84E30B05C4976501009385CB
:1047D000E56017650100130525DBEF40614CA285FC
:1047E000176501001305853D89B399476301F410EE
:1047F000976501009385855E176501001305C5D88F
:10480000EF40014A176501001305C53C05BE9147FD
:1048100063E18702976501009385455C1765010098
:10482000130585D6EF40C147176501001305053C08
:1048300031B683C4012683C7F125A204DD8C8E0422
:10484000B77702006D14BE942286A6851765010015
:104850001305053BEF40C144B7E70400FC4722863F
:10486000938511262800829793160401C182300097
:10487000A6850D4597E0FF1FE780E0C82A8419C58B
:104880001765010013058539EF404156930780F8FD
:1048900019469385C1254A85238EF124A38081265C
:1048A000EFF02F882A84E30B05B697650100938506
:1048B000E55217650100130525CDEF40613EA28545
:1048C000176501001305C5368DB199476301F402E0
:1048D0009765010093858550176501001305C5CACA
:1048E000EF40013C176501001305053681BCB7E7B1
:1048F0000400FC4F9305000417F5FF1F034585A234
:104900008297EF10301A9945B1B38D476301F402D5
:10491000976501009385854C176501001305C5C691
:10492000EF400138176501001305853301BC176599
:1049300001001305E533EF40614B1305C01297E00A
:10494000FF1FE780409F0145EFE02FA60D45EFF0E8
:10495000DF92294597E0FF1FE780E09D97E0FF1F6A
:10496000E780008F65BC99476301F40297650100F9
:104970009385C54617650100130505C1EF40413217
:10498000176501001305852F55BA03C7112683C784
:10499000012622075D8F9166BA96C2061166C18212
:1049A0001306F6EF8D476363D60297E7FF1F9387E1
:1049B00027649C4B03C6F1259386C70039C603D6EE
:1049C00007005DCA8907E39CD7FE89471307A0F853
:1049D00011469385C1254A85238EE124A38FF124B6
:1049E000EFE03FF42A84E30B05A29765010093856D
:1049F000E53E17650100130525B9EF40612AA28540
:104A0000176501001305C5280DB603D6070063021C
:104A1000E60A8907E39BF6FE8D474DBF9147630287
:104A2000F402976501009385653B17650100130546
:104A3000A5B5EF40E126176501001305E5266FF0E7
:104A4000FF8FB7E70400FC4F9305000817F5FF1F21
:104A50000345458D829705BC976501009385053810
:104A600017650100130545B2EF408123176501006A
:104A7000130505256FF09F8C2390E70017E5FF1FB6
:104A800013050557EFE080219765010093850535F3
:104A900017650100130545AFEF4081201765010040
:104AA00013050523EF40C11F2945EF40A12381478E
:104AB00031BF2390070017E5FF1F13056553EFE093
:104AC000E01D9765010093856531176501001305A9
:104AD000A5ABEF40E11C176501001305E520D9B730
:104AE000411122C406C6834705002A849DC39765E9
:104AF00001009385652A176501001305E5A8EF40BD
:104B0000211A4C40176501001305455DEF4041191E
:104B100075A05841B707CF009387777D6313F706D9
:104B20009765010093854527176501001305C5A505
:104B3000EF4001171C448356E4008355C40003C6AC
:104B40000700176501001305E55AEF406115294577
:104B5000EF4041190357E40097E7FF1F83D7277FF2
:104B60006307F7008355C4000844EFE0CF9703566E
:104B7000E4008355C40008442244B24041016FF070
:104B80004FF5B707CC009387777D631FF7029765D2
:104B9000010093856520176501001305E59EEF4030
:104BA00021101C448356E4008355C40003C607004B
:104BB0001765010013050554EF40810E2244B240F1
:104BC000294541016F400112B707CE009387777DD9
:104BD0006302F702976501009385051C17650100C4
:104BE0001305859AEF40C10B4C4017650100130572
:104BF000A54529BFB2402244410182805171CAD1EA
:104C000037E904008327C904A2D52E8686D7A6D308
:104C10002E84AA851385C125829783C7C1251307D2
:104C2000700A638DE70C636CF7001307600A6382F8
:104C3000E704BE502E549E540E596D6182801307B6
:104C4000800A6382E7121307900AE394E7FE8D4718
:104C5000630BF416976501009385051A176501002B
:104C600013058592EF40C10317650100130505AFD9
:104C700015A08D476306F402976501009385C5175B
:104C80001765010013054590EF408101176501008C
:104C9000130505A6EF40C1002945EF40A10451BF0F
:104CA000854717650100130565A617E7FF1F230752
:104CB000F768EF40A113B7750200B766020001461E
:104CC000054597E0FF1FE7800084930760F8238E77
:104CD000F124A38F01249307002623A0F126E57772
:104CE000938707212392F126B14523830126A383CD
:104CF000A1261385C125EF20C00D25BF914763E193
:104D00008702976501009385250F1765010013053C
:104D1000A587EF30F17817650100130525A19DBF28
:104D200083C4012683C7F125A204DD8C8327C9042F
:104D30006D14228693851126280082978E0493167F
:104D40000401B7750200C1823000A695094597D0CD
:104D5000FF1FE780407B930770F8238EF12499456D
:104D6000A380A12679B7914763E187029765010087
:104D7000938585081765010013050581EF30517291
:104D8000176501001305059C31B783C4012683C74D
:104D9000F125A204DD8C8327C9046D142286938536
:104DA0001126280082978E0493160401B77502001D
:104DB000C1823000A6950D4597D0FF1FE780A074F3
:104DC000930780F859BF176501001305659AEF40F6
:104DD000E1011305C01297D0FF1FE780C0550145C0
:104DE000EFD0BFDC0D45EFF04FC9294597D0FF1F2D
:104DF000E780605497D0FF1FE78080451DBDB7E76F
:104E000004004111FC4726C29384C1252E8606C6A4
:104E100022C44AC02E842A89AA852685829797654E
:104E20000100938525FF175501001305E575EF3047
:104E3000316783C5C125176501001305E5A3EF3070
:104E400031662945EF30116A83C7040041479387D3
:104E5000070693F7F70F6365F74817670100130715
:104E6000E7848A07BA979C43BA9782879D47630372
:104E7000F402976501009385E5F9175501001305C4
:104E8000A570EF30F161176501001305659FEF30E4
:104E90003161D1A283C7D125ADCF83D7012603D7F6
:104EA000E125C207D98F17E7FF1F232DF74883C7D6
:104EB0006400976501009385E5F51755010013051A
:104EC000A56C17E7FF1F230EF746EF30715D97E7DC
:104ED000FF1F938727478C4317E6FF1F034666464D
:104EE000176501001305859BEF30915B2945EF3075
:104EF000715FA38E01242244B24092440249930779
:104F000000F8238EF1249D451385C12541016F10C2
:104F1000506CEF306066239FA124935705012A84CB
:104F20002380F126935785010145A380F126EF30B8
:104F300060652381A126976501009385A5ED17552E
:104F4000010013056564EF30B15503C62126A28523
:104F5000176501001305059641BFCD476301F402B3
:104F600097650100938505EB175501001305C56191
:104F7000EF301153176501001305459509BF37E45C
:104F800004007C4441469385D1251385413D829799
:104F90001385413DEF00407D9D2583C7E12603C772
:104FA000D126A20703238405D98F17E7FF1F2319F2
:104FB000F7381306000A89452244B2409244024958
:104FC00017E5FF1F03450536410102838D47630145
:104FD000F402976501009385E5E317550100130579
:104FE000A55AEF30F14B176501001305E59D45B556
:104FF00003C4E12583C7D12597650100938585E129
:10500000220417550100130525585D8CEF305149D6
:10501000A285176501001305E58CEF30714829451D
:10502000EF30514C0D469385C1252285EFE07F8FEF
:10503000AA8415C9976501009385C5DD1755010040
:1050400013058554EF30D145A6851765010013057A
:10505000A58AEF30F1442244B240924402492945E6
:1050600041016F30314897E7FF1F2398872CB7E73E
:105070000400116603A38705130606E891452DBFBA
:105080008D476301F402976501009385A5D81755F4
:1050900001001305654FEF30B1401765010013059E
:1050A00065A1F5B303C4E12583C7D1259765010048
:1050B000938545D62204175501001305E54C5D8CF8
:1050C000EF30113EA2851765010013052584EF30EE
:1050D000313D2945EF3011410D469385C12522858B
:1050E000EFE03F84AA840DC197650100938585D2C6
:1050F0001755010013054549EF30913AA68517650C
:1051000001001305E581B1B797E7FF1F23968722BA
:10511000B7E70400116603A38705130606E89305A5
:10512000000259BD894763E18702976501009385B5
:1051300065CE1755010013052545EF30713617650B
:1051400001001305E599A1B383C4E12583C7D125E7
:1051500097650100938505CCA2041755010013053E
:10516000A542DD8CEF30D133A6851755010013051C
:10517000A57CEF30F1322945EF30D1362286938578
:10518000C1252685EFE0EFF92A84630A05169765A5
:105190000100938525C8175501001305E53EEF3042
:1051A0003130A285175501001305457A5DB5854755
:1051B00063F78714834519002244B24092440249A0
:1051C000B335B00097E7FF1F238AB71617550100C4
:1051D0001305057941016F30B12CA2852244B240FC
:1051E00092444A85024941016FF05FA199476301EA
:1051F000F402976501009385E5C117550100130579
:10520000A538EF30F12917650100130525A741B135
:1052100003C4E12583C7D12597650100938585BF28
:10522000220417550100130525365D8CEF305127F8
:10523000A2851755010013052574EF307126294505
:10524000EF30512A19469385C1252285EFE06FED95
:10525000AA840DC1976501009385C5BB1755010050
:1052600013058532EF30D123A685175501001305AC
:10527000A571C5B397E7FF1F2398870CB7E7040014
:10528000116603A38705130606E8930500082DB3EE
:105290008547976501009385E5B71755010013050C
:1052A000A52E6309F400EF30B11F17550100130557
:1052B000E56EF1BEEF30D11E175501001305856F65
:1052C000EF30111E2945EF30F1212244B2409244C3
:1052D000024997E7FF1F2395070641016F30201E03
:1052E00097650100938505B3175501001305C5297E
:1052F000EF30111B176501001305859C49BEB240B4
:1053000022449244024941018280411106C622C4CE
:10531000EFE02FE19377F50F95CB2A849765010095
:105320009385C5B01755010013050526EF305117B9
:105330009375F40F17650100130505D4EF3051166E
:105340002244B240294541016F30D119B240224474
:105350004101828001114EC697E6FF1F83D626FFCA
:10536000B28917E6FF1F035666F726CA4AC806CE5B
:1053700022CCAA842E891D2397E7FF1F83C707FD30
:10538000A9CB03C4440083C734001765010013058B
:10539000A5DA22045D8CEF30B1104A86A6852285FD
:1053A000AD37638F090297E7FF1F83C707FA8DCBDD
:1053B0006308090297E7FF1F83C747F895E3624434
:1053C000F240B249CA8526854249D24405616F1030
:1053D0005020176501001305A5D6EF303121D1B754
:1053E000F2406244D2444249B24905618280834717
:1053F000550083454500176501001305A5D2A20796
:10540000DD8D6F30F109176501001305A5D06F30F0
:10541000F11D8D4763F2B70A011126CA06CE22CCD0
:105420000344350097E4FF1F83C434F297650100FD
:105430009385C5D1B337800017E7FF1FA307F7F0A7
:1054400009C497650100938525D1176501001305EF
:1054500025D1EF30F10497E7FF1F83C717EF638370
:105460009700252C97E7FF1F83C737EE9DC385471D
:105470002306F100B7E7040083A7471770008545AE
:1054800013055030829717650100130565CEEF3084
:10549000F1159967938757EE2316F1006800854749
:1054A0009145A30781002307F100EF109012F2400D
:1054B0006244D244056182808280894763F2B708E2
:1054C000011122CC06CE26CA8344250085472A84B2
:1054D0006398F404914763F0B7040345450083479C
:1054E000340022055D8D97E7FF1F2399A7DE1D2954
:1054F0009967938767EE2314F100834734002305EF
:105500009100A305F1008347440095452800230638
:10551000F100EF10100CF2406244D2440561828029
:10552000FDF89967938767EE2314F10097E7FF1F53
:1055300083D7C7DAA305F10023050100A183F1B7E2
:1055400082800111996722CCD51717E4FF1F13043D
:10555000E4DF2314F1008347040026CA97E4FF1F09
:105560009384E4DE2305F10083D7040028009545E9
:10557000A305F100A18306CE2306F100EF1070050C
:1055800003D6040083450400176501001305C5BF59
:10559000EF300171F2406244D244056182809D6720
:1055A0007971D9172316F10097E7FF1F83C707DA30
:1055B00006D62307F1009DCBB7E70400FC47414620
:1055C0009385413D1305F10082976800CD45EF10AA
:1055D000500097E5FF1F83C565D7176501001305C8
:1055E000A5BDEF30E16BB25045618280B7E70400A2
:1055F000BC47414681451305F1008297F9B7B7676B
:1056000002036971938757AA3EC4856793872790E1
:105610002316F10097E7FF1F938747D383C707003F
:1056200023248112A30701002307F10097E7FF1F3E
:105630009387E7D183D7070037E4040023261112AC
:105640002318F10097E7FF1F938747C983D7070007
:10565000414648082319F1007C449385413D8297D7
:10566000F1452800E52A2312A1027C442C002810D1
:10567000794682973C44130561041306900D8145D9
:10568000829730109305700F0145EFD09FB48320AF
:10569000C1120324811255618280B7C7A55A011136
:1056A0009387C7333EC497E7FF1F83C717CA3EC619
:1056B000B7F7070003C7070106CE22CCA54763133F
:1056C000F70001A01164930504F093060010014651
:1056D000254597D0FF1FE78000E33000930504F0D5
:1056E000A146294597D0FF1FE780E0E197E5FF1F1E
:1056F00083C5B5C5176501001305C5BCEF30415A18
:10570000F24062440561828001119165A14630003A
:10571000938505F02D4506CE97D0FF1FE780A0DECC
:105720002247B7C7A55A9387C7336312F702B2451A
:1057300017650100130545ACB335B00097E7FF1FAF
:10574000A385B7C0EF30C155F24005618280814525
:1057500017650100130585AC97E7FF1FA38707BEF8
:10576000EF3001541D3FCDB7B7C7A55A7971938764
:10577000F7353EC6B7E70400FC47AA8506D622D413
:10578000414608088297B7F7070003C70701A547F6
:105790006313F70001A01164930504E89306001059
:1057A0000146254597D0FF1FE780E0D5700093059F
:1057B00004E8D146294597D0FF1FE780C0D417657C
:1057C00001001305E5B3EF306162B2502254456128
:1057D000828079719165D1467000938505E82D45E9
:1057E00006D697D0FF1FE78000D23247B7C7A55A29
:1057F0009387F73517650100130545AA631EF70067
:10580000B7E70400FC471385413D41460C088297E9
:1058100017650100130585A6EF30415DB250456163
:105820008280B7F7070003C70701A5476313F70096
:1058300001A091654111930600100146938505E88A
:10584000254506C697D0FF1FE780E0CBB24017651D
:1058500001001305A59841016F304159C167697670
:105860008146FD1705061397060141836364B7005F
:105870003E8582803307D50003470700B98F214753
:1058800013F81700858363050800B18FC207C18331
:105890007D171377F70F6DF78506F1B749C1A54757
:1058A000054763FFB70683471500034705003168C6
:1058B000A207D98F13978700A183D98FC207C1830D
:1058C0001308C8550547639D0705411106C622C444
:1058D00026C203442500914763FD870293075400C5
:1058E0006399F502A301C50021822302C500930438
:1058F000340091C6A302D500A1822303D5002A84D7
:10590000A685A93F26942300A4002181A300A4001A
:105910000147B240224492443A85410182800547C2
:105920003A858280B7C7A55A01119387E7343EC4F0
:105930002AC6B7F7070003C7070106CE22CC26CA3E
:10594000A5476313F70001A091642A84938504EEB0
:10595000930600100146254597D0FF1FE780A0BAA7
:105960003000A146938504EE294597D0FF1FE780BC
:1059700080B9A285176501001305C596EF30413245
:10598000EFF0FFC7F2406244D2440561828001110A
:105990009165A1463000938505EE2D4506CE97D042
:1059A000FF1FE78040B62247B7C7A55A9387E73461
:1059B0006314F702B245176501001305258897E7C0
:1059C000FF1F239DB790C205C181EF30612DEFF01D
:1059D0001FC3F24005618280D147D14517650100A0
:1059E0001305C58717E7FF1F231AF78EEF30412BEA
:1059F00017E5FF1F0355858E3537E1BF011126CA14
:105A000006CE22CC93F71500AE848DCBAD67371749
:105A100000409387A7AA1CC3B7E70400BC4F130636
:105A20000019854517E5FF1F0345258B829713C590
:105A30001400F2406244D2440561828093F725004D
:105A400063850712976501009385858F2D46480071
:105A5000EF30A11997E5FF1F83C5558F854793C484
:105A6000240063E1B70489CD97E7FF1F83C7E78D63
:105A700085C38545170500201305C5F7EF10603570
:105A80001395040197E7FF1FA382078C418155B747
:105A900041650546970500209385C5F57D15EFF016
:105AA000DF86F9BF170400200344C4F497070020E1
:105AB00083C757F422045D8CAD67C2059387B75541
:105AC000C1816306F40863E68702A9679387A75537
:105AD0006306F40897E7FF1F83C727878DE74165B3
:105AE0002E867D15970500209385C5F0EFF0FF8188
:105AF000B9A0B1679387C755630EF400B567938764
:105B0000D755E319F4FC170500201305A5EEEF1097
:105B1000402C35A00546170500201305A5EDEFF034
:105B20007F8397E7FF1F83C7678291EB4800EF30C1
:105B3000213493150501C1814800EFD0CF9AA28589
:105B4000175501001305C57DEF30811515BF1705E9
:105B50000020130525EAEFF09F89D5B7170500202F
:105B6000130545E9EFF03F8AD9BF93F7450001459A
:105B7000E38107EC175501001305C57BEF300127C2
:105B8000EF10003713C544006DB5411122C437E44E
:105B900004005C5C06C635469755010093850532C6
:105BA00017650100130545BE829701E917550100ED
:105BB0001305C579EF30812301A08327041C829748
:105BC0002A840545EF802075EF10C168EF1001476A
:105BD000EF70B0292285B2402244410182801567CE
:105BE000B71700401307575598C3D8439D66558F84
:105BF000D8C3D843FD76758FD8C3D8431367F70F42
:105C0000D8C335671307C7CC98C3828041111305E9
:105C1000800406C622C426C24AC097C0FF1FE78080
:105C2000004985457D55EFC09FDF85457D55EFC017
:105C30007FE9371400408327840A8D45130500202F
:105C400093E707202324F40AEFC07FDDB7E40400C4
:105C5000EFD0EF8EC8581309840C1304C40CEF3036
:105C6000E11817650100130525B2EF3021188327CD
:105C7000C4FF8545414593E70708232EF4FEEFC096
:105C80007FE48D4513050008EFC0DFE3EFC05FFE42
:105C90000145EFD00F8185450545894717D7FF1F7F
:105CA0002308F76AEFD08F8137070004B7E700E0D9
:105CB00023A0E710EFD07F8EEFD0FFA1F935EFF0F2
:105CC000BFA4EFF0DFCCEFE06FD78D450D65EFC0DF
:105CD0007FDF170500201305E5E185671CC589678F
:105CE0002320250140C12326250100C95CC983A7C3
:105CF000841E829783A7040817050000130545D06A
:105D0000829797D7FF1F238AA75CBC4C13060064B9
:105D100085458297E93597C0FF1FE780606C014594
:105D20008280B7F7070003C70701A547AE86631651
:105D3000F7009397450191C301A0AA850146254527
:105D400017C3FF1F6700237C4111B2862E86AA85E8
:105D50002D4506C697C0FF1FE780E07AB240014597
:105D6000410182809307000463E6C7021D71A2CC43
:105D70002A84080886CE32C6EF203167B246100862
:105D8000A285294597C0FF1FE780E077F64066446B
:105D90002561828039558280411126C2AE848D45AD
:105DA00022C406C62A84EFC0FFD1B717004099C8A5
:105DB00003A5C70C418D23A6A70CB24022449244F0
:105DC0004101828003A5870C418D23A4A70CF5B760
:105DD0008347050003471500A207D98FC2076177E3
:105DE000C187130727206397E70083452500370500
:105DF00004005DB7828097D7FF1F9387A75518428D
:105E00009C4383D645000345070083C5C70003565E
:105E100046006396A50083D5E700638DD502011186
:105E200006CE2386A7002397D700B705CF00DC4B0B
:105E30009385757D05077D162EC2230001003AC4A7
:105E40002316C1002317D10099C30A858297F24017
:105E5000056182808280DC4DDC4B81CFB7E7040096
:105E6000904503A38705914517D5FF1F0345C54EF0
:105E7000028382806D713C083EC6B707E50023228D
:105E800091103EC8AA843C083285232611103ECAD0
:105E900023248110232021112E89EF2090672A844A
:105EA000975501009385C552174501001305C56D2F
:105EB000EF20115FA2851755010013056561EF20E2
:105EC000315E2945EF201162B705CB009385757DC2
:105ED0006800EF10A043A2856800EF203059014709
:105EE00081467000CA852685EF10C06215C52A84D8
:105EF000975501009385C54D174501001305C568E9
:105F0000EF20115AA285175501001305255DEF20DA
:105F100031592945EF20115D8320C11003248110E0
:105F200083244110032901105161828097D7FF1FFC
:105F30009387474218429C43797122D406D603487E
:105F4000070083C807012A8483D64500035546000D
:105F50006396080183D82701638DD802238807013F
:105F600005072399D7003708CC00DC4B1308787D50
:105F70003ACC1307F5FF42CA23080100231EE100B3
:105F8000231FD10099C7080832C62EC48297324613
:105F9000A2452285C535B2502254456182806D717B
:105FA0003C083EC0B707E5003EC23C083EC423267D
:105FB000111023248110232291102317010023188C
:105FC000010023190100231A0100231B010097D7A8
:105FD000FF1F83D7E70599E3C167FD172316F1007B
:105FE00097D7FF1F83D7E70491EB97D7FF1F9387BE
:105FF00067369C439C43DC4783D7070017D4FF1FB9
:1060000013040403584C2317F10083574400484BF2
:106010002318F10005ED975501009385654217455A
:10602000010013056556EF20B14717550100130510
:106030006542EF20F1462945EF20D14A8320C11067
:1060400003248110832441105161828097D7FF1F60
:1060500083C777FE89EBB7E70400BC5782975C4C97
:1060600023AA0700E1BFFD1797D6FF1FA385F6FC03
:1060700003560701834704014C470A85230BF100AF
:10608000EF20F03C97D7FF1F9387C72C9C43014715
:10609000814688430A866C00EF10C047AA841DC958
:1060A000975501009385C539174501001305C54D66
:1060B000EF20113FA685175501001305653AEF2023
:1060C000313E2945EF201142584CB7E70400BC5738
:1060D000484B69B797D7FF1F83C7F7F5F5D7B7E7E1
:1060E0000400BC4F1044854517D5FF1F0345C52646
:1060F0008297A9B75C4EDC4BA9CBA1C9411122C440
:1061000017450100130545482E84975501009385D6
:10611000653106C6EF20D138A28517550100130559
:106120006536EF20F1372945EF20D13BB7E7040072
:106130002244B24003A3870517D5FF1F0345C5219D
:10614000130640069145410102838280411122C419
:1061500017D4FF1F1304C4EB1C4C06C689C7DC43CD
:1061600099C34C488297584CB7E70400BC57484B3A
:1061700082975C4CB240224423AA070041018280EE
:1061800017D7FF1F1307A715834707009306F00BC8
:10619000850793F7F70F63E9F60097D6FF1F238073
:1061A000F614034507008280930700F8FDB7835774
:1061B00045006386070E01114AC817D9FF1F13094E
:1061C00029E752C4032AC90106CE22CC03274A017B
:1061D00026CA4EC656C2F15721EF1307D00DFD5700
:1061E0006368C704B7E9040083A709072A84130575
:1061F000860042054181B284AE8A8297232AAA0092
:106200000325C9015C499DEF975501009385851FC2
:106210001745010013054537EF2091281755010058
:106220001305852EEF20D1272945EF20B12BDD570F
:10623000F2406244D2444249B249224A924A3E85DF
:106240000561828093874400B705CF002319F500CC
:106250009385757D3105EF10600B0325C9018345DA
:1062600064003105EF2090200325C9012686D685DC
:106270003105EF20D01D7146A2854A85EF20F11629
:10628000504419CA83A78905854517D5FF1F0345C3
:10629000A50C8297814769BFEFF07FD0E5BFFD571E
:1062A0003E858280411126C297D4FF1F938444D833
:1062B000D84C22C437E404003C54484B06C68297AD
:1062C000DC4C0323C4052244B240924423AA0700B5
:1062D00017D5FF1F0345450885454101028341113C
:1062E00026C297D4FF1F9384E4069C4006C622C4AE
:1062F0004AC0C9CBDC43D9C75CC12300B5002A849E
:10630000975501009385450B174501001305C527D7
:10631000EF2011192945EF20F11C9C4023A4070010
:1063200023A2070097D7FF1F938787CEDC4FDC4B54
:1063300081C72955EFF09FE197D7FF1F938747CF7C
:10634000DC4FDC4B91C3B93F37E904008327C90513
:10635000894517D5FF1F0345250082978327C90567
:10636000914517D5FF1F034525FF82979C4003A346
:1063700047016309030022852244B2409244024946
:1063800041010283B2402244924402494101828089
:106390000111328506CE22CC26CA2E84EF2070173A
:1063A000AA849755010093856504174501001305DC
:1063B000A51DEF20F10E03078400035664008355EA
:1063C0004400A686175501001305C50DEF20510D99
:1063D0002945EF20311197D7FF1F83C7C7C36398A3
:1063E00097000145EFF09FD681450A85CD3DF240EB
:1063F0006244D244056182806D712324811023267A
:1064000011102322911093F745002E846385071203
:106410003C083EC0B707E5003EC23C083EC4231717
:1064200001002318010023190100231A0100231B76
:10643000010097D7FF1F83D7A7BD99E3C167FD1759
:106440002316F10097D7FF1F83D7A7BC91EB97D7EF
:10645000FF1F938727F09C439C43DC4783D70700AB
:1064600017D7FF1F1307C7BA2317F100544F8357DD
:1064700047002318F100DC4A95EF975501009385FA
:1064800025FB1745010013052510EF207101175555
:106490000100130525FCEF20B1002945EF209104F0
:1064A000134544008320C11003248110832441102C
:1064B0005161828097D7FF1F83C7F7B52555ADCBB4
:1064C000FD1717D6FF1FA308F6B403D606018347AE
:1064D0000701CC460A85230BF100EF20407797D7C0
:1064E000FF1F938727E79C4317D7FF1F130747B268
:1064F00097660100938686C888430A866C00EF1071
:106500006001AA8451DD97550100938565F2174516
:10651000010013056507EF20A178A6851755010036
:10652000130505F4EF20C1772945EF20A17B2685CF
:10653000EFF0DFC1B5B793F725009DC3B7E70400BF
:10654000BC4741468145280882972555EFF01FC07A
:1065500028089305F00FEFF09FD81345240099B752
:1065600093F7150001459DDFEFF07FA3134514005D
:1065700015BF5C4D411106C688C317D7FF1F232BDB
:10658000F7DCB7E7040083A7070817050000130529
:10659000E5E68297B24097D7FF1F238FA7DA014520
:1065A0004101828001119307700F2316F10006CE7E
:1065B00097D7FF1F83C717DB8DE7B7E7040083A7D3
:1065C000870D17D6FF1F0346E6D16C0017D5FF1FB6
:1065D000035585D982973335A00097D7FF1FA38332
:1065E000A7D8F2400561828041119397050122C42A
:1065F00006C626C2C1872E8463D40702B7E404000E
:10660000FC5417D5FF1F0345E5CD829719C1BC5433
:1066100082972165218DB2402244924441018280BB
:1066200093F715008DC7B7E7040083A7471A17D65D
:10663000FF1F1306E6A197F5FF1F9385A55017D5F9
:10664000FF1F034525CA829713451400E9B793F746
:10665000250099CFB7E70400BC4F130600648945B5
:1066600017D5FF1F034505C882971345240065B75A
:1066700093F785009DC7B7E7040003A8871A13079F
:10668000401F97D7FF1F83C7E7C581461306400603
:10669000994517D5FF1F035525CD02981345840052
:1066A0009DBF93F745000145BDD7B7E4040083A71C
:1066B000041817D5FF1F035525CB8297BC4C130632
:1066C0000064914517D5FF1F0345C5C18297134547
:1066D000440091B797D7FF1F83D707C96396A702D6
:1066E00017D7FF1F2313B7C817D7FF1F2310C7C81B
:1066F00017D7FF1F231DD7C62E8617550100130578
:1067000065F6BE856F20C15917550100130505F7C1
:106710006F20C16D03574500011106CE22CC97D7DB
:10672000FF1F83D767C417550100130525F56310B4
:10673000F706C167F91717D7FF1F2327F7C237E4FA
:10674000040097D7FF1F23A307C27C4C894517D5A8
:10675000FF1F034525B982977C4C914517D5FF1F34
:10676000034545B8829797D7FF1F83C717BE95C7C4
:106770008547A307F100832744171306F1008545D9
:10678000130550308297175501001305A5E4EF203B
:10679000E165F24062440561828097D7FF1F83C79D
:1067A000E7BA175501001305A5E7F5F38547A307D9
:1067B000F100832744171306F10085451305503077
:1067C000829717550100130525E3D1B77D1595472D
:1067D00063E0A71A17570100130787DC0A053A95EB
:1067E0001C41011122CC06CE26CABA972E8482877C
:1067F00017550100130505E9EF20415F0DA203C7FE
:1068000025009947631DF7002E85EFF0BFF0834503
:106810006400175501001305E5E7EF20614897D79D
:10682000FF1F238407B217550100130565E8E9B778
:1068300003C7250095476317F702C16717D7FF1FE6
:10684000035787B2F91703D5A5006307F702B7E727
:10685000040083A7C717829717550100130545E663
:10686000EF20C158854717D7FF1F2300F7AE1755F4
:106870000100130565E749B797D7FF1F2396A7AE19
:1068800083D7E500B7E40400096617D7FF1F231E6E
:10689000F7AC83D705011306069017D5FF1F0345F4
:1068A00065A417D7FF1F2313F7AC83D72501A14594
:1068B00017D7FF1F231DF7AABC4C8297BC4C1306A9
:1068C0000064914517D5FF1F0345C5A18297035664
:1068D000E4008355A400175501001305A5DFEF2040
:1068E000213C49B7175501001305C5E031B783C5F1
:1068F00025009147639AF502854717550100130556
:10690000E5E0A307F100EF20614EB7E7040083A79D
:1069100047171306F1008545130550308297F24062
:106920006244D244056182809947639EF5002285C6
:10693000EFF05FDE8345640017550100130585D530
:10694000EF200136E9BF9547639FF50083471400A8
:1069500017550100130585DBE39007EA1755010081
:10696000130585DC51BD17550100130565DCC9BF52
:1069700082806D712324811023261110232291100F
:10698000328401CD89476306F5028320C1100324B8
:106990008110832441105161828017550100130535
:1069A000E5D9AE84EF208144A2852685EFE02FC58E
:1069B000E9BFB7E70400FC4728008297175501009C
:1069C000130585D8EF2081428347810039C0130722
:1069D000000B638EE7001387A7051377F70F8D462B
:1069E00063E9E602A2852800EFE04FA179BF854761
:1069F000E3FD87F88345910017450100130545F62F
:106A0000B335B00097D7FF1F238AB792EF204129F3
:106A1000ADBF03479100A207D98F35671307D7553C
:106A2000638DE7066366F7022D671307B755638129
:106A3000E70631671307C7556386E704296713071D
:106A4000A7556392E702A2852800EFE0DF9B35BFE0
:106A500039679306E7656383D70663E9F600130792
:106A6000E7556388E704A285280089B73D67930648
:106A7000F755638AD7041307F766E396E7FEEFE05E
:106A80001FB221B70146A2852800EFE0BF8CF5BDFB
:106A9000A2852800EFE0BF95CDBD8947E3F787EEDB
:106AA0009305E4FFC205C1811305A100EFC0AFA3A8
:106AB000E9BDA2852800EFE0DF95C1BDA2852800D1
:106AC000EFE0BF9FD9B5EFE0DFA7C1B5411122C408
:106AD00017C4FF1F13048459AA8617560100130612
:106AE000A6AD2285C14506C6EF20413103574400BB
:106AF00097C7FF1F938787582393E70003576400C6
:106B00002394E700B240224441018280011106CE65
:106B100022CC6D3F37E404008327841417C6FF1F7F
:106B20001306C654D54501458297832784179305DC
:106B3000F1001305503082978347F100A1C7A307E6
:106B40000100832744171306F100854513055030D3
:106B500082978327441717C6FF1F13062652CD4579
:106B60001305703082978547A307F10083274417E8
:106B70001306F1008545130550308297F2406244B8
:106B8000056182808327441717C6FF1F1306064F2F
:106B9000CD4513057030D5B7130101DE232C8120BC
:106BA00037E4040083270408232E1120232A912090
:106BB000232821212326312117050000130505A3D1
:106BC000829717C9FF1F1309E9719947854423006C
:106BD000A9002318F100975501009385E5A69307B6
:106BE0004006174501001305259A2314F1102304CC
:106BF000910097C9FF1F93898975EF20610A83D59A
:106C00000900175501001305E59BEF20610929458F
:106C1000EF20410D03D50900EFF05FEB8327441708
:106C2000300085451305503082978327441717C6D7
:106C3000FF1F1306A644CD451305703082978327A6
:106C4000441717C6FF1F13066641B545130560308C
:106C500082978327441710088945130510318297BE
:106C600083274417300289451305203182978327F3
:106C70004415930500320D458297832744159305EB
:106C8000003211458297A301910023029100230451
:106C90009100232401102308010083278416300269
:106CA000914513057040829783278416130631009F
:106CB000854513050040829783278416500085453B
:106CC0001305104082978327841610088545130505
:106CD0002040829783278416300085451305504055
:106CE0008297832704157D558297832744137D550A
:106CF00082977D55EFC0CFC68327440C8297EFC0A3
:106D00000FA48327841417C6FF1F13062636D54504
:106D10000145829789471306700F814508082302B1
:106D2000F100EFB08F848D471306700F8145280264
:106D30002308F100EFB06F8391472304F11097C748
:106D4000FF1F9387A75A984383C747003AC4230677
:106D5000F100EFE0DF8A500085450545EFC06FC7C1
:106D600010089305700F0945EFC0AFC630029305B8
:106D7000700F0D45EFC0EFC5300095451145EFC0D0
:106D80004FC5C16717C7FF1F1307075EF9171CC35D
:106D90002322070017C5FF1F13058554EFC04FC2FC
:106DA0008327C41D17C5FF1F1305455B82973C4809
:106DB00003450900854582978320C1210324812151
:106DC00083244121032901218329C12013010122A8
:106DD00082800111C16726CA06CEAA8422CC17C5BB
:106DE000FF1F03556558F9176306F50437E40400DF
:106DF000832784122E862315B10001478146ED4575
:106E000082977C440356A1002AC6A68582972C004F
:106E100017C5FF1F03554555EFC04FC701CD175587
:106E2000010013056583EF10717C8327C412ED45C3
:106E300028008297F2406244D244056182800111A9
:106E400006CE22CC2DC9854717C7FF1FA30DF720FB
:106E500097C7FF1F238A072037E40400832784177E
:106E60009305F1001305503082978347F100A9CBB9
:106E7000A3070100832744171306F1008545130576
:106E8000503082978327441717C6FF1F1306061D2D
:106E9000B5451305603082978547A307F100832726
:106EA00044171306F1008545130550308297F240D0
:106EB00062440561828097C7FF1FA386071A49BFF6
:106EC0008327441717C6FF1F13064619B545130538
:106ED0006030E9BFC16717C5FF1F0355E548F917C3
:106EE0006307F500B7E7040003A3C7170283828096
:106EF00001118547A307010017C7FF1F2304F746A9
:106F0000B7E7040083A7471706CE1306F1008545AF
:106F1000130550308297F24005618280EFA25FE056
:106F20002A8408452E89B28909C900C19705000045
:106F30009385C5746105EF00810181447D5AEF108E
:106F4000C00963C3A4048144EF10200A63C6A404EB
:106F500097F7FF1F9387C7BF9C43DC47B307F940F0
:106F600091872302F400638109048327C900B307D2
:106F7000F4409587A302F4001C4C89C79C4799C331
:106F8000228582976FA01FDD5C441397140085044F
:106F9000BA972390470165B71C48139714008504DE
:106FA000BA97239007004DB7832789000547B30799
:106FB000F4409587A302F40083570400638EE70230
:106FC0008DC309476384E7040D47E397E7FA9757B2
:106FD0000100938727CA1CCC97570100938787CA63
:106FE00011A897570100938767901CCC9757010011
:106FF0009387C7905CC849B7974701009387077C80
:107000001CCC974701009387677CEDB79757010029
:10701000938707CB1CCC97570100938767CBD9BFC9
:1070200085E1EFA29FD10046184483479400758301
:107030009D8B6315F700EF00501C48C46FA03FD232
:107040008280EFA2FFCD13893500C164420941114E
:10705000AA890144F11413590901054A2EC6EF000B
:10706000D077B2456346A400014541016FA09FCE91
:1070700083A7090013171400BA9783D70700638802
:10708000B7006394970063742A010504C1BF0545E6
:10709000E9BFEFA21FC8AA892E89328BB6843A8A2B
:1070A000BE8AEF80204C55C12685EF1030368D47C3
:1070B00063E5A7007D556FA05FC983DB4400EF0047
:1070C000D0772A84EF00B0789307740031443305F9
:1070D000850263C5A702EF005076EF0010762A8480
:1070E000EF00F0769307740031443305850263CDD9
:1070F000A702EF0090749307450019A8EF003075C0
:10710000330585021307F0179307C017E357A7FC51
:107110002D55E3C277FB63000B02D6865286A68507
:107120004A85EFE0106341BFEF00707233058502BE
:107130009307C5FFF1BF832749001385C90083D595
:107140002700EFF01FF071F9B5B76955ADB797F7A4
:10715000FF1F2391A7A097F7FF1F9387679F904377
:1071600081470C463307F500420741836393B7001C
:1071700082805446139847008507C2962390E60004
:10718000D5B797F7FF1F9387A79C9C4303C587003C
:10719000828017F5FF1F0355E59B8280EFA2FFB9A0
:1071A000C1671387D7FF6307E5026368A700F1177C
:1071B000630EF50001456FA09FBA1387E7FF630ECA
:1071C000E500FD171D8D13351500F5B7EF40003DA7
:1071D0007D15D5BFEF40801AE5BFEF40E018CDBF69
:1071E000EFA2BFB54111AA8401442EC6EF00F05FA3
:1071F000B2456346A400014541016FA05FB69C48BB
:10720000131514003E9583570500E387B7FE050468
:10721000E9BF03485500814693F7F60F63E5070180
:1072200081473E858280584593975600BA9703D789
:1072300027006316B70003D70700E304C7FE8506DF
:10724000E1BF8346450001479377F70F63E4D7001A
:10725000814711A81C45131657000507B29703D69E
:107260000700E313B6FE3E858280EFA27FAB931743
:107270000501C18797FAFF1F938A8A8D6355F0082D
:1072800083A70A00C0479C4703570400198D420595
:1072900041816366F500014422856FA0BFAB1205F2
:1072A0002A94DDBFDC4713944900014A3E9483478A
:1072B00044006341FA02014A834754006347FA02DB
:1072C0008509C20993D9090183A70A009847E3EB0E
:1072D000E9FCD1B71C4413195A00A6853E994A858A
:1072E000EFF01FF011ED050AD9B75C4413195A00ED
:1072F000A6853E994A85EFF0BFEE19E1050A6DBFFC
:10730000E30009FC51BFAA8481497DBFEFA2FFA21F
:107310001C452A8481E79307C5001CC51C44231221
:1073200004001CC09307F00F63E9B70093F5F50F55
:107330002285EF10B0136FA09FA293940501C1673F
:10734000C18063F7F500A6852285EF10D015E5B75B
:10735000C18193F5F50F2285EF105011A685228586
:10736000EF101012C9BF97E7FF1F9387677E88430E
:1073700082801C4599C797E7FF1F23ABA77C014577
:1073800082807D55828097E7FF1F9387677C9843B3
:1073900083474500484792073E958280EFA2FF99B8
:1073A000617100451C183EC6B70780013EC81C1815
:1073B0003ECA8357440002CE02D002CC231EF10005
:1073C000834784002A8902D22301F1023C083ED47B
:1073D00002D6EFF05FFB835705002316F102EF3072
:1073E000706B2307A1025C4003556400F18313F71F
:1073F00017008347F10252055181F99BD98FA307EA
:10740000F102EFE0702639C5AA8403550500EF802C
:10741000401683D704002AD26800231CF10083D7CA
:107420002400231DF1001C4803D647008C43EF10B5
:1074300010028347B400CA8617460100130686313E
:107440008117A305F4006C004810EFE090305D61F7
:107450006FA0FF902155E5BF1C45B1CF03C5A70024
:10746000894613576500630BD7028D46630ED7021A
:1074700085466300D702130740063305E50203C7BC
:10748000B700418B15CB83C7B700BD8B3355F54093
:1074900082801375F5031307803EC5B7096713751E
:1074A000F50313070771D1BF372709001375F503DB
:1074B0001307077CD9B701458280EFA21F8803A973
:1074C0008500630509048347B900AE8493F7070E6E
:1074D00091CF03459900930520030D810505B30560
:1074E000B50288446105EFF0B0320DA02E85EFF0B3
:1074F000BFF62A8401CD11238325C900B307B54007
:1075000063F887002E94B305A440E1FD6FA03F858A
:107510008545C1BFEFA27F822A8403D505000111F2
:1075200032C636C43AC22EC002CA02CC02CEEF80A6
:10753000400482452ACA22852ECCEFF0DFE40357AF
:107540000500231EE100EF30F054A2463246924778
:10755000230FA10036874C08B28622850146EFF042
:107560005FB305616FA0AFFFEFA22FFD61711C1823
:107570003EC6B70780013EC81C183ECA3C080045FD
:107580003ED4AA8402CC02CE02D002D202D6EFF0C0
:107590009FDF8357050035592316F102EF30904FD6
:1075A0002307A10209C48357440091E721594A8562
:1075B0005D616FA0CFFA0355640052055181EFE081
:1075C000B00A2A8965D58347B40093F7070E89C7A7
:1075D00013058401EFF0502583574400231EF1006A
:1075E000834784002301F1025C4003550900D983DD
:1075F00013F7070883471102231CA10093F7F7072D
:10760000D98FA300F10283572900231DF1005C40AC
:10761000F18313F717008347F102F99BD98FA30772
:10762000F102EF7010752AD251D18347940068009F
:10763000139757008347B400FD8BD98FA305F4003F
:107640001C4803D647008C43EF106060A68717479D
:10765000010013072710740005464C102685EFF033
:107660005FA32A8929D58347B400A685FD8BA3058E
:10767000F400EFF09FE425BFEFA22FEC832485FEFA
:107680002A8441112685EFF03FDD834734FF93F7CD
:10769000070E9DC32AC62685EFF05FD019C9834720
:1076A00034FFB245FD8BA309F4FE81C52285EFF0BE
:1076B000301641016FA0AFEA6DDD8327C4FF268538
:1076C000829765F9834734FF93F7070E81C72285B8
:1076D000EFF09015032584FEEFF01FE9D9BFEFA26C
:1076E000CFE29C4141112A8903C7070089472E84B4
:1076F00093566700638CF6020D466382C6049307B7
:10770000F0076302F7022E85EF10A060AA8481497A
:10771000C16B130C490097E7FF1F938767439C4396
:10772000984763ECE90241016FA0EFE103D7450000
:107730008547E3FAE7FE2E85EF108061C1BF03D7CE
:107740004500E3F2E7FE2E85EF10A05CAA842285B7
:10775000EF10805DC204C98C5DBFDC470355A900F2
:10776000139A49003E9A93170501C187635DF000A3
:1077700083570A006395A70263E574038327CA0051
:10778000034D5A001DA0A1672167A98F1307F7EFCA
:10779000E374F7FE63950900EFF05FA071FD8509C2
:1077A0009DBF83278A00034D4A00835DA9000357CC
:1077B0006900216A138BC7003AC6814A33CA4D015A
:1077C000631E5D0197E7FF1F938707399C43E1DB49
:1077D000A2866286814526858297D1B7A167938765
:1077E000F7EF930C4BFF63F04703B2455A85EFF078
:1077F0005F8519CD03278B00104719CA104363809A
:10780000C4023107D5BFEE856685EFF07F9D71FD1F
:1078100093861A0093FAF60F130B0B0255B7835693
:1078200044005C43E3EDF6F622853AC6EF10603D76
:10783000A1679387D7042A8A035D4400324763E82F
:1078400097008347D90093E707F8A306F9001C4780
:1078500066852286E2858297C1670844FD17337AE0
:10786000FA00529508C02312A40115BF97E7FF1F25
:107870009387072E9843814715C31447814763FFB9
:10788000D500939745004C47BE9519C903C75500CD
:1078900081476375E600DC451606B2973E85828017
:1078A00003C745008147E37BE6FE16069C45F5B716
:1078B000EFA20FC7AA892E8A814497EAFF1F938AF5
:1078C0002A2983A70A00984763E4E4006FA08FC8C1
:1078D000DC471394440001493E9413BB14008347D2
:1078E0004400634BF900014913BB14008347540063
:1078F000634FF9008504F1B7084493175900528784
:10790000DA860146A2853E9582990509C9BF484499
:10791000931759005287DA860546A2853E958299CB
:107920000509E9B7EFA26FC1814517F5FFFF130500
:10793000255F97E7FF1F239F0720EFF07FF76FA0DA
:107940000FC297E7FF1F9387A7209C4381CFEFA229
:10795000CFBE814517F5FFFF1305855CEFF05FF59E
:107960006FA0EFBF8280EFA2AFBB37E40400832794
:10797000841241112315E100AE893289368A3A8694
:1079800081460147ED45AA8482972AC621C5035640
:10799000A100D285EF1061258327C413CE852685EB
:1079A0008297058915C58327440D231421010146BB
:1079B0002C00268582972A8401C9B7E7040083A793
:1079C000C712ED4528008297228541016FA08FB82C
:1079D0004944E5B76554CDBF5C41FD175CC1828069
:1079E000EFA2AFB5B7E70400FC5F82979547330578
:1079F000F50281450D816FA08FB6EFA20FB4B7E7F6
:107A00000400FC5F829795473305F5020D816FA056
:107A10000FB5EFA28FB2B7E7040083A7870B03551A
:107A2000050082976FA0AFB3EFA22FB103550500F9
:107A30003287AE8617B6FF1F0356666A97E5FF1FAB
:107A40009385C511EFF03FF26FA06FB1EFA2EFAEDB
:107A5000B7E7040083A7C71782976FA04FB0EFA2C4
:107A6000CFADB7E7040083A7871397E5FF1F938582
:107A7000E50E829701456FA08FAEEFA20FACB7E77E
:107A8000040083A7C71F814517B5FF1F0355256154
:107A900082976FA0CFACEFA24FAAB7E7040083A7ED
:107AA000871397E5FF1F9385650C829701456FA0AB
:107AB0000FABEFA28FA8B7E7040083A7C71F8145CC
:107AC00017B5FF1F0355A56382976FA04FA9EFA2BB
:107AD000CFA62E85EF600055EF60900D6FA02FA808
:107AE000EFA2AFA5EF60D0176FA06FA75C49E117B9
:107AF0005CC95CC583572501A1072319F50083578D
:107B00000501A1072318F5008280F1473305F5022E
:107B100097E7FF1F938787079C433E9582808D4799
:107B20006317F60603D74600854763F2E706EFA220
:107B3000CFA0368536842E89EF10A01D39C183571A
:107B4000440093140501C18063ED97022285EF1074
:107B5000401CFD14231294009307A002630EF5004D
:107B60009307B0026301F50293079002631BF500CF
:107B70002285EFC0B07E31A00146CA852285EF8004
:107B8000000F6FA0CF9D2285EF001059DDBF8280CE
:107B900097E6FF1F9386C6FF9C42014599CF984305
:107BA000D44217E6FF1F2325E6FE6396D70097E62B
:107BB000FF1F23A1E6FE1385C7FE8280EFA2EF9789
:107BC000E9267144330585029145EF70606201E555
:107BD00065556FA0CF9897E7FF1F23A7A7FA7526D3
:107BE000330585029145EF70A0607DD197E7FF1FB7
:107BF00023AEA7F8592E97E7FF1F2391A7F8712608
:107C000097E7FF1F239DA7F6974701009387C7B902
:107C100017E7FF1F2328F7F697070000938747ED24
:107C200017E7FF1F232EF7F4014565B7EFA2EF908A
:107C3000AA8517E5FF1F130565F4EF1060216FA0FB
:107C40000F92EFA28F8FEFF07FFEEF10E02197E70A
:107C5000FF1F9387E7F39C4381CF1387C7FE09CBB0
:107C600083D5C7FF17E5FF1F130505F3EFF0403A73
:107C70006FA0EF8EEFA26F8CEFF09FF119C98347D1
:107C800085002A8493F7070499E70355E500EFF090
:107C90005FFB6FA0CF8C8347C5009304450117E9B4
:107CA000FF1F1309E9EE85E3832709005CC997E705
:107CB000FF1F23AF97EC83274900E1FF97E7FF1FE2
:107CC00023AA97ECF9B7FD172306F5006105EF60CD
:107CD000E07E8307840063CB07048347840093E737
:107CE00007F82304F400B7E704009C5F829742057D
:107CF000A94741813375F5028347840093F707FC58
:107D0000C98F2304F4008347D4003E951C402318F8
:107D1000A40089CF984319CB8347C40050408145C4
:107D200085073305F5024205418102978327090043
:107D30005CC897E7FF1F23AD97E48327490089E7D5
:107D400097E7FF1F23A897E48347C400B9D383555F
:107D5000040117E5FF1F130525E4EFF0602B15BFA5
:107D6000EF92BFFD97E7FF1F938747089C470144A9
:107D70008583858B81EFAE84B2853A86EF1020141F
:107D80002A8409C5EF10200B829408CC22856F90BD
:107D90001FFDEF92FFF841112E8932C6AA89712C7E
:107DA000324713060502CA8697050000938525D63B
:107DB00017E5FF1F130585DCEFF09FFA2A8429CD14
:107DC0009304C50065261946AA852685EF0030680C
:107DD00085452685EF001065174501001305859A36
:107DE0004E95834505002685EF0050685C48314676
:107DF0008145A1075CC85CC483572401E11723199E
:107E0000F40083570401E1172318F4001C4C3E854D
:107E1000EF90BFF5A3042501228541016F909FF3E8
:107E2000EF92BFF14111AA842EC632C4EF100003B5
:107E3000004DB2452246834784000CC050C093F7E2
:107E4000F70393E707042304F400231804002685AE
:107E5000EF00707E83479400A9462317A40013D730
:107E6000370005073307D7029D8B85072306F400EB
:107E7000A306E40083C70401D8488507230FF7FE53
:107E800017E7FF1F1307C7D05843232A040093079F
:107E900044011DEB17E7FF1F232EF7CE17E7FF1F47
:107EA0002328F7CE17E4FF1F130404CF2285EFF039
:107EB000A00B1C44858B5D8D09E581452285EFF083
:107EC000201541016F90BFE91CC317E7FF1F232353
:107ED000F7CCC9BFEF927FE697050000938565C494
:107EE0000145EFF0DFBE01456F907FE7EF92FFE4C1
:107EF000EFF01FBF6F90BFE68347C500A1E7EF9289
:107F0000DFE32A840355E500EFF05FD215C983470C
:107F1000840093F7F7FB2304F4001C4091C7DC4373
:107F200081C74C4001458297EFF09FC617E5FF1FC0
:107F3000130585C6EFF0400F0355E400EFF07FD046
:107F40006F90FFE18280EF925FDF97E7FF1F9387DB
:107F500027C497050000938525D217E5FF1F130559
:107F6000A5C323A0070023A20700EFE0507E6F9077
:107F70001FDF1C4D91CBDC4381CBEF921FDC83458F
:107F8000070082976F90BFDD828097E7FF1F93877E
:107F9000E7C29C4303C50700828097E7FF1F9387D2
:107FA000E7C19C4303C51700828097E7FF1F9387B3
:107FB000E7C09C4303C52700828097E7FF1F938794
:107FC000E7BF9C4303C54700828097E7FF1F938765
:107FD000E7BE9C4303C53700828097E7FF1F938766
:107FE000E7BD9C4303C55700828097E7FF1F938737
:107FF000E7BC9C4303C56700828097E7FF1F938718
:10800000E7BB9C4303C57700828097E7FF1F9387F8
:10801000E7BA9C4303C58700828097E7FF1F9387D9
:10802000E7B99C4303C59700828097E7FF1F9387BA
:10803000E7B89C4303C5A700828097E7FF1F93879B
:10804000E7B79C4303C5B70011E11D45828097E760
:10805000FF1F9387A7B69C4303C5C700828097E79D
:10806000FF1F9387A7B59C4303C5D700828097E77E
:10807000FF1F9387A7B49C4303C5E700828097E75F
:10808000FF1F9387A7B39C4303D50701828097E71F
:10809000FF1F9387A7B29C4303C52701828097E700
:1080A000FF1F9387A7B19C4303D54701828097E7C1
:1080B000FF1F9387A7B09C4303D56701828097E792
:1080C000FF1F9387A7AF9C4303D58701828097E763
:1080D000FF1F9387A7AE9C4303C5A701828097E744
:1080E000FF1F9387A7AD9C4303C5B701828097E725
:1080F000FF1F9387A7AC9C4303C5C701828097E706
:10810000FF1F9387A7AB9C4303C5D701828097E7E6
:10811000FF1F9387A7AA9C438857828097E7FF1F7A
:108120009387C7A99C4303D5C702828097E7FF1FA7
:108130009387C7A89C4303D5E70219E11305800C78
:10814000828097E7FF1F938767A79C4303C50703B8
:10815000828097E7FF1F938767A69C43C85B828056
:1081600097E7FF1F938707A58843828097E7FF1F44
:10817000938787A48843828019E17D558280F5DE4C
:10818000984265DFFDD917E7FF1F130727C6184779
:10819000AA877155058B6319072203C50700154788
:1081A000E37DA7FC03C737001305F0057D171377A0
:1081B000F70FE364E5FC03C35700E30003FC83C847
:1081C0006700E38C08FA03C77700494579171377EE
:1081D000F70FE364E5FA03C7A70011481305F7FF9B
:1081E0001375F50FE36BA8F803CE97000D48130540
:1081F000FEFF1375F50FE362A8F803C8B700630923
:10820000080065181378F80F1305600DE36705F78C
:1082100003C5C700794879151375F50FE36FA8F406
:1082200003C8D7000D457D181378F80FE36705F5EF
:1082300003D80701930E401751184208135808013C
:10824000E3ED0EF303C8E7007D181378F80FE3663B
:1082500005F303C827017D181378F80FE36F05F1C4
:1082600003C88700C54E75181378F80FE3E70EF1C1
:1082700003D86701856E938EBEE06D1842081358CF
:108280000801E3EC0EEF03D847016D1842081358BC
:108290000801E3E40EEF03D8870179184208135868
:1082A0000801E36C05ED03C8A7017D181378F80FEA
:1082B000E36505ED03C5B7011D487D151375F50F81
:1082C000E36DA8EA03C5D701714879151375F50F59
:1082D000E365A8EA03D5E7011308E00F7D15420521
:1082E0004181E36CA8E803C5070249487915137575
:1082F000F50FE364A8E8C85301C937C8340059151D
:10830000130858BFE36BA8E603A8870237C53400FB
:10831000130555BF5918E36205E717E5FF1F232D25
:10832000C58803C6050117E5FF1F2329F588054504
:10833000E375C5E403D82501D04933760603E31E6F
:1083400006E203C61501E30A06E217E6FF1F232330
:10835000B68683C5270001466387A50003C61700BC
:10836000F1453306B60283C707039305C00272972F
:108370001A071307C70516031A9796084697B38777
:10838000B70241553E97329742074183636EE80238
:10839000EF92BF9A3685EF60D06FEFD0B0212A847C
:1083A000EF80B01D2A94EFC090252A94EF7040070B
:1083B0002A94EFF0BF802A94EF2050632A94EF5064
:1083C000406622956F90BF998280EF921F9741116E
:1083D000A307A100EF80801E9305F10017050000A0
:1083E000130565B9EFF0CFCC014541016F903F9780
:1083F000EF923F9217E4FF1F1304449F0328840069
:1084000079599368180097E4FF1F23A5149F1378E8
:108410001800631E0800BA84BE89368B328A2E8902
:10842000AA8AEFE01FD67D15269509E531594A85C0
:108430006F90BF91EFE0FFD47D152695A167E357BC
:10844000F5FE97E7FF1F938767D198433E8C814BDA
:1084500011C70145EFC0B03E933B15004A85DA864F
:108460005686D285EF7070372A8911CD1C44F99B4E
:1084700017E7FF1F2320F79883270C00CDDBE38845
:108480000BFA82976DB7268597E7FF1F23A2079601
:10849000EFE0FFCB4146CE8517E5FF1F1305859E14
:1084A000EF00A174EFA070080325040BEFA0700A81
:1084B0000545EFA070100545EFF03FF18DBF97E740
:1084C000FF1F9387A7929C47858BD5C7EF92FF86A6
:1084D00017E5FF1F1305459997E7FF1F23A807908E
:1084E00097E7FF1F23A6079097E7FF1F23A4079096
:1084F000EFE09033EF40C002EFE0F00AEFE0700FE2
:1085000097E7FF1F9387078D9C4381C70545EF6061
:10851000B03397D7FF1F9387A7759C4389C74165E1
:108520007D15EF50A06BEFC0703AEFA0F00097E719
:10853000FF1F9387A7A09C4313971701635407005D
:10854000EFC0A04597E7FF1F23AE079297E7FF1FF5
:1085500023AC079297E7FF1F23AA079297E7FF1F15
:1085600023A80792EFF09F984923EFF0AFBBEFC02D
:1085700080676F90CFFE828097E7FF1F9387078702
:1085800088438280EF926FFBEF60B07EEF708000D7
:108590006F90EFFCEF92CFF82A849304140201113C
:1085A0002E85B289A685214636C63A89EF008161BB
:1085B0001DE1B24638082686CE8513059404EF40A7
:1085C000604321462C084A85EF00C15F1335150032
:1085D00005616F902FF80145E5BFEF920FF6930507
:1085E000450617D5FF1F1305A55DEFE070226F90BC
:1085F0000FF7EF928FF441112EC6EFF00FC0B24586
:1086000088C141016F90AFF5EF928FF1AA842E845B
:10861000EF605078AA8985452285892D83C7E401BA
:108620001389940899E313890403CE8522853D2D8F
:108630002146930519022285192D97D7FF1F93878D
:10864000E77A8C432285EF00E06821469385840217
:108650002285F52B6F900FF0EF92AFEB3971EFC0E1
:10866000E04E9305400645EDEF60D06F630E0510B8
:1086700097D7FF1F83C7875613B7170097D6FF1FDB
:10868000238EE654014489CFC16417D9FF1F130913
:10869000E9759309400EFD14EFF03F986348A40874
:1086A000EFF0AFB54169B7290900096AFD7A2A8B55
:1086B00081447D199389F97B130A0A71938A8AC7C9
:1086C000EFF0BF9563D5A4041304400EB387840272
:1086D00017D7FF1F130787710324070B3E94835797
:1086E000C4016386270918403307EB4063EAE900B9
:1086F000834744008507B3874703D6976369F70626
:10870000014681450945EFF0CFE8AA8B29E1EF202A
:10871000105A8547631FF50489659385057117D540
:10872000FF1F1305E549EFE0B00EA1A8B30734031E
:108730000327090BBA9703D7C7016308970003C73C
:108740005700A38207002382E7000504B1B7930511
:10875000C5002285EFF05FEB5E852286973501002C
:1087600093858503EFF0CFEB5E85EF00E06F850426
:1087700081BF97D7FF1F938767679C478D83858B42
:10878000C1FF21616F906FDC01468545094502D02C
:1087900002D202D402D6EFF0CFDFAA847DD1EFC09F
:1087A000203A1389C4002A8481454A85C1210C409E
:1087B00041464A85692983294400638809084E8512
:1087C00002D802DA02DC02DEEF00816A2ACE14103F
:1087D00005462C0808184ECCEF4060191375F50FAC
:1087E0002DE58355840093E525004A856D291146C2
:1087F0000C104A85A929014697350100938545FA51
:108800002685EFF0EFE12685EF0000665C40B5DBE2
:10881000014685450D45EFF0CFD7AA843DD14840AC
:108820001389C400EF00C1642AC64A85C5263246B2
:10883000636AC5004C404A85192901468145268551
:10884000EFF00FDE26850D252DBF8355840071BF07
:10885000EF92AFCE97D7FF1F938747599C4719CD0B
:1088600093E7870017D5FF1F1305853517D7FF1F1F
:108870002322F758EFE060786F906FCEDD9B17D71B
:10888000FF1F2329F756EF2090427DF517D5FF1FD4
:1088900013050533EFE04079C5B7EF928FC7416903
:1088A000AA892E8AB28A368BBA8B814417DCFF1FC5
:1088B000130CCC53930C400E7D19EFF00FF663C4EC
:1088C000A40001442DA03384940383270C0B3E9411
:1088D0008357C401638027055A87D6865286CE8582
:1088E00013050403EFF01FCB11C523800B00228575
:1088F0006F90AFC58347F40191CF5A87D6865286D1
:10890000CE8513059408EFF0FFC809C5854723807D
:10891000FB00F1BF850455B783574500638D0716EB
:10892000EF920FC001112A84ED2619C58547630A0D
:10893000F50405616F900FC2EFC040217DF98357A8
:1089400044004947ED9BE396E7FEC1452285452457
:10895000AA842285F52E0357440002CE91472A8926
:108960006317F700228539293C082ACC3ECEEFC098
:10897000201D5C55DDDF74084A86A6850545829773
:108980004DBF03574400D147E3F5E7FA032A04003B
:10899000C169014997DAFF1F938A4A45130B400EBC
:1089A000FD19EFF08FE76344A90C2285032A040028
:1089B0008D26A1452A8922851D2CAA842285D926A7
:1089C00014402A86AA8978082685CA85EFF0FFEC2C
:1089D000AA8425D103C7F40189476315F7008347AB
:1089E000C101A1DB5546D28513856400EF00E11F6C
:1089F0000145EF60103801C583D7C401B1EB97D7AB
:108A0000FF1F9387A73E9C4793551900858913D76D
:108A10003700058B11CB8983858B6397B7000145A0
:108A20002EC6EFF0FFE2B2454E85EF60703C034684
:108A3000C1012A84937519002685EF70703131C900
:108A40002685EF607037268511C00145EF60D06143
:108A5000EF20F0258547E31EF5EC83C7540013078C
:108A6000F00FE388E7EC8507A382F400D9B5B304DF
:108A7000690383A70A0BBE9483D7C40163893701B6
:108A80005546D28513856400EF00C11371D10509E5
:108A900009BF5DDC5DBF8280EF928FA8EF60902CF4
:108AA00011CDC164014417D9FF1F1309293493095B
:108AB000400EFD14EFF06FD6634AA40017D5FF1FD8
:108AC00013050510EFE060536F90CFA83305340312
:108AD0008327090B3E958357C501638697002312B0
:108AE0000500EF60702D0504F1B797D7FF1F93873E
:108AF000E72F9C478D83858B99EBEF920FA417D5B9
:108B0000FF1F1305E50BEFE020526F904FA5828009
:108B1000EF92AFA297050000938545B417D5FF1FCC
:108B20001305050AEFE0A0426F906FA3EF92EFA04C
:108B30008841B7E70400BC5B050542054181829787
:108B400009C585472300F50005056F904FA183C730
:108B5000F5FF2E858507A38FF5FE828083C7F5FF7D
:108B6000FD1793F7F70FA38FF5FE99EBEF92EF9CAC
:108B7000B7E70400BC571385F5FF82976F902F9ECF
:108B800082801C41035745008D8FBA951CC123126A
:108B9000B5003E85828093D78500A2051441DD8D06
:108BA000835745001387E6FF18C189072312F50094
:108BB00013D685004111238FB6FEA38FC6FE410157
:108BC000828018419307F7FF1CC183574500850732
:108BD0002312F500A30FB7FE8280835745008D8FC7
:108BE0002312F5001C41BE950CC12E858280AA87F8
:108BF00003D7470008410D8FAA952392E7008CC345
:108C00008280184108453305A7408280835745007C
:108C1000035765001D8F1C4108453385A740330568
:108C2000A7408280EF926F9141112EC62A84EFF007
:108C3000FFFDB2456373B50001A0835744000840AF
:108C4000BE952312B4003E9541016F904F91EF9273
:108C5000CF8E41112E84B28532C6EFF0BFFC324672
:108C6000A285EFF0907841016F906F8FEF92EF8CBB
:108C70002E848545EFF01FFB230085006F902F8E1B
:108C8000EF92AF8B41112317B1008945EFF09FF9A7
:108C90008347E1002300F5008347F100A300F500BE
:108CA00041016F90CF8BEF924F8993D78500A2053A
:108CB0004111DD8D2317B1008945EFF0BFF68347E1
:108CC000E1002300F5008347F100A300F500410116
:108CD0006F90EF88EF926F861397850193D7850188
:108CE000C166938606F0D98F13D78500758FD98F0B
:108CF000A2053707FF00F98D4111DD8D2EC6914584
:108D0000EFF05FF26C001146EFF0306E41016F90B2
:108D10000F85EF928F821C41854503C40700EFF059
:108D2000DFEB22856F90AF83EF922F811C414111C1
:108D3000894503C7070083C717002307E100A3077E
:108D4000F100EFF09FE90355E10041016F902F81A1
:108D5000EF82BFFE1C414111894503C7070083C74D
:108D600017002307E100A307F100EFF01FE7835787
:108D7000E100410113D58700A2075D8D42054181C5
:108D80006F80FFFDEF827FFB0C4141112A84114669
:108D90006800EFF0906591452285EFF01FE4B2473F
:108DA000C166938606F01397870113D58701598D05
:108DB00013D78700758F598DA2073707FF00F98FEA
:108DC0005D8D41016F80BFF91C45BE950CC182804D
:108DD000AE87944391E6584101EF0CC15CC182809B
:108DE00003C7570013671700A382E700B687D5B7FC
:108DF0000CC3EDB7AA87084119CD1841D44398C3D5
:108E00006313D500D8C32A8703465700937616000C
:108E100081E6232007008280944381CA8C4203A804
:108E200047008CC363930601CCC3799A14C3A30291
:108E3000C7003687D1BF1C45DC471D8DB777DBB631
:108E4000938777DB09853305F502420541818280EE
:108E5000F147B385F50248452E958280834745004A
:108E600085072302F5008280EF823FED2A8419E016
:108E70006F80FFEE83474400E5DFFD1793F7F70FA0
:108E80002302F400F5F71C4403D7270005072391BC
:108E9000E700DC4399C3228582974C4889CD8347FC
:108EA0005400898B99E71C4422859C479C439C472E
:108EB0008297232A04000040232004004DBFEF8244
:108EC000DFE78357250041112EC691E70144228533
:108ED00041016F80DFE8035705008147F146E30752
:108EE000F7FEB385D702404585072E94834544009D
:108EF00008C4F5F5B247AA8481E7232A040009A82B
:108F00001C456C0022859C439C43829748C85DDDCC
:108F100085472312F400B2472320040023180400DD
:108F20002319F4005C485CC483D72400FD17239107
:108F3000F40071BFEF827FE097D7FF1F938747CA86
:108F4000884323260500232405004105EFE0C00DDA
:108F50006F80FFE0EF827FDE17D4FF1F130444C849
:108F60001C40411189CF9C472300B5002AC65CC133
:108F7000EFF05FFC1C40DC4399C33245829741010E
:108F80006F80FFDD034745001DEB584DAA877D55D7
:108F90000DCBEF829FDA1CC3DC4797D6FF1F23A1BE
:108FA000E6C4F156130507012390D700970500008A
:108FB00093858501EFD0B07901456F805FDA7D55EB
:108FC00082808280EF827FD701116146814528002F
:108FD000EF80BFD997D7FF1F938787C09C43280096
:108FE0009305F00FDC473EC6EFF0DFF605616F80BA
:108FF0001FD797D7FF1F9387A7BE9C43D847A1676A
:109000009387C7026312F70A397106DE22DC26DA7B
:1090100080004AD84ED652D456D23285B284EFF070
:109020005FCFAA892685EFF03FD02318A4FC2685C0
:10903000EFF09FCF2319A4FC2685EFF0FFCE83D756
:1090400044000A8A231AA4FC858393F7F70F230EA2
:10905000F4FC8607BD0793F7073F3301F1408A8A86
:1090600001498347C4FD6365F902CE85130584FC7D
:10907000232C54FDEFF01FEE5281130104FCF2503B
:109080006254D2544259B259225A925A2161828072
:109090002685EFF07FC993171900D697050923900D
:1090A000A7001379F90F75BF828097D7FF1F9387A9
:1090B00027B39C43D847A1679387A7026310F70A99
:1090C000397106DE22DC26DA80004AD84ED652D428
:1090D00056D23285B284EFF0DFC3AA892685EFF03D
:1090E000BFC4FD572318A4FC26852319F4FCEFF018
:1090F000BFC383D744000A8A231AA4FC858393F74D
:10910000F70F230EF4FC8607BD0793F7073F3301E3
:10911000F1408A8A01498347C4FD6365F902CE851F
:10912000130584FC232C54FDEFF0DFE25281130180
:1091300004FCF2506254D2544259B259225A925A03
:10914000216182802685EFF03FBE93171900D697E4
:1091500005092390A7001379F90F75BF828097D76F
:10916000FF1F9387E7A79C43D847A1678907631828
:10917000F708397106DE22DC26DA80004AD84ED69E
:1091800052D456D232853289EFF0BFB8AA894A85C7
:10919000EFF09FB9835749000A8A2318A4FC8583FE
:1091A00093F7F70F230CF4FC8607BD0793F7073FEF
:1091B0003301F1408A8A8144834784FD63E5F402E8
:1091C000CE85130584FC232A54FDEFF0BFD85281CD
:1091D000130104FCF2506254D2544259B259225A3B
:1091E000925A216182804A85EFF01FB49397140050
:1091F000D69785042390A70093F4F40F75BF82805F
:1092000097D7FF1F9387C79D9C43D847A167938734
:10921000E7046312F70A397106DE22DC26DA8000E1
:109220004AD84ED652D456D23285B284EFF07FAEB1
:10923000AA892685EFF05FAF2318A4FC2685EFF0FE
:10924000BFAE231AA4FC2685EFF01FAE83D74400DF
:109250000A8A2319A4FC858393F7F70F230EF4FCE5
:109260008607BD0793F7073F3301F1408A8A01491A
:109270008347C4FD6365F902CE85130584FC232C66
:1092800054FDEFF03FCD5281130104FCF2506254C3
:10929000D2544259B259225A925A2161828026856B
:1092A000EFF09FA893171900D69705092390A70000
:1092B0001379F90F75BF828097D7FF1F9387479265
:1092C0009C43D847A1679387C7046310F70A397195
:1092D00006DE22DC26DA80004AD84ED652D456D298
:1092E0003285B284EFF0FFA2AA892685EFF0DFA3D2
:1092F000FD572318A4FC2685231AF4FCEFF0DFA207
:1093000083D744000A8A2319A4FC858393F7F70FB7
:10931000230EF4FC8607BD0793F7073F3301F140A6
:109320008A8A01498347C4FD6365F902CE85130526
:1093300084FC232C54FDEFF0FFC15281130104FC87
:10934000F2506254D2544259B259225A925A21616F
:1093500082802685EFF05F9D93171900D697050947
:109360002390A7001379F90F75BF828097D7FF1F4D
:10937000938707879C43D847A167DD07631BF702E4
:10938000EF82BF9B797132853284EFF09F982AC6B5
:109390002285EFF07F992311A1022285EFF07F97BC
:1093A000B2452300A1022808EFF0DFBA45616F80C3
:1093B0001F9B828097D7FF1F938787829C43D84744
:1093C000A16793878704631BF702EF821F97797168
:1093D00032853284EFF0FF932AC62285EFF0DF94C6
:1093E0002311A1022285EFF0DF92B2452300A102F2
:1093F0002808EFF03FB645616F807F96828097C75F
:10940000FF1F9387E77D9C43D847A1679387A704F5
:10941000631CF700EF827F92011128008145EFF075
:109420007FB305616F80BF93828097C7FF1F9387CB
:10943000277B9C43D847A167938757026311F702A4
:10944000EF82BF8F01113285EFF0BF8C2308A1009E
:1094500081452800EFF01FB005616F805F9082802A
:1094600097C7FF1F9387C7779C43D847A167938708
:10947000E702631FF702EF825F8C011132853284AD
:10948000EFF09F8AAA842285EFF01F8A854719E5AD
:109490002285EFF01F884205B337A00028008145E0
:1094A000231891003ECAEFF0FFAA05616F803F8B41
:1094B000828097C7FF1F9387A7729C43D84799471D
:1094C000631FF704EF827F87797132853284EFF072
:1094D0005F842AC62285EFF03F852310A1022285F2
:1094E000EFF03F832301A1022285EFF09F82A301C9
:1094F000A1022285EFF0FF812302A1022285EFF075
:109500005F812313A1022285EFF0BF80B2452314AF
:10951000A1022808EFF01FA445616F805F8482805C
:1095200097C7FF1F9387C76B9C43D847A167938753
:10953000C703631FF704EF825F807971328532843D
:10954000EFF02FFD2AC62285EFF00FFE2310A102B7
:109550002285EFF06FFD2311A1022285EFF06FFB52
:109560002302A1022285EFF0CFFAA302A1022285F5
:10957000EFF02FFA2303A1022285EFF08FF9B24515
:10958000A303A1022808EFF0FF9C45616F802FFD27
:109590008280EF828FFA01112A84EFF08FF7AA847C
:1095A0002285EFF06FF82285EFF00FF803574400A3
:1095B0008D4763F5E7002285EFF00FF72285EFF086
:1095C000AFF62800A685EFF0FF9805616F802FF9B0
:1095D00097C7FF1F9387C7609C43D847A167FD07C4
:1095E0006319F700EF826FF53285EFF09FFA6F8015
:1095F0000FF7828097C7FF1F9387875E9C43D847EA
:10960000A167E5076311F706EF822FF379713285C1
:109610003284EFF00FF02AC62285EFF0EFF02285BA
:10962000EFF08FF02310A1022285EFF0EFEF52054B
:1096300051812311A102228523020102EFF06FED77
:10964000A302A1022285EFF0CFEC2303A102228521
:10965000EFF02FECB245A303A1022808EFF09F8F93
:1096600045616F80CFEF828097C7FF1F9387475771
:109670009C43D847A1679387E7036319F700EF82FC
:10968000CFEB3285EFF0FFF06F806FED828097C7F0
:10969000FF1F9387E7549C43D847A16793874704EC
:1096A0006314F702EF826FE9797132853284EFF04B
:1096B0004FE62AC62285EFF02FE7B2452808EFF0E3
:1096C0007F8945616F80AFE9828097C7FF1F9387CD
:1096D00027519C43D847A167938787026316F702F7
:1096E000EF82AFE5797132853284EFF08FE22AC6DE
:1096F0002285EFF00FE2B2452300A1022808EFF027
:109700007F8545616F80AFE58280EF820FE30111B5
:10971000EFF02FE0AA852800EFF0DF8305616F806E
:109720000FE497C7FF1F9387A74B9C43D847A167B8
:10973000D1076319F700EF824FE03285EFF0FFFCAD
:109740006F80EFE1828097C7FF1F938767499C4333
:10975000D847A167C5076319F700EF820FDE32858E
:10976000EFF0BFFA6F80AFDF828097C7FF1F93874C
:1097700027479C43D847A167B9076319F700EF82D1
:10978000CFDB3285EFF07FF86F806FDD828097C787
:10979000FF1F9387E7449C43D847A167AD07631930
:1097A000F700EF828FD93285EFF03FF66F802FDB25
:1097B000828097C7FF1F9387A7429C43D84789475A
:1097C0006310F702EF826FD70111328532C8EFF0D4
:1097D0004FD4AA852800EFF0EFF705616F802FD8EE
:1097E000828097C7FF1F9387A73F9C43D847A167F5
:1097F0008D076317F702EF824FD40111328532844F
:10980000EFF02FD113066100AA844C002285EF20CF
:10981000D00C2800A685EFF0EFF305616F802FD400
:10982000828097C7FF1F9387E73B9C4381CBDC4334
:1098300091C7EF828FD082976F806FD28280EF8244
:10984000CFCF79713C08AE843ED2A165B7070A003C
:109850002A843ED448103C08DD053ED636C432C6C4
:109860003AC2EFD0BFAA12474810BA85EFF00FC036
:1098700032464810B285EFF0AFC0A2464810B68518
:10988000EFF0CFBE501001478146A6852285EFD06C
:109890007FC845616F80AFCCEF822FCA01117C0079
:1098A0000329C501AE843ECAA165B70707002A8413
:1098B0003ECC48087C00C5053ECEEFD03FA5834591
:1098C000D9004808EFF08FBA500801478146A685B5
:1098D0002285EFD03FC405616F806FC8EF82EFC56E
:1098E00083C7950093F7F707A384F500EFF0DFFA3D
:1098F0006F80EFC6EF826FC479713C08AE843ED2B0
:10990000A165B70709002A843ED448103C08938516
:1099100045043ED632C636C4EFD05F9FA2464810FB
:10992000B685EFF0AFB432464810B285EFF04FB5D0
:10993000501001478146A6852285EFD0BFBD456105
:109940006F80EFC1EF826FBF83C7950041112A84FA
:1099500093F7F707A384F50032852EC6EFF0CFBC4E
:1099600085672AC4637CF500EF50B0402246B245BB
:1099700009E9114781462285EFF07FEC41016F80B4
:109980000FBE01478346F501FDB7EF826FB90111A4
:109990003C003ECAB7070A003ECC3C003ECE83C71F
:1099A0009500AA89328593F7F707A384F5002E84E2
:1099B000EFF08FB785676371F504A165AA8493857D
:1099C00085044808EFD09F942685EF50903A2A8965
:1099D0001DE591454808EFF06FA9A6854808EFF00E
:1099E0002FAACA854808EFF06FA8014781465008A2
:1099F000A2854E85EFD01FB205616F80AFB581455E
:109A00004808EFF0AFA603490902C1BFEF824FB18A
:109A100079711C103ECAB7070F003ECC404D1C1098
:109A2000AA84AE894808994532C636893ECEEFD021
:109A3000FF8D32464808B285EFF04FA36304090258
:109A4000A5454808EFF00F9E2546CA85EFF0E019BE
:109A5000500801478146CE852685EFD0BFAB4561D2
:109A60006F804FAF8355C4024808EFF06FA10355D4
:109A7000E402814515C185478545630FF500C1673F
:109A8000FD179305F00F6309F5007D15EF50207465
:109A90009305150093F5F50F4808EFF02F9D8345CA
:109AA00004034808EFF08F9C834514034808EFF047
:109AB000EF9B835524034808EFF08F9C83554403A4
:109AC0004808EFF0EF9B69B7EF822FA783C7950097
:109AD0008146014693F7F707A384F500EFF01FF3E3
:109AE0006F80EFA7EF826FA579713E841C103ECA8C
:109AF0002E89B7070F00A1653ECCFD051C10AA8476
:109B0000480842C03AC23ECE36C432C6EFD01F80AB
:109B100032464808B285EFF06F95A2464808B685F0
:109B2000EFF00F9612474808BA85EFF06F9502489C
:109B30006304080291454808EFF0CF8E1146A285D4
:109B4000EFF0A00A500801478146CA852685EFD06C
:109B50007F9C45616F80AFA089454808EFF08F8CEE
:109B6000834704002300F50083471400A300F50099
:109B7000D1BFEF82EF9A83C7950001112A8A93F72C
:109B8000F707A384F5003285AE8432C6EFF0CF9993
:109B900032462A893285EFF0CF978567637FF900D7
:109BA000AA894A85EF50F01C2A8419E91147814699
:109BB0004A86A6855285EFF09FC805616F808F9910
:109BC0009387E9FF93F7F70F0547E368F7FE8347AD
:109BD000F50195E78947E382F9FE8346F401528552
:109BE00001474A86A685EFF09FC5A167D9074808B7
:109BF0003ECC230A010002CEEFF0BFC27DBF639CC2
:109C0000E7008947639CF90093071020231FF500A4
:109C1000EF50901AD9B70947E391E7FC8D47E39ECF
:109C2000F9FA2285EF50D03B97C7FF1F9387871A19
:109C30009C4399E797C7FF1F938787039C4389C776
:109C400003D50400EF60300C231F04002285C9B740
:109C5000EF82AF8E01113C003ECAB7070B003ECC2D
:109C60003C003ECE83C795002A89328593F7F707DB
:109C7000A384F500AE84EFF02F8B93170501C18705
:109C8000635EF004A1652A849385E5024808EFD05D
:109C9000EFE7A2854808EFE0BFFE97C7FF1F938755
:109CA00027FD9C439DEF01449375F40F4808EFE0B6
:109CB000FFFB9355844093F5F50F4808EFE01FFB39
:109CC0009355044193F5F50F4808EFE03FFA01473B
:109CD00081465008A6854A85EFD0DF8305616F80F5
:109CE0000F88416585460546A2857D15EF30706772
:109CF0005DD95105EFD04027130440063344850257
:109D000065B7EF828F830111B70706003EC683C790
:109D1000950021642A8993F7F707A384F500AE84A0
:109D200028009305A4040AC40AC8EFD02FDE30002F
:109D300001478146A6854A85EFD0CFFDEFE02FF899
:109D400013049404480822CC230A010002CEEFF049
:109D50005FAD05616F80AF80EF729FFCC1642A899F
:109D6000014497C9FF1F93896908130A8002FD14F3
:109D7000EFE0AFAB6345A40001456F70BFFDB307D3
:109D8000440303A7C90ABA9703D7070063069700DD
:109D900083D72700638427010504D9BF0545F1BF98
:109DA000EF721FF82A8A2E8999C123A005008149E4
:109DB000814497CAFF1F938A2AE3614BEFE02FADDE
:109DC00063C5A4004E856F70FFF83384640383A7D6
:109DD0000A003E948357040099E763040900232096
:109DE00089008504E1BF4146D28513054400EFE0B8
:109DF000705D65F9A289F5B7EF729FF239717C0841
:109E00003ED4B7070A003ED67C083ED883C79500EB
:109E10002A8A328593F7F707A384F5002E8932C684
:109E2000EFE09FF085676373F5063246AA843285BA
:109E3000EFE03FEE8547AA8963EAA704A165938511
:109E400085042810EFD08FCC2685EF5080722A84AD
:109E500029E191452810EFE07FE1A6852810EFE089
:109E60003FE2CE852810EFE07FE0014781463010C9
:109E7000CA855285EFD00FEAA16793877704481807
:109E80003EDC230A010202DEEFF0BF9921616F7010
:109E90007FEC81452810EFE07FDDA6852810EFE0FC
:109EA0003FDE97C7FF1F9387272B9C4391C72285CF
:109EB00063870900EFB0600C8345040265B7EFB01B
:109EC000200BDDBFEF72DFE583C795004111AA8942
:109ED00093F7F707A384F5003285AE84328AEFE06A
:109EE000BFE48567637BF5022A89EF5080682A8486
:109EF000914621C18347F50105476383E70291C776
:109F00000D47636EF702AD462DA0930505030325AB
:109F10000A004146EFE0104B1DE141016F709FE3E5
:109F20009305950803250A004146EFE0B0498146B4
:109F300079F94A86A6854E85EFF0DF9BF9BF832528
:109F40000A0013059408EF60600119C1C146D5B736
:109F500097C7FF1F938707E89C4399E797C7FF1FA1
:109F6000938707D19C4389C72285EF60A05479FD70
:109F70008547A30FF4002285EF80B05D2285EF5066
:109F8000A0634E8581464A86A685EFF0BF96A167FD
:109F90009387570448003EC42302010002C6EFF035
:109FA0005F88A5BFEF72FFD683C795004111AA89CC
:109FB00093F7F707A384F50032852E89B28AEFE084
:109FC000BFD685676370F50CAA84EF50805A2A8447
:109FD0001DE9416B014A97CBFF1F938B2BE1130CBB
:109FE000400E7D1B19A833048A0383A70B0B3E94F4
:109FF0008357C401638D6703050AEFE00F82E344D2
:10A00000AAFE954639A88357C50163929702930526
:10A01000050303A50A004146EFE0D03A994611E155
:10A0200081462686CA854E85EFF0DF8CA1A883A5E0
:10A030000A0013050403EF507072C1467DF12285BA
:10A04000231E9400EF80F0502285EF50E05697C712
:10A05000FF1F938767109C438DCB2300040222854A
:10A06000EFA090614E8581462686CA85EFF09F88D5
:10A07000A1679387070448003EC42302010002C67B
:10A08000EFF02FFA41016F705FCC89472300F40293
:10A09000D1BF397106DE22DC4AD8800052D456D2B4
:10A0A0005AD026DA4ED65ECE2E8A32892A8BEFD04F
:10A0B000DFF30605710541998A8A3301A140232205
:10A0C00024FC231404FCEFD05FF283479A000605BA
:10A0D000350593F7F7072315A4FCA304FA004A8576
:10A0E000232624FCEFE05FC493170501C18763407A
:10A0F000F0025681130104FCF2506254D2544259CA
:10A10000B259225A925A025BF24B21618280AA8490
:10A110004A85EFE07FC1AA894A85EFE0FFC0A165CB
:10A120009385C5022A89130544FCEFD02F9E26850E
:10A13000EFD0AF93854501C94A86CE85EFD06F8DAC
:10A14000AA8B15ED8945130544FCEFE03FB2A685C7
:10A15000130544FCEFE0DFB2CE85130544FCEFE0CD
:10A160003FB2CA85130544FCEFE09FB10147814629
:10A17000130644FCD2855A85EFD0CFB99DBF8145E7
:10A18000130544FCEFE09FAEA685130544FCEFE009
:10A190003FAFCE85130544FCEFE09FAECA851305A3
:10A1A00044FCEFE0FFAD8144EFD03FE4E3D0A4FCFA
:10A1B00083A70B0113971400BA9783D5070089C5AD
:10A1C000130544FCEFE0DFAB8504F9BF797106D6D7
:10A1D00022D44AD000184ECE52CC56CA26D25AC8E3
:10A1E000AE893289AA8AEFD05FE0060569054199F8
:10A1F0000A8A3301A140232A24FC231C04FCEFD04B
:10A20000DFDE83C7990006052D0593F7F707231DA9
:10A21000A4FCA384F9004A85232E24FCEFE0DFB0E0
:10A2200093170501C187634FF0005281130104FDAC
:10A23000B250225492540259F249624AD24A424BD5
:10A2400045618280AA844A85EFE01FAEA1659385AF
:10A25000A5022A89130544FDEFD04F8B2685EFD048
:10A26000CF80854519C5CA85EFC0BFFD2A8B0DE992
:10A270008945130544FDEFE07F9FA685130544FD46
:10A28000EFE01FA0CA85130544FDEFE07F9F014763
:10A290008146130644FDCE855685EFD0AFA771B732
:10A2A0008145130544FDEFE07F9CA685130544FD21
:10A2B000EFE01F9DCA85130544FDEFE07F9C8144BC
:10A2C000EFD0BFD2E3D5A4FC83270B011397140072
:10A2D000BA9783D5070089C5130544FDEFE05F9A5F
:10A2E0008504F9BFEF727FA583474500404DD5E750
:10A2F000FD574DC0834694000947636DD708034658
:10A30000B400854663E8C6088306E40063C4060813
:10A310005C45F9562390D70097C7FF1F83C7078D69
:10A3200099E3A304E40097C7FF1F938767949C43B6
:10A3300081E78947A306F40097C7FF1F9387C7E10A
:10A340009C4381E789472306F40097050000938525
:10A350004505AA8413050401EFC0703FFD57231A79
:10A36000F40281471CDC014897C7FF1F23AC878696
:10A3700097C7FF1F93874787232E040304C080439A
:10A38000EFD0FFD061463306C50281452285EF70CC
:10A39000DF9D81473E856F709F9CFD57E5BFEF7243
:10A3A000DF992A8403554502EF50A01C09E5231EBE
:10A3B00004006F70DF9A8357E401E5DF930504FF23
:10A3C0001715010013058577EFB01063DDB7EF7245
:10A3D000DF962E89A16541119385E5032A8436C451
:10A3E00032C6BE843AC2EFC07FF212472285BA85D8
:10A3F000EFE0DF8732462285B285EFE07F88A24614
:10A400002285B685EFE0DF87630D0900914522853F
:10A41000EFE05F811146A685EFE0207D41016F707E
:10A420001F9489452285EFE0EFFF83C704002300D6
:10A43000F50083C71400A300F500CDB7EF72FF8FBE
:10A4400083C79500444D054793F7F707A384F500AC
:10A450001C42411183C70700636DF7042E842A89CB
:10A4600085CC03C7D4006309F70217C7FF1F130782
:10A470002780184301CFA386F400EF80902B83C779
:10A48000D40089E741657D15EF30407583D72403FB
:10A49000918B99C3EFB0B0624A85A285EFF0CFBF30
:10A4A000A167C10748003EC42302010002C6EFF0C5
:10A4B0004FB741016F70BF8AEF723F8803D74500E5
:10A4C0008D47AA8441112E8432892E8563EDE700E1
:10A4D000EFE09F85AA85230009002685EFC07FD67F
:10A4E00041016F70DF87EFE03F842AC62285EFE0ED
:10A4F000BF83B24585472A862300F9002685EFC031
:10A500005FD1F9BF397106DE22DC26DA80004ED633
:10A5100052D456D24AD85AD05ECEAE89B284AA8AD4
:10A52000EFD0BFAB06051305250241990A8A330116
:10A53000A140232224FC231404FCEFD01FAA83C7CC
:10A54000990006054D0593F7F7072315A4FCA3848E
:10A55000F9002685232624FCEFE00FFD9317050163
:10A56000C1876340F0025281130104FCF25062542F
:10A57000D2544259B259225A925A025BF24B21618B
:10A580008280AA8B03AB0400EFC03FCE35E983D7AE
:10A59000440001498544F11793B71700A301F4FC67
:10A5A000834734FCA165BDC79385E504130544FCCE
:10A5B000EFC0DFD5A685130544FCEFE02FEBDE8569
:10A5C000130544FCEFE0CFEB834734FC114691E3E5
:10A5D0000946DA85130544FCEFE06FE78144630820
:10A5E0000900416B7D1BEFD05F9F63C8A402014748
:10A5F0008146130644FCCE855685EFC0BFF1A5B752
:10A60000A685130634FCEFF03FEB933415002A893E
:10A61000860479B79385C50451BF8327C900139772
:10A620001400BA9783D5070063866501130544FCBF
:10A63000EFE00FE5850445BFEF72AFED79711C10B7
:10A640003EC4B7070F003EC61C103EC883C7950026
:10A65000AA8A328593F7F707A384F500AE8932847E
:10A66000EFE08FEC93170501C1876350F0062A8A4B
:10A670002285EFE06FEB2A895285032B0400EFC09F
:10A68000DFBE39E58357440081440544F11793B791
:10A690001700A303F10083457100DA872287CA8679
:10A6A00052862800EFF0BFD2014781463000CE85A8
:10A6B0005685EFC03FE6A1679387D70348083ECC95
:10A6C000230A810026CEEFF0CF9545616F70EFE74A
:10A6D000A28513067100EFF03FDEAA84094445DD30
:10A6E0003544E30A55FB4A85EFF00FE70D4445D5A5
:10A6F0000144EFD09F8E634BA400C16B0144FD1B4E
:10A70000EFD0BF8D634EA400154471B7DC4413171E
:10A710001400BA9783D70700638127030504D1BFCC
:10A72000D84493171400BA9703D707006319770129
:10A73000239027012685EF80C0540144A9BF05045A
:10A74000C1B7EF72EFDD83C7950041112A8A93F7F5
:10A75000F707A384F50032852E893284EFE0CFDC41
:10A7600093170501C187635BF004AA892285EFE096
:10A77000AFDB2311A1004E85832A0400EFC0FFAE9A
:10A7800029E18357440085440144F11793B717002A
:10A79000A300F1000348110003572100D68752851A
:10A7A000CE862686CA85EFF0EFB3A167F107480091
:10A7B0003EC42302910022C6EFF0AF8641016F70C4
:10A7C0006FD9A28513061100EFF01FCF2A848944A8
:10A7D00071D18357210011678544BA97C207116769
:10A7E000C1831307F7EFE367F7FA97B7FF1F938764
:10A7F000675E9C4391C7854513052100EF40300EED
:10A800008355210022858144EFC09F9D41D52310AF
:10A8100005002285EF808048B5BFEF728FCF83C7D8
:10A82000950041112A8B93F7F707A384F500328531
:10A830002E8A3284EFE04FCF93170501C187635909
:10A84000F004AA8A2285EFE02FCE2A895685832B31
:10A850000400EFC09FA121E18357440081440544D7
:10A86000F11793B71700A301F10003483100DE8709
:10A870005A854A87D6862286D285EFF0AFA6A16791
:10A88000ED0748003EC42302810026C6EFE07FF9B1
:10A8900041016F708FCBA28513063100EFF0DFC14D
:10A8A000AA84094479D19167CA97C2071167C18305
:10A8B0001307F7EF0544E36AF7FACA85EFC05F9222
:10A8C000014445F58149EFD04FF263DBA900984878
:10A8D00093971900BA9703D7070015E7239027012C
:10A8E000EFD0AFF01544E382A9F82685EF80003B56
:10A8F00097B7FF1F9387074E9C430144BDD74A85F6
:10A90000EF4040769DB785097DBFEF726FC17971C9
:10A910003E847C083EC82E8AB7071400A1653ECA53
:10A92000E5057C08AA89080836C4428932C6BA8A75
:10A93000C6843ECCEFC09F9DCA850808EFE00FB3E8
:10A9400032460808B285EFE0AFB3A246630E0902B3
:10A950009D450808EFE00FAD1D468145EF70EFC043
:10A9600063870A0691450808EFE0CFAB1146A6853C
:10A97000EFE0A027100801478146D2854E85EFC041
:10A980007FB945616F700FBDB6850808EFE04FAF26
:10A990001C400808D8439355C70185891207518385
:10A9A000B205D98DEFE0CFAD1C40080883C5870004
:10A9B000EFE0CFAB1C40080883C5A700EFE00FAB6A
:10A9C0001C40080883C59700EFE04FAA51BF894596
:10A9D0000808EFE02FA583C704002300F50083C714
:10A9E0001400A300F50079B7EF728FB383C7950009
:10A9F0004111AA8993F7F707A384F5003285AE8445
:10AA00003284EFE06FB293170501C1876357F004FA
:10AA10002A89032A0400EFC05F8519E9835744009F
:10AA20000548F11793B71700A307F100814621A845
:10AA30001306F100A285EFF03FA81DC11C459DC380
:10AA400083D6470001480347F10093078500D28869
:10AA50004A86A6854E85EFF05FEB41016F708FAFA0
:10AA60000948E9B71D48D9B7EF728FAB65715C082B
:10AA70003EC4B7077B013EC65C083EC883C795004D
:10AA80002A8A328593F7F707A384F500AE89EFE0B1
:10AA90004FA88357E100C5C389452800EFC01F8731
:10AAA00081452800EFE08F9CEFC0FF8B97B7FF1F19
:10AAB0009387876A9C4317B4FF1F03442413AA8417
:10AAC0003334800099C31364240097B7FF1F938722
:10AAD000271A9C4399C31364440097B7FF1F9387B9
:10AAE000672F9C4399C31364840083D50400280016
:10AAF0000149EFE0EF9883D524002800EFE04F985C
:10AB000083D544002800EFE0AF97EFD00FC993152D
:10AB10000501C1812800EFE0AF96A2852800EFE093
:10AB20002F969C44636CF900014781463000CE8526
:10AB30005285EFC03F9E59616F70CFA1DC44131462
:10AB4000490028003E94EFE06F8C834744000347A0
:10AB5000540089070607BA978607E36EF5FC83550C
:10AB600024002800814AEFE0AF918345440028008B
:10AB7000EFE0CF8F834554002800EFE02F8F83470D
:10AB8000440063C9FA00814A8347540063CFFA0046
:10AB9000050941BF1C4413975A002800BA9783D572
:10ABA0000700850AEFE0CF8DD9BF032BC400939730
:10ABB0005A0028003E9B83552B00850AEFE04F8CFE
:10ABC00083550B002800EFE0AF8B7DBFEF72EF964F
:10ABD0005C4993E717005CC9EF8020336F702F98B2
:10ABE000EF72AF952E848145EFF08F9B05C183579F
:10ABF0000500FD172310F50009C483572500231015
:10AC0000F400EFF0BFFC01456F706F9531456DDCCE
:10AC100023100400D5BFEF72AF9083C79500411198
:10AC20002A8A93F7F707A384F50032852E893284A8
:10AC3000EFE08F8F93170501C187635EF004AA8947
:10AC4000C1452285EFD0BFFA2A8B4E85832A0400A6
:10AC5000EFC0AFE121E58357440023110100054413
:10AC6000F11793B71700A300F100814403481100C6
:10AC700003572100D6875285CE862286CA85EFE00B
:10AC80007FE6A1679387170248003EC42302810034
:10AC900026C6EFE01FB941016F70CF8B130611007C
:10ACA000A285EFF07F81AA8409E523110100094400
:10ACB00075BF930521005A85EFF09FF2835721005D
:10ACC0002A84CDD797B7FF1F9387C7109C4391C79E
:10ACD000854513052100EF408040835521002685DE
:10ACE0003144EFC0EFCF59D1231005002685EF7016
:10ACF000F07A0144A5BFEF724F8441112E896C0098
:10AD0000AA8402C6EFF0CF8909CD035705000507D5
:10AD10002310E500EFF09FEB81473E8541016F7006
:10AD20000F843247954775DBCA852685EF20D0080A
:10AD3000C147E34405FE3244854741462310F400F1
:10AD400083570900A685130544002311F400EFD0B2
:10AD5000D0692285C1B7EF62BFFC83C7950041115E
:10AD6000AA8A93F7F707A384F5003285AE89328467
:10AD7000EFD09FFB93170501C187635EF0042A8A19
:10AD8000C1452285EFD0BFE6AA845285032B04007B
:10AD9000EFC0AFCD21E58357440023110100854466
:10ADA000F11793B71700A300F10001440348110005
:10ADB00003572100DA875685D2862686CE85EFE0B6
:10ADC0007FD2A1679387070248003EC42302910007
:10ADD00022C6EFE01FA541016F60DFF7A2851306D1
:10ADE0001100EFF06FED2A8409E523110100894479
:10ADF00075BF268593052100EFF0FFEFAA845DF56E
:10AE0000835521002285EFC0AFBD4DF10149EFD040
:10AE1000CF9D635DA900184893171900BA9703D70F
:10AE200007001DE7035721002390E700EFD0EF9BB9
:10AE30006302250397B7FF1F9387C7F99C4389C710
:10AE400003552100EF4000222285EF703065B9BF25
:10AE5000050975BF954499BF05C19307F00F630FAE
:10AE6000F500C547630CF5009307F5FF054533155D
:10AE7000F5004205418182800145828041657D1552
:10AE80008280B9E1EF627FEB034506033284EFF085
:10AE9000BFFC9305803EB305B502C205C18191C9CF
:10AEA0000357E402854763F6E70013050401EFC08A
:10AEB00020168357E40241677D176385E700FD177D
:10AEC0002317F4026F60BFE98280EF629FE40042C3
:10AED00083C79500444D0349140093F7F707A384F3
:10AEE000F50083470400220911673369F900A1675F
:10AEF000B347F90041112A8BAE8A63ECE70C834714
:10AF000024001307C00EB91793F7F70F6371F70EFC
:10AF100003473400C14763ECE70C83474400130741
:10AF2000E00793C707086373F70A834984008347E0
:10AF30007400A209B3E9F900856763F9F908034AC7
:10AF40006400834754004E85220A336AFA00EF40BA
:10AF5000406245C123962403834B3400137AFA00E0
:10AF6000239A3403238874032399440393890401A7
:10AF7000631A090023A60402239804024E85EFC039
:10AF8000A00A1DA0034924004A85EFF0FFEC239797
:10AF9000A402834744004E85A388F402E3810BFE9C
:10AFA000E30F09FCEFC06005EF7090798146014620
:10AFB000D6855A85EFE09FA5A167938797033EC486
:10AFC00023020100480002C6EFE0BF8541016F6027
:10AFD000DFD78544A2862686D6855A85EFE01FA353
:10AFE000A167938797033EC423029100E1BFBD444C
:10AFF000D5B79144C5B7EF62BFD201111C08404DCF
:10B000003EC2B7070F003EC41C083EC62A89AE895F
:10B01000EFC01F9D585C1C5C634CB70A6394E5004D
:10B0200063E8A70A3385A740B3B7A700B305B740C5
:10B030001306803E81469D8DEFD0407B9314050121
:10B04000C180A1659385C5034800EFC02FAC814541
:10B050004800EFD0BFC1835504044800EFD05FC261
:10B06000835524044800EFD0BFC1814599C8C1670A
:10B07000FD179305F00F6386F4002685EF40201539
:10B08000AA854800EFD09FBE03554404814511C9ED
:10B09000C167FD179305F00F6305F500EF4020131E
:10B0A000AA854800EFD09FBC834564044800EFD0D8
:10B0B000FFBB834574044800EFD05FBB50000147DD
:10B0C0008146CE854A85EFC0EFC405616F609FC899
:10B0D000814485BFEF627FC683C7950093F7F7076A
:10B0E000A384F500EFF03FF16F607FC7EF625FC3AD
:10B0F00083C795004111404D93F7F707A384F500EE
:10B100002A8A3285B284AE89EFD01FC22A8B268567
:10B11000EFD09FC12A892685EFD0BFBF93170B01BF
:10B1200063CA0702E177CA97C207C183116763E365
:10B13000E70293070910C207C1831307B00F637BAF
:10B14000F70093170901C187AA8A6348F000C54731
:10B1500063FA570141016F60FFBFEFC08F83E31BAC
:10B1600025FFF5B763060B02630409028144638778
:10B170000A02B7077F0023106405231124057CC051
:10B180005685EFF07FCD9304803EB304950239A03D
:10B19000B7077F00232004047CC0814403552404A6
:10B1A000EFB0101095CCEFC0BF83269593D7F44134
:10B1B00033379500AE97BA9708DC5CDCCE855285B4
:10B1C000EFF07FE399E023220404A1679387B7039C
:10B1D00048003EC42302010002C6EFE08FE49DBF99
:10B1E000814701481CDC232E0403C9BFEF62FFB472
:10B1F000EFC0FFE9E1473305F5029145EF30507F9D
:10B20000E55711C597B7FF1F23A0A79E81473E852D
:10B210006F60FFB4854717B7FF1F2309F79C828033
:10B22000EF62BFB197B7FF1F9387C79B80432DC0C5
:10B2300083570404639EA70483572404639AB704C6
:10B240003689B284EFC0CFF95C5C63C3B704639501
:10B25000B7001C5C63EEA7028347640463F3F40049
:10B26000A6872303F4048347740463F39700A68737
:10B27000A303F4048357440441677D176385E70003
:10B2800085072312F4043C4481C7CA85268582972A
:10B290006F60FFAC97B7FF1F9387C7949C4301452E
:10B2A00099C303C587008280EF623FA90111B707E8
:10B2B00007003EC683C79500584D0AC493F7F707A9
:10B2C0000AC8A384F5002A89AE8401CB1C4283C737
:10B2D00007002304F700EF70D04521649305540262
:10B2E0002800EFC0AF82EFF0FFFAAA852800EFD068
:10B2F000FF97300001478146A6854A85EFC08FA1A0
:10B3000013044402480822CC230A010002CEEFE0D5
:10B310004FD105616F60BFA4EF623FA201117C00B5
:10B320003ECAB70707003ECC7C003ECE83C79500DF
:10B330002E84AA8493F7F707A384F500A16593856B
:10B3400055024808EFB09FFCEFF0DFF4AA854808EB
:10B35000EFD0DF91500801478146A2852685EFC0D6
:10B360006F9B05616F60BF9F97B7FF1F93878787AC
:10B370009C43094599C303C59700828097B7FF1F77
:10B38000938747869C43094599C303C5D7008280AC
:10B3900097B7FF1F938707859C43014599C303C552
:10B3A000A7008280EF62DF970111B70708003EC651
:10B3B00083C79500404D0AC493F7F7070AC8A384D2
:10B3C000F5002A89AE8429C01442854703C70600C8
:10B3D00063EEE7068347940009468149638EC70000
:10B3E000B307F740A304E400B339F00083C71600A5
:10B3F0002305F400EF70F03303572403058B09C7CE
:10B4000063840900EFA0B06B2164930584022800D7
:10B41000EFB0DFEFEFF05FF5AA852800EFD01F85D2
:10B42000EFF01FF7AA852800EFD05F84014781461F
:10B430003000A6854A85EFC0EF8D130474024808DA
:10B4400022CC230A010002CEEFE0AFBD05616F60A0
:10B450007F90EF629F8E01117C003ECAB707080003
:10B460003ECC7C003ECE83C795002E84AA8493F701
:10B47000F707A384F500A165938585024808EFB01E
:10B48000FFE8EFF07FEEAA854808EFD02FFEEFF03F
:10B490003FF0AA854808EFD06FFD5008014781466C
:10B4A000A2852685EFC00F8705616F605F8B97A728
:10B4B000FF1F938727739C43014599C303C5B700BA
:10B4C0008280EF629F870111B70707003EC683C7DE
:10B4D0009500404D0AC493F7F7070AC8A384F50006
:10B4E0002A89AE8405C41C42054783C70700636AE6
:10B4F000F7040347B400630BF700A305F400EF70F3
:10B5000050238347B400A9C3EFD00FD9216493051A
:10B51000B4002800EFB09FDFEFF07FF9AA85280084
:10B52000EFD0CFF4014781463000A6854A85EFB0C1
:10B530007FFE2904480822CC230A010002CEEFE056
:10B540004FAE05616F60BF81EFD02FDAC1B7EF62F8
:10B55000CFFE01117C003ECAB70707003ECC7C003D
:10B560003ECE83C795002E84AA8493F7F707A38461
:10B57000F500A165AD054808EFB05FD9EFF03FF3E6
:10B58000AA854808EFD08FEE500801478146A28572
:10B590002685EFB03FF805616F606FFC97A7FF1F2E
:10B5A000938747649C43094599C303C5C7008280BC
:10B5B000EF62AFF801117C00AE843ECAA165B70707
:10B5C00007002A843ECCD1057C0048083ECEEFB06F
:10B5D000FFD3EFF0BFFCAA854808EFD02FE9500851
:10B5E00001478146A6852285EFB0DFF205616F60D5
:10B5F0000FF7EF628FF483C7950093F7F707A384E3
:10B60000F500EFF0FFFA6F608FF5EF626FF183C71F
:10B6100095000329C501411193F7F707A384F500AD
:10B620001C4283C90700854763EC370597B7FF1FA6
:10B63000938787B29C432E84AA8495C7EFF01FF6A8
:10B6400089476302F502630009028347C900638CDE
:10B65000370123063901EF70D00D83572903898BF9
:10B6600099C3EFA0D0452685A285EFF07FF4A167AE
:10B67000CD0748003EC42302010002C6EFE06F9AE6
:10B6800041016F602FED97A7FF1F9387A7559C433C
:10B690001D4599C303C5E7008280EF620FEA0111DF
:10B6A000B70707003EC683C79500584D0AC493F7F5
:10B6B000F7070AC8A384F5002A89AE8405C71C428F
:10B6C00083C7070093968701E18663C80604854611
:10B6D0006385D7048346E7006386F6002307F700F7
:10B6E000EF70300521649305E4002800EFB01FC21D
:10B6F000EFF07FF9AA852800EFD04FD701478146A8
:10B700003000A6854A85EFB0FFE03504480822CC1A
:10B71000230A010002CEEFE0CF9005616F602FE4B5
:10B72000EF62AFE101117C003ECAB70707003ECCD3
:10B730007C003ECE83C795002E84AA8493F7F7073A
:10B74000A384F500A165B9054808EFB03FBCEFF050
:10B750009FF3AA854808EFD06FD150080147814672
:10B76000A2852685EFB01FDB05616F604FDFEF62BA
:10B770002FDBAA84014417A9FF1F1309E946E149F9
:10B78000EFC0FF906344A400014519A833053403BA
:10B79000832709003E95835725006395970011057F
:10B7A0006F604FDB0504E9BF032E850063040E10B4
:10B7B00017A3FF1F13030362032303006315030092
:10B7C0002943639A060E03234E01631503001D43AC
:10B7D0006393070EEF62EFD3C689428A3E89BA8A25
:10B7E000B684328BAE8B2A84A1E903554E0009E55D
:10B7F00001431A856F606FD5A167A98F116763F741
:10B80000E700EFF0DFF68145EFF08FBD0844B707A2
:10B8100000E05841F98F18455CC1B707001FF98F48
:10B820001CC55C4981C76105EFB01000E38209FCCB
:10B830002285EF70606E6DBF3285EFA0E0620D4330
:10B840004DD91C44116703D54700A167A98F63F741
:10B85000E700EFF0DFF18145EFF08FB803238400BC
:10B8600093164B01D1828347B3000356630085884A
:10B87000FD8BA305F300FD777D8E558EFD76FD16BD
:10B88000B204F18E83274301C58E23127301231363
:10B89000D3002304530123052301A3044301D9D773
:10B8A0002285EFB07FBBAA850844B5DD6105EFB006
:10B8B0002076ADBF1D431A858280EF626FC6056991
:10B8C000AA84AE89328A0144FD5A7D19EFC0EFF097
:10B8D0006345A40001456F60EFC7D8449317140077
:10B8E000BA9703D70700631B3703239057016305FB
:10B8F0000A002685EF70E0389C448DC383D767002B
:10B90000B3F72701639C3701D2880148814701477B
:10B910008146014681452685EFF01FE905047DB784
:10B92000EF620FC079711C103EC4B7070F003EC60E
:10B930001C103EC883C79500AA8A328593F7F70783
:10B94000A384F5002E893284EFD00FBE9317050132
:10B95000C1876350F006AA892285EFD0EFBC2A8AFE
:10B960004E85032B0400EFB05F9039E58357440008
:10B9700081440544F11793B71700A303F1008345F1
:10B980007100DA872287D2864E862800EFE03FA436
:10B99000014781463000CA855685EFB0BFB7A16721
:10B9A0009387F70348083ECC230A810026CEEFD0C8
:10B9B0005FE745616F600FBAA28513067100EFE083
:10B9C000BFAFAA84094445DD5285EFE0EFB80D44CE
:10B9D0005DD50546D2852685EFF03FEE2A8445B732
:10B9E000EF62AFB5835507000346270041112A8453
:10B9F0002E8532C62EC4EFE02FB611C53246A245C1
:10BA00002285EFF09FEB41016F606FB5EF626FB081
:10BA100083C795004111AA8A93F7F707A384F5001D
:10BA20003285AE893284EFD02FB093170501C187DC
:10BA30006357F008C1452A8A2285EFD04F9B2A8D93
:10BA40002285EFD06FAE2A892285EFD08FAC930785
:10BA500005F893F7F70F1307E007AA8B6371F70652
:10BA60002285EFD00FAB2A8C2285EFD08FAAAA8C2B
:10BA70005285032B0400EFB04FFF29E583574400A4
:10BA8000231101008144F11793B71700A300F100BF
:10BA9000054403471100835621009387840056858F
:10BAA000DA8822885286CE85EFE03FE6A167E90773
:10BAB00048003EC42302810026C6EFD09FD6410134
:10BAC0006F60AFA813061100A285EFE0FF9EAA8465
:10BAD00009E52311010009446DBF930521006A8522
:10BAE000EFF06FA12A8455F5835521009356C900C4
:10BAF0001316490185486688E2875E87858A5182E8
:10BB00002685EFF07FCA2A8469B7EF628FA083C7CA
:10BB1000950041112A8B93F7F707A384F50032852E
:10BB2000AE893284EFD04FA093170501C1876352CD
:10BB3000F0082A8A2285EFD02F9FAA8A2285EFD08B
:10BB4000AF9E2A892285EFD0CF9C930705F893F703
:10BB5000F70F1307E0072A8C637DF7042285EFD0E7
:10BB60004F9BAA8C2285EFD0CF9A2A8D5285832BAA
:10BB70000400EFB08FEF29E183574400854401446E
:10BB8000F11793B71700A301F100034731009307A2
:10BB900084005A85DE882688D6865286CE85EFE0D8
:10BBA000DFD68D4748003EC42302910022C6EFD065
:10BBB0005FC741016F606F99A28513063100EFE006
:10BBC000BF8F2A84894471D19356C9001316490145
:10BBD00085486A88E6876287858A5182D685EFF034
:10BBE000BFBCAA845DB7EF62AF932A898144014448
:10BBF000617A916A17ABFF1F130BCB1DEFC0EFBE2D
:10BC000063C5A40022856F60EF9483270900939990
:10BC10001400CE9703D5070033074501420741833F
:10BC20006362570311CD03270B0009C785453E8585
:10BC3000EF30E04A832709000504CE9723900700E0
:10BC400085046DBFEFF0BFB2832709000504CE97CE
:10BC50002390070075D58145EFE09FF8D5B7EF62D7
:10BC60002F8C83C7950041112A8A93F7F707A38485
:10BC7000F50032852E893284EFD00F8B93170501A2
:10BC8000C1876354F004AA89832A0400EFB0EFDD72
:10BC900021E18357440085440144F11793B717000D
:10BCA000A301F10003483100D68752850147CE86B3
:10BCB0002686CA85EFD01FE3A167F50748003EC47A
:10BCC0002302910022C6EFD0DFB541016F608F885B
:10BCD000A28513063100EFE02FFE2A84894479D132
:10BCE00097A7FF1F9387070F9C4381CB0449EFC0A1
:10BCF000CFAFAA852685EF30803E13050401EFF013
:10BD00009FEE2285EF609079814469BFEF626F807A
:10BD100083C795004111AA8A93F7F707A384F5001A
:10BD20003285AE89328423110100EFC0FFFF9317E3
:10BD30000501C187635CF0042A8AC1452285EFC0F2
:10BD40001FEBAA8B5285032B0400EFB00FD231E119
:10BD50008357440085440144F11793B71700A300AB
:10BD6000F1000348110003572100DA875685D28677
:10BD70002686CE85EFD01FD7A1679387270248007C
:10BD80003EC42302910022C6EFD0BFA941016F50EB
:10BD9000DFFBA28513061100EFE00FF22A8489442D
:10BDA00069D197A7FF1F9387E70298433E8901CB8C
:10BDB0000449EFC08FA3AA852685EF3040321305D2
:10BDC0000401EFF05FE2EFC04FA2954459D993050B
:10BDD00021005E85EFE03FF2AA8441F51C4803573D
:10BDE000210022852390E700EF60506B8327090034
:10BDF000ADDB03552100EF30E026A5B7EF527FF110
:10BE000083C795004111AA8A93F7F707A384F50029
:10BE10003285AE893284EFC03FF193170501C187A7
:10BE20006359F0042A8A2285EFC01FF02A895285BF
:10BE3000032B0400EFB06FC321E183574400854416
:10BE40000144F11793B71700A301F1000348310033
:10BE5000DA8756854A87D2862686CE85EFD09FC858
:10BE6000A167F90748003EC42302910022C6EFD023
:10BE70005F9B41016F507FEDA28513063100EFE01B
:10BE8000AFE32A84894479D19167CA97C2071167C1
:10BE9000C1831307F7EF8544E36AF7FA97A7FF1FFB
:10BEA000938747F39843BE8B01CB0449EFC0EF93D0
:10BEB000AA852685EF30A02213050401EFF0BFD23A
:10BEC000EFC0AF92954459D11C48228581442390FC
:10BED0002701EF60B05C83A70B00ADDB4A85EF3034
:10BEE0006018ADB7EF527FE52A844105B284EFF0C8
:10BEF0009FCF01C52285EF60705A81460146A68515
:10BF00002285EF70C00B1C4C89C7DC4799C3228582
:10BF100082976F50DFE497A7FF1F9387A7CC9C43BE
:10BF2000014599C313850701828097A7FF1F938757
:10BF300067CB88438280EF525FE09317C600DD8DA8
:10BF4000C2054111C1812A8432C6EFC07FD3324677
:10BF5000228511829375F60FEFC05FD141016F50BA
:10BF60001FE0EF52FFDB79713C083ED2B7070C00AF
:10BF70003ED43C083ED683C79500AE842A8993F709
:10BF8000F707A384F500A165938535044810EFB049
:10BF9000EFB7C165FD15014417AAFF1F130A0AE593
:10BFA000930A400EAE892E8B2EC6EFC00F87420536
:10BFB000931704014181C183B24563E3A702C167BE
:10BFC000FD176385F5004810EFC09FCB5010014767
:10BFD0008146A6854A85EFB0EFD345616F509FD764
:10BFE0003307540383270A0BBA9703D6C7016308A4
:10BFF0003601638835014810EFF0FFF3DA85050458
:10C0000065B7B285EDBFEF52DFD079717C083EC8CD
:10C01000B70711003ECA7C083ECC83C79500AA89A9
:10C02000328593F7F707A384F5002E89EFC0DFCFA1
:10C030008567637EF502A165AA8489050808EFB0CB
:10C04000EFAC2685EF30E052133415000A04A285C8
:10C050000808EFC0BFC1A6850808EFC07FC235C081
:10C06000014781461008CA854E85EFB0AFCA4561C9
:10C070006F50BFCDB30754030327CA0ABA9703D73B
:10C080000700631A970003D62700638A6503080830
:10C09000EFF07FEADE8505042EC6EFB01FF94205FA
:10C0A000931704014181C183B245E3E5A7FCC16751
:10C0B000FD17E387F5FA0808EFC09FBC55B7B285B6
:10C0C000D9BFC165FD15014417AAFF1F130A0AD283
:10C0D000930A80022E8BAE8BC1B7EF521FC6184158
:10C0E0008347170083460700A207D58FD207D18365
:10C0F0002390F50083472700034717008D45A207CB
:10C10000D98F91832310F600EFC03FAD6F503FC52C
:10C11000EF521FC1C164014417A9FF1F130909CDC4
:10C1200093098002FD14EFB05FF06345A400014560
:10C130006F505FC2330534038327C90A3E95835786
:10C140000500E38797FE0504F9BFEF527FBD2A8AF9
:10C15000AE89B284B68AEF30C04109E591473E8589
:10C160006F505FBF2A894E85EF9010502A84638AF2
:10C170000A048D476DD503570500C547E31147FFF6
:10C180000347F9018546AD47E31BD7FC83474500CC
:10C1900091CB4146A6855D05EFC0D022814761D194
:10C1A000AD4775BF130965012302E500CA852685E1
:10C1B000EF10202D15CDA547E3830AFA23020400D2
:10C1C00079BF11CD83570500E39A47F94146A6850B
:10C1D0001905EFC0301F814759D1994749B74E859E
:10C1E000EFF01FF32A8495473DD9130955007DBF11
:10C1F0004146A6852310440123113401130519007B
:10C20000EFC0B01E2285EF60B03C814789BFEF527E
:10C21000DFB279717C003ECCB7070A003ECE7C00CD
:10C220003ED083C79500B2842E8493F7F707A3848A
:10C23000F5001306A1002A892C002685EFF0FFE9FE
:10C24000A16528088D05EFB06F8C90408355A10043
:10C25000035581008546EFF05FEFAA84AA85280880
:10C26000EFC0DFA00356A100835581002808EFF03E
:10C270009FCC300801478146A2854A85EFB08FA93F
:10C28000854748103ED42302910202D6EFD06FD9E1
:10C2900045616F50DFACEF525FAA79717C003ECCF4
:10C2A000B7070A003ECE7C003ED083C79500B2841B
:10C2B0002E8493F7F707A384F5001306A1002A89BB
:10C2C0002C002685EFF07FE1A16528088D05EFB0F1
:10C2D000EF8390408355A100035581008146EFF024
:10C2E000DFE6AA84AA852808EFC05F980356A1005C
:10C2F000835581002808EFF01FC4300801478146AC
:10C30000A2854A85EFB00FA148102302910202D402
:10C3100002D6EFD00FD145616F507FA4EF52FFA13D
:10C32000EFF0BFE26F50BFA397A7FF1F9387C78BA4
:10C3300088438280EF527FA0835725004111AE844D
:10C340002A842307B10017F5FFFF1305A5696C00C8
:10C350002316F100EFB0CFD581C42285EF60B02D58
:10C36000FD572310F40013062002814513055400E5
:10C37000EF50BF9F41016F509F9EEF527F9A79719E
:10C380007C003ECCB7070A003ECE7C003ED083C77F
:10C390009500AA89AE8493F7F7073285A384F50048
:10C3A0001306A1002C00EFF05FD303558100114468
:10C3B000EF30201C15C10355A1000144EF90D02A95
:10C3C00001CD035705008357810045446316F700EC
:10C3D0008545EFF03FF601442169930539002808AF
:10C3E000EFA0DFF2A2852808EFC05F880356A10006
:10C3F000835581002808EFF01FB4300801478146BB
:10C40000A6854E85EFB00F9148104AD423028102D1
:10C4100002D6EFD00FC145616F50DF93EF525F90AE
:10C420009797FF1F9387077C2A8488432E8915C11D
:10C43000035745038357C401631DF70023260502F4
:10C44000231805024105EFA0303E63040900EF60A8
:10C45000302F814497A9FF1F93894999130A8002BD
:10C46000EFB0BFBC63CCA40297A7FF1F93874780A0
:10C470009C4389C70355C401EF104076630509004A
:10C480002285EF6050031306400E81452285EF5050
:10C49000DF8DFD57231EF4006F50DF8B338544037F
:10C4A00083A7C90A3E95035705008357C401631546
:10C4B000F700CA85EFF01FE885045DB7EF525F868D
:10C4C00083C795004111AA8993F7F707A384F50064
:10C4D0003285AE84EFC05F8585676370F5042A8975
:10C4E000EF302009014411C983D704003144638629
:10C4F00027018545EFF09FF201444E85A2864A86CA
:10C50000A685EFD02FBFA1679387170448003EC4CC
:10C510002302810002C6EFD0CFB041016F509F834C
:10C52000EF521F809797FF1F9387C76B80431DCCE7
:10C530000145EFA0E05681470148C1641CDC232E71
:10C5400004032320040417A9FF1F1309298A0144A7
:10C550009309400EFD14EFB05FAC634BA40081451E
:10C560001705000013054598EFB08FB46F508FFE8C
:10C57000330534038327090B3E958357C501638533
:10C5800097008545EFF09FE90504F1B79357050142
:10C5900013D78700A380F50093170501C183A183FA
:10C5A0002380E5002381F500A381A5008280EF525E
:10C5B000CFF82300050083C71500A300F50083C74B
:10C5C00025002301F50083C73500A301F50083C7CB
:10C5D00045002302F50083C75500A302F50083C779
:10C5E000650093059500A30305002303F5002304CC
:10C5F00005003285EFF09FF96F506FF6EF524FF262
:10C600004111E9541DC995C993F9C5FF2E842A89A2
:10C61000AA84338AA900B7EA040063149A020D8839
:10C62000854401CCB7E704009C5F82972AC6228626
:10C630006C0033053901EFC0405B268541016F5026
:10C640006FF183A78A039104829793170501C18331
:10C65000A183A38EF4FE93570501238FF4FEA183DB
:10C66000238EA4FEA38FF4FE4DBF63E0D502EF52EC
:10C67000CFECB28741113686BE8536C6EFC0E05694
:10C68000B246410136856F508FED814636858280F6
:10C69000838705001387F5003D05FD8793F777082D
:10C6A000834607007D158606B58FA300F500630756
:10C6B000B7007D17834717009D83DDB78280EF5257
:10C6C000CFE7B7E7040083A7070932872A863A85B0
:10C6D0008297133515006F508FE801CD814799C9B6
:10C6E000EF52AFE54146EFC0405085473E856F5061
:10C6F0000FE781473E8582801DC5EF520FE441461A
:10C7000081452A84EF506FE64146814513050403B5
:10C71000EF50AFE50147C1672322040438C87CC845
:10C7200005456F50CFE301458280814729CDA1CDDA
:10C73000EF52AFE0B2842E891306800581452A842A
:10C74000EF50AFE2CA8524C42685EFF01FF94146B9
:10C7500081452285EF506FE13044A2852285EFF0BC
:10C760001FF693040401A2852685EFF07FF2A685CB
:10C7700013050402EFF0DFF12285EFF0FFF78547A4
:10C780003E856F50CFDD3E858280EF526FD94111DB
:10C79000E9541DC995C993F9C5FF2E842A89AA8435
:10C7A000338AA900B7EA0400639444030D888144E6
:10C7B00001CCB7E704009C5F82972AC622866C00F2
:10C7C00033053901EFC06042268541016F508FD893
:10C7D00083A78A039104829793170501C183A183DC
:10C7E000A38EF4FE93570501238FF4FEA183238EBD
:10C7F000A4FEA38FF4FE4DBF71CDEF526FD2B28471
:10C8000001E605456F500FD52A842E890145FDD9D3
:10C810003C487848B3E6E700F5D69386F7FFB3B710
:10C82000F6007D17032A4404BA9734C87CC8630F06
:10C830000A04C14913050A03B38949412295637B60
:10C840003601B2862E86A685EFF03FE27C40BE948C
:10C8500064C045BFCE862E86CE85EFF01FE1C114A1
:10C86000D2944E9923220404A2879306040103C79D
:10C87000070003C607038507318FA38FE7FEE39800
:10C88000F6FE3044A2852285EFF07FE32699C14968
:10C890003306994063EA9900ADD4A686A6851305B0
:10C8A0000403EFF09FDC6DB78147B306F400330754
:10C8B000F6000347070083C5060085072D8F2380F8
:10C8C000E600E39437FF3044A2852285EFF03FDF96
:10C8D000C1147DBF0145828019C9EF520FC61306EE
:10C8E00080058145EF506FC805456F504FC7014522
:10C8F000828081473DC9B5C9EF522FC4FC414146F2
:10C900002E84AA846393C70413860501A2878146F7
:10C91000C14503C7070003C507038507298F3305F2
:10C92000D600034505008506298FA38FE7FEE39215
:10C93000B6FE3044A2852685EFF07FD82285EFF041
:10C94000BFF985473E856F508FC1138507031D8E44
:10C9500081452295EF506FC17C40130700F8130604
:10C960000402A2972388E70255B73E858280EF52E2
:10C97000CFBC6D712E84B284AA85901028003689B0
:10C98000EFF0BFDA19E9D55705A050400C40280058
:10C99000EFF09FE66DD9FD142104E5F82C004A85DF
:10C9A000EFF03FF5814765D13E8551616F502FBB58
:10C9B000EF52AFB841112EC432C62C000546EFF03D
:10C9C0001FFB41016F50AFB9EF522FB701112A84FD
:10C9D0002EC602C802CA02CC02CEEFC06049B246DF
:10C9E0002A86A2850808EFF0BFFC1375F50F0561D4
:10C9F0006F50EFB6EF526FB47971B2872A84214637
:10CA00002308B10013051101BE853AC436C6EFC034
:10CA1000C01DB246930591013685EFF03FB72285E0
:10CA2000141035460C08EFF0BFF82A84224711E5B0
:10CA300021460C103A85EFC0401B228545616F509E
:10CA40000FB2EF528FAF7171AE84AA850A8532841E
:10CA5000EFF0BFC801C90A86A6852285EFF03FC660
:10CA6000814711E1C5473E854D616F504FAFEF5291
:10CA7000CFA91D712A8AB289BE8435468547130520
:10CA800011012E8CB68A3A8BC28C468D2308F10098
:10CA9000EFC0A01510100C085285231F0100EFF005
:10CAA0005FFA2A842DE9A147631BFD0693079005D1
:10CAB00091E0E5473546E2851305110113990A0116
:10CAC0002308F10013590901EFC020121357890000
:10CAD00093978A00D98F90080C085285231FF10084
:10CAE000EFF03FF62A8405E9A1E09387FA009183ED
:10CAF0001379F9003EC6631309004149668B8144EE
:10CB0000C14B854DB2476397970C6A868C0033857D
:10CB10005C01EFC0800D228525616F50CFA2930785
:10CB20009004C9F8A54779B7834701050947C14B68
:10CB30002308F10083471105A58FA308F10093870F
:10CB40002400814463EFFB02014714083386E600AA
:10CB50008C08B386E400BA95DA9683C6060083C5CE
:10CB600005000507AD8E2300D600E390E7FE4147A0
:10CB70006398E70490080C085285EFF09FEC35D5D8
:10CB800035A8B3069B00BA871008B305F6009008D5
:10CB90003E9603C506000346060085078506298ED6
:10CBA0002380C500E39277FF998F90080C08528587
:10CBB000BE94EFF01FE98947014749D52A84A1BFF8
:10CBC00090083E96034606001408BE962380C600D1
:10CBD000850779BFB2478504638B97128147180890
:10CBE000B306F70098083E973386F900034707001D
:10CBF000034606008507318F2380E600E39177FF27
:10CC000090080C085285EFF0DFE34DF93546E285D8
:10CC1000130511012308B101EFB0307D1397040112
:10CC20004183939784002183D98F10180C08528573
:10CC3000231FF100EFF0FFE051F181471018338717
:10CC4000F9003E960347070003460600B306FB00C3
:10CC50008507318F2380E600E39277FF75A01808DF
:10CC6000B306F70098083E973386F900034707009C
:10CC7000034606008507318F2380E600E3E127FFA6
:10CC8000CA876398770990080C085285EFF07FDB1C
:10CC900015F581479800B306F700900818103E97E5
:10CCA0003E9603470700034606008507318F238021
:10CCB000E600E39177FF3546E2851305110123086D
:10CCC000B101EFB0907213970401418393978400F0
:10CCD0002183D98F10180C085285231FF100EFF023
:10CCE0005FD6E31D05EC814710183387F9003E96A7
:10CCF0000347070003460600B306FB008507318F94
:10CD00002380E600E3E227FFC109410BE5BB814731
:10CD1000B5B79408BE9683C6060018083E97230050
:10CD2000D7008507B9BF638E062CEF421FFE5971ED
:10CD30002A84BE89B28B85473546130511022E8B96
:10CD4000468C4289BA8A368A2300F102EFB0F06934
:10CD500010180C10228523170102EFF09FCE631EDE
:10CD60000510A1476319FC0693079005639309001A
:10CD7000E5473546DA851305110293140A012300AD
:10CD8000F102C180EFB0706693178A0013D7840058
:10CD9000D98F90080C1022852317F102EFF07FCA7B
:10CDA00069ED639009049307FA00BD88918391E0CF
:10CDB000C144C207C183DE8C814A3EC6414DB247A1
:10CDC00063EAFA0C6286B3854B018810EFB0905F7E
:10CDD0004DC53D555DA093079004E39C09F8A54718
:10CDE00049BF834701050947C14C2300F10283472E
:10CDF0001105B3C7F900A300F10293872900814907
:10CE000063EFFC02814618103306D7008C08338785
:10CE1000D900B69556970347070083C505008506D8
:10CE20002D8F2300E600E390D7FE4147639AE70485
:10CE300090080C102285EFF0DFC035D53DA8B386F1
:10CE40003A01BA871010B305F60090083E9603C564
:10CE500006000346060085078506298E2380C50047
:10CE6000E39297FF3387EC4090080C102285BA9923
:10CE7000EFF03FBD8947014741D565616F40BFEC89
:10CE800090083E96034606001410BE962380C60006
:10CE9000850769BFB247850A93990A01939D8A0065
:10CEA00093D909016399570D85473546DA851305EE
:10CEB00011022300F10293D98900EFB01053B3EDB2
:10CEC0003D0190000C1022852317B103EFF07FB7CE
:10CED0004DF58147A68963E6970626860C084A85A4
:10CEE000EFB0B05081471810B306F700100898084B
:10CEF0003E973E9603470700034606008507318F9D
:10CF00002380E600E3E197FE639DA90590080C10DD
:10CF10002285EFF01FB335F181479810B306F70073
:10CF2000900818183E973E960347070003460600F0
:10CF30008507318F2380E600E391A7FF4109C10CEB
:10CF4000BDBD18089000B306F7003E963387FC007D
:10CF500003470700034606008507318F2380E6005C
:10CF600095BF98084E97034707001C10CE97238063
:10CF7000E700850951BF85473546DA85130511025B
:10CF80002300F10293D98900EFB03046B3ED3D01A3
:10CF900090000C1022852317B103EFF09FAAE31E27
:10CFA00005EC814718089000B306F7003E963387DA
:10CFB000FC0003470700034606008507318F2380E6
:10CFC000E600E391A7FF41460C084A85EFB0F04127
:10CFD00081471810B306F700100898083E973E9650
:10CFE00003470700034606008507318F2380E600CC
:10CFF000E391A7FF90080C102285EFF09FA41DDDA0
:10D00000ADBD7D558280EF425FD301112A842E850C
:10D0100093055100328902C002C202C402C69304C1
:10D020007400EFF0AFD61D46A68513059100EFB052
:10D03000D03B10088A854A85EFF0BFA019ED930711
:10D040001400180883C60700034607008507050774
:10D05000B18EA38FD7FEE397F4FE05616F403FD0FA
:10D06000EF421FCC2E848C414111AA898387150081
:10D070003289914463D30700A1449797FF1F938798
:10D08000A70D9C43B1C3B5CE8D472310F10083C7D4
:10D0900025004A852301F10083C73500A301F10073
:10D0A00083C745002302F10083C75500A302F100A6
:10D0B00083C7650093059100A30301002303F100DA
:10D0C00023040100EFF08FCC0C404A860A85EFF074
:10D0D0000FCE0328040083564400A6881D0881470C
:10D0E0000147E51642868A854E85EFF05F982A89CA
:10D0F00009E5A6852285EFB0FFB24A8541016F4060
:10D100007FC54A860A85EFF08FCA7DBFEF425FC1B7
:10D110002E848C414111AA8983871500328991445C
:10D1200063D30700A1449797FF1F9387E7029C43AF
:10D13000B1C3A5CE8D472310F10083C725004A85D2
:10D140002301F10083C73500A301F10083C7450027
:10D150002302F10083C75500A302F10083C76500D5
:10D1600093059100A30301002303F10023040100B0
:10D17000EFF0CFC10C404A860A85EFF04FC38356CB
:10D180004400032804008A85858EC2061D08C182DA
:10D190002312D400A68881470147E51642864E85B2
:10D1A000EFF07FB841016F40FFBA4A860A85EFF081
:10D1B0000FC0C9B7EF427FB8B335B0000111850584
:10D1C0002A891315F601336515012308B10093056B
:10D1D000110136843AC632C03EC442C2EFF00FBBE2
:10D1E000A2471248425593D68700230BF1009305BE
:10D1F000910193578800A30AD100A30BF100230CDF
:10D200000101EFF0AFB83247024603280400B337FC
:10D21000E000835644009207914411C2A1444A851C
:10D22000A68842860C08EFF09F842A8909E5A68526
:10D230002285EFB03F9F4A8505616F405FB2EF42A4
:10D240003FAE01113EC68647B335B0008505AA89B9
:10D250001315F6015D8D2308B10093051101368485
:10D260003A89B28442C446C2EFF04FB22248924893
:10D27000164593578800A30AF1009305910193D7AF
:10D280008800230B0101A30BF100230C1101EFF027
:10D29000EFAF3247104083564400B337E0009207A7
:10D2A00003280900914891C0A1480C084E85EFF071
:10D2B0009FA7AA8411E5835544004A85EFB09F9645
:10D2C000268505616F401FA9AA959307F00F17F7F0
:10D2D00000001307278A6317B50013C5F7FF1375FE
:10D2E000F50F828005058346F5FFB58FBA9783C792
:10D2F0000700D5B70357450014419307F00F17F601
:10D3000000001306268736974207418313950601CE
:10D310004181631BE500AD8FB29703C5070013057C
:10D3200015F3133515008280850603C5F6FFA98F16
:10D33000B29783C70700D9BFEF423FA0B2873684B8
:10D340002E86BA86AA853E85BA84EFF06FE6634BD7
:10D3500005002285EFB0D0312A86A686A2852685D3
:10D36000EFF00FE56F40BF9FEF429F9B5D712A8BEF
:10D37000AE8A17E500001305657D2C00B284368A5D
:10D38000BA893E89EFF04FE42A8459E534104146CA
:10D39000DA852800EFF0CFE12A843DED8547A3032D
:10D3A000F100A6C2930771002408BEC4A686854773
:10D3B0000D462C18281002DC02DED6C0BEC6EFF0E7
:10D3C0000FDB2A8431E983477102A6860D4693F765
:10D3D000F7072300FA00C1473EDE2C1889472810C2
:10D3E00026DCA303F100EFF08FD82A8415E541462F
:10D3F000A6854E85EFB0607F8D47A6860D462C181A
:10D400002810A303F100EFF08FD62A8411E54146DE
:10D41000A6854A85EFB0607D228561616F409F934C
:10D42000EF42BF9197D700009387070C984383C7BB
:10D43000470079712A89AE8417E5000013058571CC
:10D440000C083AC42306F100EFF00FD82A8415E542
:10D4500014104146CA850808EFF08FD52A8411EDD3
:10D46000140815462C000810EFF08FD42A8411E51B
:10D4700021462C082685EFB04077228545616F4014
:10D480001F8EEF429F8B97D700009387E7059C473D
:10D490007971AA842E8417E500001305256C0C0809
:10D4A0003EC6EFF06FD20DE514104146A685080880
:10D4B000EFF00FD011ED140811466C000810EFF0DA
:10D4C0002FCF19E58347F10193F7F7032300F40009
:10D4D00045616F40DF88EF425F863688A14881470B
:10D4E0000147E546EFF0AFD86F407F87EF42FF84FA
:10D4F0003688A14881470147E546EFF0DF826F405B
:10D500001F86EF429F8301112A842E850C0832C6A4
:10D51000EFF08FCB19E9324797E6000093868662D9
:10D520001008C1452285EFF03FE105616F403F8360
:10D53000EF42BF804111C1472EC032C48A850946DF
:10D540003EC23EC6EFF0AFC241016F405F81EF4285
:10D55000CFFE4111AE8613061009AA850A8502C0C6
:10D5600002C202C402C6EFF0AFC441016F402FFFF8
:10D57000EF42AFFC328797E600009386A65E2E86C8
:10D5800093050002EFF05FDB6F406FFDEF42EFFAB3
:10D590007971C1472ACC2ED032D42C080D462800F0
:10D5A0003ECE3ED23ED602C402C602C802CAEFF048
:10D5B0000FBC45616F40AFFAEF422FF80111AA840A
:10D5C0002E8417E500001305655A8A85EFF0CFBF5A
:10D5D00005E514084146A6850A85EFF06FBD09ED03
:10D5E0008347E1010347F101A207D98FCA07C98325
:10D5F0006177D98F2310F40005616F404FF605C99C
:10D60000EF42AFF39787FF1F938787629043978519
:10D61000FF1F938525621785FF1F1305655DEFB01A
:10D6200080091785FF1F1305A55C6F404FF3178511
:10D63000FF1F1305E55B82809DC5EF420FF09787C2
:10D64000FF1F9387E75E944301112E840A86978516
:10D65000FF1F9385255EEFB0800A0A85029401457D
:10D6600005616F40CFEF7D558280EF420FEDEFB047
:10D6700080149787FF1F23ADA75A17F5FFFF1305E7
:10D6800025F8EF90D0406F408FED1787FF1F1307ED
:10D69000675C9317150008433E95FD572310F5006E
:10D6A0008280EF428FE92A84084019E16F402FEB16
:10D6B0001C4158401CC06313E5005CC08347550003
:10D6C00023200500F99BA302F500EFB0EFF9E9BFB5
:10D6D000EF420FE59787FF1F9387C75998432A8426
:10D6E00011CB8347350093F7070289C7035505001F
:10D6F0008945029713054401EF90101383550400E8
:10D700000355E400EF20701B485809C5EFB0CFF572
:10D71000232A040213058403EFF0BFF88144B149C2
:10D72000EFA0FF9A63C5A4028347340023200404BA
:10D7300093F727FCA301F4000048EFA05F9A1316AB
:10D74000150081452285EF404FE26F40AFE0B3877F
:10D7500034030329040385043E994A85EFF07FF4DE
:10D760002304090075BF8347350093F7070299E347
:10D77000014582808357E500E39CB7FEC167FD1732
:10D780006316F600054582800545B9A0EF42EFDA41
:10D7900093170601C187B2842A8401496359F002B4
:10D7A000835705008DCB01456367F6000345840070
:10D7B0003E953325A6001375F50F39A81C4813179D
:10D7C0001900BA9783D70700E38097FC0509EFA0FB
:10D7D0001F91E345A9FE01456F406FD8EF424FD43A
:10D7E000AE89AA84EFA07F852A84EFD0BFAAAA863B
:10D7F00001471306840197050000938545E91785C5
:10D80000FF1F13056545EFA0AFD52A8921CD8C44B4
:10D810001304C50022859E0593F50508EFB00FC5DA
:10D82000CC4083877400E18163D1070493E5050848
:10D830002285EFB0AFC30D46938544002285EFB03B
:10D840000FC183D504002285EFB0EFC583D5240036
:10D850002285EFB04FC503D6490083A50900228574
:10D86000EFB0EFBE4A856F40EFCE93F5F507C9B72D
:10D87000EF42AFCC01112A84328532C6EFB06FB4CB
:10D88000EF903F91835704001787FF1F1307075638
:10D890003246231BF100930700F8A30DF1001C474B
:10D8A0001843231AA1008983858BB307F740B285FB
:10D8B00048083ECE231C0100230D0100EFF01FF2AB
:10D8C00005616F40CFC9EF42AFC50041014529CC8A
:10D8D0009304C40026853289AE89EFB08FB2954596
:10D8E0002A8A2685035B0401EFB02FAF2685EFB0AF
:10D8F0002FC68D45AA8A2685EFB02FAE2685EFB0BC
:10D900002FC55C48420A135A0A01D2975CC42318F7
:10D910006401814763983A0146054D8133062541EC
:10D920009337160013F5F70F6F40CFC2EF426FBE6B
:10D9300089692A8BAE8B328AB68A81440144314C84
:10D94000FD19EFA0CFF863C9A400EFA04FFB018D34
:10D9500033B5AA006F406FBF3389840383270B0060
:10D960003E9963170A008347890085043E94D1BF1E
:10D9700003560A00DE854A8533F6C900EFF0BFF48E
:10D980007DD10545C1BFEF424FBB01112A847C0008
:10D990000355E5003ECAB70707003ECC7C003ECEEB
:10D9A000EF10303D2A8985454808EFB0EFC1994511
:10D9B0004808EFB02FA7AA844A85EF10B03D238016
:10D9C000A4009787FF1F938767429C434166130615
:10D9D00006F09396870113D78701558F93D687005A
:10D9E000F18E558FA207B706FF00F58FD98F11462C
:10D9F0002C00138514003EC4EFB0201F5008A382F2
:10DA0000040089452285EFF0BFE609C9AA85130500
:10DA10008403EFB0EFBB3C4085073CC005616F401D
:10DA20000FB4EF428FB1EFA08FED2A840504EFA071
:10DA30000FEC3305A402F14791453305F502EF10D1
:10DA4000207B01E565556F408FB19787FF1F23ABA2
:10DA5000A720EFA0CFEA2A840504EFA04FE9330501
:10DA6000A40289450605EF10A07869DD9787FF1F9E
:10DA700023A2A71EEFA0AFE82A840504EFA02FE79A
:10DA80003304A4029787FF1F2398871CEFA02FE77A
:10DA90002A84EFA0CFE5930714003385A702978768
:10DAA000FF1F239CA71A97E700009387E7CF1787EC
:10DAB000FF1F2327F71A014579B7EF426FA6AA8403
:10DAC0002E8901449789FF1F93894932130A8006E2
:10DAD000EFA0EFE16345A40001456F40AFA7330518
:10DAE000440383A709024A86A6853E95EFF0BFC787
:10DAF00019E10504F1BF0545CDB7EF428FA1AA8A10
:10DB00002E8BB28B368C3A8A814401448149978CA2
:10DB1000FF1F938CAC2D130D8006EFA04FDD63C764
:10DB2000A40011E085494E856F402FA23389A403DC
:10DB300083A70C025E86D6853E994A85EFF0BFC268
:10DB400019CDEFA0CFDB0544636B4501D286628619
:10DB5000DA8513050903EFF07FDD11C185498504DE
:10DB60006DBFEF42EF9BC16441112A89014497893F
:10DB7000FF1F9389A927130A8006FD1436C632C4F5
:10DB80002EC2EFA0CFD692452246B2466346A400ED
:10DB9000014541016F400F9C3305440383A70902EF
:10DBA0003E9509C683473500C18B9DC791C6834703
:10DBB000350093F707028DC3630699008357E5008C
:10DBC000639C27010357050001CB63E7E50083470A
:10DBD0008500BA97E3CFF5FA05044DB7EF424F94AD
:10DBE000C1642A8901449789FF1F93892920130A58
:10DBF0008006FD14EFA0AFCF6344A4006F408F9563
:10DC00003305440383A709023E958357E5006388E3
:10DC100097006304990063942701EFF07FAB05043C
:10DC2000D1BFEF428F8E89692A8AAE8A328BB68B3A
:10DC30008144178CFF1F130C6C1B930C8006314D15
:10DC4000FD19EFA0CFCA63C4A4006F40CF8F338902
:10DC5000940383270C028355CA015A863E994A854C
:10DC6000EFF07FB005CD814D05A03384AD03832750
:10DC7000090303D60B00D68533F6C9003E942285EE
:10DC8000EFF07FC419E5850DEFA06FC4E3CFADFCC5
:10DC900031A02285EFF0FFA023040400850455B7CE
:10DCA000EF422F874169AA8A014A178BFF1F130B86
:10DCB000EB137D19C14B054CEFA06FC36344AA0061
:10DCC0006F40AF8893098006B3073A0383290B029C
:10DCD000BE9983D7E900638C270163842A01639886
:10DCE000570103A4890311E44E85EFF0DFC9050A4B
:10DCF000E1B783570401639977079304C40026852D
:10DD0000EFA03FF085452A8D2685835C0401EFA0B6
:10DD1000DFEC2685EFA0FFFF62056185635F0502EA
:10DD20008D452685EFA07FEB89452685EFA0FFEA8C
:10DD300089452685EFA07FEA85452685EFA03FEB44
:10DD400083470500094793F7F7076398E70099456C
:10DD50002685EFA0DFE9A30285014848337D2D0128
:10DD6000231894016A9548C40040B5BFEF32FFFC08
:10DD700037E404008327041D82979787FF1F83C71A
:10DD8000E7F31755FF1F1305E53CA300F5008327B4
:10DD9000441C82978327841C81461306F00F81451B
:10DDA000014582976F30BFFB1787FF1F130707E1FD
:10DDB00018439785FF1F83C565F09787FF1F9387DB
:10DDC00067EE83468703034697036397D5009787DB
:10DDD000FF1F2385C7EE828083C587010347A70302
:10DDE0006317B6009787FF1F238AE7EC828003C67C
:10DDF00087016317C7009787FF1F2381D7EC8280B5
:10DE000083C68701130750026319D7009307600286
:10DE10001787FF1F2304F7EA828083C68701130652
:10DE200060026315D60093077002DDB783C78701D0
:10DE300055BF9787FF1F9387E7E6D44B0947638554
:10DE4000E608EF329FEF1789FF1F1309E9E23E84CE
:10DE500083470900918B9DCFB7E4040083A7041D7D
:10DE6000829783A7441C1785FF1F130565E18297DE
:10DE700083A7841C81461786FF1F034666E28145FF
:10DE80000145829721C183470900ED9B1787FF1F3A
:10DE90002304F7DE8347040093F7F70F85C7914704
:10DEA0001787FF1F232AF7E0EFF05FECEFF0DFEFBB
:10DEB000B7E70400BC4F414691451785FF1F034556
:10DEC000E5DE82976F30BFE98280EF321FE78D4732
:10DED00041116304F504C5476306F50285476310E5
:10DEE000F5029787FF1F238DA7DCB7E70400BC4B23
:10DEF000930500101785FF1F034545DB82974101FD
:10DF00006F30FFE585471787FF1F230BF7DAB7E769
:10DF10000400BC4B93050020F1BF9787FF1F938738
:10DF200067D8D44B1147638DE600B7E7040083A799
:10DF3000071D8297B7E70400BC4B930500045DBF43
:10DF400005491787FF1F232927D783C7070032C634
:10DF50002E8493F7F70FC5D7B7E4040083A7041DF9
:10DF60007D141374F40F8297E37689FCB2459947C8
:10DF700003C61500E3F0C7FCFC4409061785FF1F24
:10DF8000130545D48297BC48930500081785FF1FE9
:10DF90000345C5D1829779BFEF323FDA1787FF1F5C
:10DFA000130747D04047184B1C409786FF1F23A1FB
:10DFB000F6D06316E4001787FF1F232DF7CE130555
:10DFC00084FEEF907FF3035564FFEF903FC6EFA010
:10DFD000BFE96F30DFD8EF325FD69787FF1F938797
:10DFE00067CCD84BDC4799C3EFF01FFB85471787F9
:10DFF000FF1F2323F7CC9787FF1F938727BC9C43E2
:10E00000930500021785FF1F034545CA83C7870391
:10E010001787FF1F2304F7CAB7E70400BC4B82979A
:10E020006F30FFD39787FF1F23A0A7C88280EF32EE
:10E030003FCF37E404007C4CA1451785FF1F034503
:10E04000E5C682977C48A1451785FF1F034505C695
:10E050009784FF1F938404C58297DC4489E7EFF01F
:10E060005FDD6F303FCF03D567FFEF903FBCAA89DC
:10E070007DD5D84891476310F7027C4C91451785B0
:10E08000FF1F0345A5C282977C4891451785FF1F56
:10E090000345C5C1829703A9490103D409018947F2
:10E0A000B7E904001787FF1F2328F7C083A7091DBE
:10E0B00021044204829783C784011755FF1F13056B
:10E0C000650961191757FF1FA306F70883A7491CA5
:10E0D000418082979787FF1F238407BE83A7C91CAF
:10E0E000814609469375F40F4A85829711E997870F
:10E0F000FF1F83C727CD89C79740FF1FE780407761
:10E10000B7E70400BC4F2146A1451785FF1F034513
:10E11000E5B98297B9B7EF325FC293F705200111D5
:10E120002E8481CBEFF03FEB1345042005616F3067
:10E130001FC393F70510A9CB9784FF1F938484B660
:10E14000DC48EFF07FC61787FF1F130727A7184388
:10E1500083C78401034787036316F700DC4499C330
:10E16000EFF09FE385471787FF1F2327F7B4B7E733
:10E170000400BC4B930500021785FF1F034505B340
:10E180008297134504105DB793F70508ADC79787CD
:10E19000FF1F83C737B3E91719469785FF1F93857C
:10E1A00085B21305D10093F4F70F1789FF1F0349B8
:10E1B00069B1EFA0902393970401C1831787FF1FD4
:10E1C0001307C7B0231DF100231CF1009787FF1F21
:10E1D000938747AD3ACE3ACAD8432306010009CB0C
:10E1E000DC439315890154080D46E1856800829748
:10E1F0001345040825BF93F72500B1CF9787FF1F6C
:10E20000938747AAD84B89476306F7029787FF1F72
:10E2100083C787A613F7270011EF918B99CFB7E734
:10E220000400BC4F1306000A89451785FF1F0345EC
:10E23000E5A7829713452400D5BD9787FF1F9387D5
:10E24000E7979C4383C787031787FF1F2308F7A619
:10E25000EFF0FFDDC5B793F7050291C7EFF03FDDA3
:10E2600013450402E1B593F7850091C7EFF0BFD6DF
:10E270001345840065BD93F7150091C7EFF07FBB90
:10E280001345140065B593F7450091C7EFF07FBAC9
:10E290001345440061BD93F7050485C39787FF1FAD
:10E2A00083C747A081CBEFF07FAC91471787FF1F53
:10E2B0002324F7A01345040495BD93F705010145F8
:10E2C000E38607E69787FF1F9387C79DD84B914743
:10E2D0006310F7049787FF1F9387079A9C4313D710
:10E2E00027008583D98F858B91E7B7E7040083A743
:10E2F000071D8297B7E70400FC4F91451785FF1F64
:10E300000345C59A829785471787FF1F2326F79AEB
:10E310001345040121BD9787FF1F2385A7AA82808B
:10E32000EF32BFA19787FF1F23A407989787FF1F8E
:10E3300023A2079885471784FF1F13042488178793
:10E34000FF1F232BF7961C4083C787031787FF1FE8
:10E350002306F796EF90FFDF39C19757FF1F23AFD2
:10E36000A7DE1C4017050000130525DB83C78703C4
:10E370001787FF1F2304F7941757FF1FA30CF7DC21
:10E380009787FF1FA3800792B7E7040083A70708BA
:10E3900082979787FF1F238BA7906F305F9CB7C72B
:10E3A000898E938767ED1757FF1F2329F7DA55BF2B
:10E3B0001787FF1F0347078F795555E39787FF1F7F
:10E3C0009387478E03C7170005079786FF1FA38B08
:10E3D000E68C03C717008D463377D7029786FF1F59
:10E3E000A382E68C83C617001777FF1F1307077DEC
:10E3F000184393F6F60FA9EA834787031787FF1F91
:10E40000230EF78A85471787FF1F230DF788978705
:10E41000FF1F938767869C430145998BA9E3EF32E1
:10E42000DF9137E404007C48C1451785FF1F034591
:10E43000E58782973C4885451785FF1F034505877B
:10E44000829701456F30BF9183C71700854663955A
:10E45000F600834797035DB78347A70345B78280DC
:10E460009787FF1F83C70784A1CBEF321F8D37E447
:10E4700004009787FF1F238707827C4885451785FF
:10E48000FF1F0345A58282977C4C91451785FF1F8E
:10E490000345C58182977C4891451785FF1F034539
:10E4A000E58082973C48C1451785FF1F03450580DD
:10E4B000829701456F30BF8A79558280EF32FF879E
:10E4C0002A84035565FFEF906FF69777FF1F9387B8
:10E4D000677DD847BE841DEBEFA05F989C48232042
:10E4E00004008DEB9777FF1F23A6877C9777FF1F8C
:10E4F00023A0877CB7E70400BC4B89451775FF1F35
:10E500000345C57A829701456F307F85630A87008E
:10E510001843D1B780C39777FF1F23AD8778D9BF42
:10E520007955DDB7EF327F819787FF1F9387C789C2
:10E53000884323260500232405005105EF80D02EB3
:10E540006F30FF81EF326FFF1784FF1F1304C48702
:10E550001C40411189CF9C472302B5002AC61CC12B
:10E56000EFF05FFC1C409C4B99C332458297410100
:10E570006F30EFFEEF326FFC4111444D3285328433
:10E580002EC6EFA00FF92AC42285EFA0EFF903A849
:10E590004400630C0800B2458357440018402246EB
:10E5A00083D54500AA862685029841016F302FFB4E
:10E5B000EF32AFF8404D1DC408C0970500009385A9
:10E5C000E50213054401EF8090189777FF1F9387AA
:10E5D000A77F9C43014589E79777FF1F23A6877E86
:10E5E0006F30EFF77D55EDBFEF322FF50111680069
:10E5F0009305F00F02C602C802CA02CC02CEEFF0A9
:10E600007FF405616F30AFF59777FF1F9387C77B66
:10E610009C43D847A1679D076311F702EF32EFF1E2
:10E6200001113285EFA0EFEE230AA10081456800B9
:10E63000EFF05FF105616F308FF282809777FF1FF7
:10E64000938787789C43D847A167938777036311A3
:10E65000F702EF328FEE01113285EFA08FEB230A24
:10E66000A10081456800EFF0FFED05616F302FEFED
:10E6700082809777FF1F938727759C43D8479547DC
:10E68000631CF702EF326FEB011132853284EFA089
:10E690004FE8230AA1002285EFA00FE98357440029
:10E6A000231BA10081453ECC1C4068003ECEEFF00C
:10E6B0007FE905616F30AFEA8280930785FF89CFDC
:10E6C0008327C5FF91CBDC4B81CBEF320FE70325CE
:10E6D00085FF82976F30AFE88280EF320FE62A84A1
:10E6E0003285EFA00FE3BD4763EBA7001844937793
:10E6F000F5000345B70041995D8DA305A7006F3074
:10E700000FE6EF328FE301117C003ECAB707070026
:10E710003ECC7C003ECE5C4D8DCF2A841385870095
:10E72000AE84EF807004A1652A899D054808EF80BA
:10E73000FFBD9305803EB345B902480893F5F50F38
:10E74000EFA0CFD2014781465008A6852285EF80F1
:10E750007FDC05616F30AFE0EF322FDEEFF07FFA44
:10E760006F30EFDFEF326FDD01117C00AE843ECA07
:10E77000A165B70707002A843ECC48087C00938532
:10E7800075033ECEEF809FB81C44480883C5B70090
:10E79000BD89EFA0AFCD500801478146A6852285EF
:10E7A000EF805FD705616F308FDBEF320FD92A849E
:10E7B000AE84EFF09FF2A6852285EFF0BFFA6F30AE
:10E7C0000FDAEF328FD7EFF0FFF96F304FD9EF321A
:10E7D000CFD60329C5014111630409022A84328579
:10E7E000B284EFA00FD32AC62685EFA0EFD38327EC
:10E7F00049002A8691C7DC4781C7B24522858297A6
:10E8000041016F30CFD5EF324FD3444D81CC2A84B4
:10E810003285EFA06FD1DC40AA8589C79C4799C398
:10E82000228582976F30AFD3EF328FCF032AC50195
:10E83000411163030A062E89AA84954532853284E4
:10E84000EF80DFAC85452285EFA0CFBDAA89CA85C0
:10E850002285EFA0EFC283274A009DC7DC438DC706
:10E860002285EFA0AFBA83274A00104083564400A8
:10E87000DC437115A307A100B2961307F1004E8681
:10E88000CA852685829701C52380090031A083456A
:10E89000F1002285EFA00FB941016F30AFCBEF320D
:10E8A000CFC965711C083EC2B70780013EC41C0871
:10E8B00032893EC62A84AE84EFF07FF14A85EFA00C
:10E8C000AFC68357A10089CFAA8550002285EFF0FB
:10E8D000BFF5014781465000A6852285EF809FC382
:10E8E00059616F30CFC7EF32AFC365711C08832900
:10E8F000C5013EC2B70780013EC41C082A84AE840D
:10E9000032893EC6EFF03FF0638409024A85EFA0EA
:10E91000AFC18357A100AA8581CF50002285EFF0B7
:10E92000BFF0014781465000A6852285EF809FBE3B
:10E9300059616F302FC2EF324FC065711C083EC263
:10E94000B70780013EC42A841C0832853EC6AE84C7
:10E95000EFA08FBD8357A10089CFAA8550002285E3
:10E96000EFF09FEC014781465000A6852285EF809D
:10E970007FBA59616F30AFBEEF322FBC444D91E882
:10E980008347450093B71700B307F0403E856F30CB
:10E990000FBD1845FD577DDB9707000093870703E0
:10E9A0002A845CCB97050000938565D1138584008C
:10E9B000EF80E05980C003474400814761FB17772F
:10E9C000FF1F23259740D9B7EF328FB58329C501A3
:10E9D0004111032985008147638B0908032409013C
:10E9E00091452A8A2285EF807F9285452285EFA076
:10E9F0006FA38945AA8A2285EFA0CFA2AA84EF80BF
:10EA00009F9683A749002A8B9DC79C438DC722856B
:10EA1000EFA0CF9F83A74900A306A1001040835613
:10EA200044009C431307D100B296D6851306E1003B
:10EA30005285829709CD83570B002380F400A18370
:10EA4000A380F40023800A00A306010029A88357AD
:10EA5000E10022852380F4008345D100A183A380B7
:10EA6000F400EFA02F9C8347D100B337F000034799
:10EA7000B900920701453D9BD98FA305F9004101DB
:10EA80006F304FADEF326FAB41111DE99777FF1F2C
:10EA90009387C733804305C80440130984009DC58C
:10EAA0005C4099C79C4B89C726852EC68297B24584
:10EAB0009307803EB385F5024A85EF80605521A01B
:10EAC000404DAA8479F841016F306FA94A85EF80E3
:10EAD000A0555C40EDDBDC4BFDD726858297E5B782
:10EAE000EF32AFA52A843285EFA0AFA2AA85228596
:10EAF000EFF05FF96F30AFA6EF322FA42A84AE8417
:10EB0000EFF01FFEA6852285EFF0BFBF6F302FA567
:10EB100008413355B50005898280EF320FA2177482
:10EB2000FF1F1304A42C1C5C0111231701008D830B
:10EB3000858BA303F1008327040B231801002319FD
:10EB4000010003D7C7013ECA3C002314E1007D57F2
:10EB50002315E1000357C4023ECC02CE2316E10088
:10EB6000EF802FE38357E101231EA10093F707E015
:10EB700093E71710231FF1009777FF1F83C7A7297B
:10EB800085C305470145638AE7008347840393E70C
:10EB900027001777FF1F2307F72805616F302F9C89
:10EBA000814717D700001307271C854613067100FD
:10EBB00085454808EF70E04B6DF183478403F59B72
:10EBC0001777FF1F2300F72685471777FF1F2304BA
:10EBD000F724E1B7EF326F93977DFF1F938D0D21DF
:10EBE00003A6CD0639712A89814781449306000224
:10EBF0003357F600058B01C7850493F4F40F85079E
:10EC0000E398D7FE83A70D0B2317010223180102F7
:10EC100003D7C7013EDA3C102314E1027D572315C8
:10EC2000E10203D7CD023EDC231901022316E102E3
:10EC300002DEEF800FD68357E103231EA1020145B8
:10EC400093F707E093E71710231FF1029777FF1F51
:10EC500083C7671CA9EF9777FF1F83C7B71C3EC602
:10EC60009779FF1F938989180144014D9D4A054BEF
:10EC7000954B177CFF1F130CAC1E977CFF1F938CCA
:10EC8000AC1D03DAC90563090A00EA856314590358
:10EC90006685EFF0FFE71DC1050DA1478909E31265
:10ECA000FDFE2DE09777FF1F23AA071A014521617A
:10ECB0006F306F896285EFF0BFE579DD3247B3874A
:10ECC0008400E3F0E7FE9C001306140006043E9463
:10ECD00013178A0093578A00D98FC207C183A30EE6
:10ECE000F4FCA183230FF4FC03A70D07B317AB01BA
:10ECF000D98F1777FF1F2323F71663047601328419
:10ED000061BF15449777FF1F83C7C710138717008C
:10ED10009776FF1F2380E61093161400230EF10050
:10ED200017D7000013074704814785067008CA8576
:10ED30004818EF700034E34705F68347C1010545E5
:10ED40001777FF1FA308F70C9777FF1F2385270D61
:10ED5000B9BFEF22FFFC0111AA892E84EFD0EF9CEE
:10ED60002A899774FF1F938464086399090A9C5C3D
:10ED7000414793F707036393E70A1777FF1F03479A
:10ED8000D709894763ECE70883A7040B2317010021
:10ED90002318010003D7C7013ECA3C002314E10039
:10EDA0007D572315E10003D7C4023ECC231901008F
:10EDB0002316E10002CEEF80CFBD231EA100EFC0DD
:10EDC0006FCD8357C101230FA100914613D7870050
:10EDD000A207D98F2312F1009777FF1F83D7A704CB
:10EDE00013D78700A207D98F2313F10017D700008C
:10EDF000130707F78147500095454808EF706027D3
:10EE000005889317240003C484036D985D8C97775D
:10EE1000FF1F2389870005616F20DFF3EF70B07853
:10EE20001775FF1F13058500EF80002083A7040BD3
:10EE30009775FF1F83D545FE03D5C701EF10E02767
:10EE40009777FF1F83C707FE93F60702014789E6FE
:10EE50001777FF1F035747FC9776FF1F2396E6FCA3
:10EE60001777FF1F130747F7184309CBC18B99C7C3
:10EE700089451775FF1F035525FA02979777FF1FDE
:10EE800023AC07F89777FF1F238707F89777FF1FB3
:10EE900023A407FC9777FF1F23A207FC9777FF1F88
:10EEA00023A007FC83D7840393F7270C93E717006D
:10EEB0001777FF1F2318F7F683572903A18B99C3F0
:10EEC000EF70E03F11C49777FF1F23A307F4A1B7AA
:10EED0008D471777FF1F232DF7F2EF902FA593058E
:10EEE000803EB305B5021775FF1F130525F4EF80AB
:10EEF000201215B79777FF1F938747EFD85325C781
:10EF000091C99777FF1F238807F09777FF1F23A7E3
:10EF100007F48280EF227FE283C7F70241112EC6F9
:10EF200085071777FF1FA30AF7EE9777FF1F239E2A
:10EF3000A7EE9D471777FF1F232CF7ECEF900F9E4E
:10EF40002A84EF90AF9DB24501E5EF902F9DAA85F1
:10EF5000B305B4401775FF1F130545EDEF80400B57
:10EF600041016F20DFDF82809777FF1F938707E8DB
:10EF7000D85331C7EF227FDC03C7F7020507977626
:10EF8000FF1FA38CE6E811CD8C5F0D4701458981F9
:10EF900085899776FF1F23ADE6E6EFF09FDB6F20B4
:10EFA0001FDC85479305C0441775FF1F130505E84F
:10EFB0001777FF1F232EF7E4EF808005CDB78280FF
:10EFC000EF22BFD71777FF1F0347E7E48547631E8C
:10EFD000F7009777FF1F938767E183C7870393C77E
:10EFE00087001777FF1F230FF7E21775FF1F130521
:10EFF000E5E3EF806003EF807FEF99471777FF1F0E
:10F000002328F7E09777FF1FA38907E09777FF1F73
:10F01000238307E0EF90AF8F930740063305F50297
:10F020009777FF1F23ACA7DE6F207FD39777FF1F53
:10F0300083C747DFC18B99C7EF223FD0EFF0FFAD09
:10F040006F20FFD1695582809777FF1F938707DA7A
:10F05000DC5381CBEF227FCE8545EFF09FCF6F2031
:10F060001FD082801777FF1F130747D801468146BC
:10F07000BA852148631E06019DCA2390A60083C756
:10F08000850393E717001777FF1F230DF7D805A017
:10F090008357C705631DF502F8598547B397C70025
:10F0A00093C7F7FFF98F1777FF1F232BF7DA9C5DC4
:10F0B0009183858B85C79777FF1F83C7C7D599EF46
:10F0C000EF22BFC71D45EFF0FFB06F205FC981E69B
:10F0D00099E39306C7050506090769BF8280EF22F9
:10F0E0005FC38605AA84B309B500977AFF1F938A88
:10F0F000AAD6054B977BFF1F938B4BD6214C63946D
:10F1000034039777FF1F938767CE9C5F9183858B2E
:10F1100089CB9777FF1F83C707D081E72145EFF0A1
:10F120007FAB6F209FC203DA0400630B0A041779D8
:10F13000FF1F1309A9CB0144CA8C8357C905639DDE
:10F140004703A2855685EFF0BF9C11E5A2855E8539
:10F15000EFF01F9C05C903A74C07B3178B00D98F8D
:10F160001777FF1F232EF7CE83C78C0393E7170073
:10F170001777FF1F2308F7CA05040909E31F84FB5B
:10F180008904B5BF231E0904C5BF1777FF1F0347B6
:10F1900087C88547631AF700EF223FBAEFF05FE2B6
:10F1A000EFF0BF976F20BFBB828081478545130674
:10F1B000000293861700B397F500E98F13F7F60F57
:10F1C00089E7B687E397C6FE01473A858280FD4707
:10F1D00085457D56B396F50013871700E98E1377A2
:10F1E000F70F89E6FD17E397C7FE01473A8582804E
:10F1F00089E901473A85828001473A8541016F20BC
:10F200001FB6EF229FB341112AC62E852EC4EFF000
:10F21000DFF9A2457D158547B397A700E39EF5FC6E
:10F2200032469377360099C3719A11069777FF1F7C
:10F23000938787BB94433E871778FF1F130808BA4C
:10F2400089EA832708009107F19B9776FF1F23AD7A
:10F25000F6B8032588001843B307A700B3F7B70231
:10F26000B387F540FD15FD8D83274800AA95B306A9
:10F27000B600E3F3F6F8E371D5F82E979777FF1F02
:10F2800023A2D7B63DDB3A858145EF201FAE2A8702
:10F29000ADB718419777FF1F938747B423A40700A2
:10F2A00098C35841D8C39777FF1F23AF07B2828016
:10F2B000EF221FA7AA8401441779FF1F130909B37E
:10F2C0009309400EEF807FD56345A40001456F2070
:10F2D0007FA8330534038327090B3E958357C50167
:10F2E000E38797FE0504F9BFEF22BFA29779FF1FBE
:10F2F0009389C9AF3E84BA848347060003A70900F7
:10F3000041119D83058B3D8F83C74401AE8A2A89B5
:10F31000F99BD98F238AF4001C44B685231204007C
:10F320001CC02285328A36C6EF90DF8FB246D28566
:10F330003686EF90900BDC4883A509000840858B4A
:10F3400056869D8DEFD03FCC61E918407D558347AF
:10F35000570003476700A207D98FC207C1872394CC
:10F36000F4006358F00A83C7440193F70703B5CB51
:10F37000D0489377160003A609001D8E9777FF1FCC
:10F38000938787DD9C43ADEB814641A003A70B002B
:10F3900093172A00BA971840944383475700834530
:10F3A000670033F65601A207CD8F6311F60283473B
:10F3B00037000346470003472700A207D18F4207C3
:10F3C000D98FBD82B3F76701638AF604050AEF801F
:10F3D000DFC3420593170A014181C183E3E8A7FA1D
:10F3E00041BFA16A370B0200014A977BFF1F938B35
:10F3F000ABADFD1A7D1BE1BF83C7440113070003BA
:10F40000854693F70703E391E7F8A2854A85EFD095
:10F41000FFCF41016F207F936155E5BF7955D5BF7F
:10F42000EF221F909774FF1F938484849C40D9EF30
:10F430009777FF1F9387079A9C436399070CEF8088
:10F44000DFBE930780023305F5028945EFF05FDAEE
:10F4500041C99777FF1F23A1A7A4EF801FBC930783
:10F46000400E3305F5029145EFF09FD835C99777E7
:10F47000FF1F23A5A7A2EF805FB201CDEF80FFB1F0
:10F4800091450E05EFF0DFD621CD9777FF1F23A919
:10F49000A7A0EF801FCB11CDEF80BFCAD94733059E
:10F4A000F5028945EFF0DFD405CD9777FF1F23A341
:10F4B000A79EEF809FB591450A05EFF07FD30DC160
:10F4C0009777FF1F23A2A7A0014521A8EF803FC285
:10F4D000930780063305F5029145EFF07FD101E5F2
:10F4E00065556F203F879777FF1F23A1A79201449F
:10F4F000130A80061779FF1F1309498FB14AEF805D
:10F500001FBF6364A4029C40E38407F2EF803FBE08
:10F510009307A0043305F5028945EFF07FCD69D14B
:10F520009777FF1F23A6A79A19BFEF805FBB894576
:10F530000605EFF0FFCB4DD5B309440303270902BD
:10F540004E9708CBEF80BFB8330555039145EFF0D8
:10F550003FCA59D58327090205041374F40FCE97C7
:10F5600088DB71BF9777FF1F938747888847058996
:10F570008280C167FD176319F5009777FF1F938796
:10F58000E78603A5070B8280EF222FFBEFF05FD207
:10F590006F20EFFC814709C58347E501B337F000D1
:10F5A0001777FF1F1307878418470983058B19C333
:10F5B00093E727003E858280EF222FF82A84EFF020
:10F5C0007FFD8347E401AA851305940899E3130599
:10F5D00004039776FF1F93866681944213061502F3
:10F5E0001307840213059504EFD0CFC06F202FF7C7
:10F5F000EF220FF39764FF1F9384447F98442A8976
:10F600002E840983058B9C4019C76314F500638021
:10F61000050E014401A2E3FEA7FE1387A702E36AD9
:10F62000A7FE850763FCA70883A9440BEF80FF961C
:10F630001316350081454E85EF202FF39767FF1F86
:10F6400023A6277B9767FF1F23A4077A49CC9C44F6
:10F6500093E747001767FF1F232EF7789777FF1F61
:10F6600023820780630F040C9767FF1F23A027796D
:10F6700001440549EF807F926341A40AEF80FF9423
:10F6800093050006B3C5A502B7F73600938707E8D0
:10F690001765FF1F1305457D416901449309400E1D
:10F6A0007D19B385F502EF70B016EF801F97634F99
:10F6B000A4080145EF3040700544A9A86398A7024B
:10F6C0009DE583A9440BEF805F8D131635008145BE
:10F6D0004E85EF208FE99767FF1F23A92771976752
:10F6E000FF1F23A707709C44ED9BADB785C5176727
:10F6F000FF1F034727779307F005E3FCE7F021F8A6
:10F70000EF60F03C6DD19C4493E707021767FF1F41
:10F710002322F76E22856F20EFE383A7440B131596
:10F7200034003E958357050081CB8347250099C758
:10F7300021468145EF206FE305042DBF23012501FC
:10F74000E5BF9767FF1F23A5076A0DBF3305340385
:10F7500083A7040B3E958357C50163842701EFF00F
:10F76000BFE5050499B7EF224FDDEF801F86130434
:10F7700000063345A4029764FF1F9384246783C760
:10F7800084073E951375F50F9767FF1F238CA76CB1
:10F790009307F00563E7A7020545EF30E061EF80CE
:10F7A000DF823345A402B7F53600938505E8B3053B
:10F7B000B5021765FF1F1305256BEF7070056F20ED
:10F7C0000FDA9C4405458983858B81CBEF904F8868
:10F7D00088408145EFF0DFE1DDB7EF30E05DC5B790
:10F7E000EF220FD4130495082A8913069005A285E9
:10F7F00013050503EF90603F1306900581452285B0
:10F80000EF20AFD64A85EF30C0548144176AFF1FFE
:10F81000130ACA5D930A8002EF803F8163C4A4008B
:10F820006F204FD3338454038327CA0A3E9403576F
:10F8300004008357C9016317F702834744009DC33F
:10F84000930964014546CE8513055400EF90E039D5
:10F85000454681454E85EF204FD122852302040085
:10F86000EF30005785044DBFEF222FCD9767FF1F64
:10F87000938707409C432A8491C70DC50355C50152
:10F88000EFE00FC29777FF1F9387078D9C4389CBCB
:10F89000EFB0DFD085476315F5002285EF50C05DDE
:10F8A0006F20EFCB41657D15E1BFEF220FC91764D3
:10F8B000FF1F1304A4534440938714001767FF1FCE
:10F8C0002328F752EF30605E1C448983858B9DE7C7
:10F8D0005840B7E7B0009387075063F1E70201454E
:10F8E000EFF01F9D01CD0545EF809FF6084085454F
:10F8F0000505EFF0FFCF0145EFF01FF726856F20DC
:10F900000FC6EF22EFC1A1642A8901449769FF1F46
:10F910009389895BFD14338AA500EF800FEF634460
:10F92000A4006F202FC303A7090093172400BA97E0
:10F930009843658F42074183634C2701635A47010F
:10F9400023800700A380070023810700A38107000D
:10F950000504E1B7EF226FBB83594500C54741114C
:10F9600063F537310441C1E533853401834785FFB1
:10F97000034795FF0348B5FFA207D98F0347A5FFAB
:10F98000C207220733670701D98F0347C5FF034822
:10F99000D5FF2207336707010348E5FF0345F5FF5D
:10F9A000420722083365A800498FB98F1767FF1FE8
:10F9B0001307474F1768FF1F1308C8503A8583285D
:10F9C00007006384172B1107E31B07FF1767FF1F4F
:10F9D0001307474F18431318270042951CC105070A
:10F9E000A1473367F7029767FF1F23ADE74C93F7F3
:10F9F00035001397470083474601C16B368993F75B
:10FA0000F7FCD98F32842E8A230AF600814A176CBC
:10FA1000FF1F130CAC3DFD1B976CFF1F938C4C25F7
:10FA2000176DFF1F130DCD4AEF802FDF63C7AA00AC
:10FA3000E154268541016F200FB11308400EB387B2
:10FA40000A0303280C0BB30DF800638E0D2083D737
:10FA5000CD01638A772183A70C00014B63970716BA
:10FA60009767FF1F938707379C436390071683C7E9
:10FA7000040003C70D0493F7F707631BF71ACA873F
:10FA80002287CE86268693859D0613851D04EFF07A
:10FA9000BF85631F051883D7CD01032709002320E5
:10FAA000B4012312F400FD572313F4008347170019
:10FAB00093F6F7078347D40093F707F8D58FA3068B
:10FAC000F40093F7F707B337F000B307F0402307CC
:10FAD000F400834717009D839396370083474401C2
:10FAE000DD9BD58F230AF400834737008346470008
:10FAF000A207D58F83462700C206D58F1CC883472F
:10FB0000770003478700A207D98F2315F4000D471C
:10FB10006304EA00BD5491DF93870710C207C183D5
:10FB20001307B00FBD54E376F7F0EF800FC981449F
:10FB3000E31105F09766FF1F83C6463993871600C9
:10FB40001767FF1F2304F7381767FF1F1307C7370F
:10FB5000231BD40093972600144303578400E175B8
:10FB6000BE96A1671386F7FFB377C70098426D8FE3
:10FB7000D98F9CC21848F18F3E07D98F9CC2EF8065
:10FB8000CFC89767FF1F83C7673433F5A70297670E
:10FB9000FF1F238DA73271BD9307A004B308FB029A
:10FBA00083270D00BE9803D7080083D7CD01631DBE
:10FBB000F70083C7040003C7880093F7F707630BB8
:10FBC000F70083C7FD019DEB050BEF804FD2E345A6
:10FBD000ABFC71BD9385980113859800CA87228775
:10FBE000CE86268646C6EFF02FF0B24879F98347D5
:10FBF000440193E74700230AF40071BD83C7040062
:10FC000003C7980293F7F707E310F7FCCA87228728
:10FC1000CE8626869385A8031385A802EFF0CFEC45
:10FC200045F58347440193E72700230AF400C1B751
:10FC300083C7FD018DCB83C7040003C79D0993F7DC
:10FC4000F7076312F702CA872287CE862686938536
:10FC50002D0C1385AD09EFF02FE911E58347440121
:10FC600093E7270049BF850AC1B3FD54D9B3EF22FA
:10FC70004F8A797183544500AA8B2E84B28AEF8013
:10FC8000CFBB590563499504B7E4040003A90407F1
:10FC9000EF80AFBA59054205418102992A8905CD05
:10FCA0002AC623180100EF804FB959052319A10076
:10FCB0006146814528089769FF1F938929134ACA1D
:10FCC000EF20AF8A2302810203A48900058819E48A
:10FCD000BC544A85829745616F202F877400300895
:10FCE000D6855E85EFF01FC765F56800EF807FF170
:10FCF000176AFF1F130A4A4683270A00AA84035B78
:10FD0000010189CB89476397FA00835501025E851B
:10FD1000EF50203003552102EF704FC819E503550D
:10FD20002102EF708FD43334A00093176400034492
:10FD3000C1022C0868001374F4FB5D8C2306810259
:10FD4000EF60B056E9576314F5028356E1029767F6
:10FD5000FF1F938767179C43139726006176BA9716
:10FD60009843718F98C39767FF1F2381D716831716
:10FD700021026345F00085476396FA00B25793F776
:10FD8000070C95E7D247C2040347C102C180BE9465
:10FD900026C62318610113770703C147631DF700C7
:10FDA00083475102054793F7F7076390E704B7E7E6
:10FDB0000400BC5739BF92570544A18393F7F70756
:10FDC000E377F4FE15C78347C1021307000293F7D8
:10FDD00007036397E700EFB06FFC8547E319F5FC75
:10FDE0008347C10293F7070389CFEFB0AFCA21A8B9
:10FDF000EFB08FD7E30985FCEFB04FFAE31985FA2E
:10FE0000D9B7EFB0EFD8AA8501460545EF707FF866
:10FE10002A8451DD8347C102414793F70703638476
:10FE2000E70232478347170093F707F8A300F7006C
:10FE30003247925783461700A18393F7F707FD17C0
:10FE4000D58FA300F70003560101B245130BC40080
:10FE50005A85EF80DFDFE24A130690058347C1022F
:10FE600083C4EA01918BB384C402138514045695AC
:10FE700095C35444B3879A0083C7070403C7060099
:10FE8000137707F82380E600584483460700D58F90
:10FE90002300F700B25703A609008146858B1D8E0B
:10FEA000DA85EFD0EF9B15E9B25783A509004844E6
:10FEB00013869406858B56969D8DEFD0CF9411EDC9
:10FEC00083270A0099EFB257054791838D8B63878B
:10FED000E7049DCF09476389E7042285EF80DFF8B7
:10FEE000F9B5EFB0AFEB85476309F5008347C10271
:10FEF000414793F70703E398E7FC835521025A85AE
:10FF0000EF40907C69D183172102E35EF0FAF1B7EC
:10FF1000EFB08FC57D151335150061D101468145C0
:10FF20002285EF70FFEF55BFEFB04FE7E5B7EF1257
:10FF3000DFE09764FF1F9384E4EC2685EF809FEB5E
:10FF40002A8419E16F10BFE11305C40005468145FD
:10FF5000EFF0FFD12285EF803FF1C5B7EF12FFDD53
:10FF60004111AE842A849307950313071501930664
:10FF7000F10005466C00268523060100EFD0CFBEB8
:10FF80001DEDA68541462285EF8030468347F1006E
:10FF90009305140226852308F400EFD06FC805E10D
:10FFA0009767FF1F9387471B9C4389EF13069404B1
:10FFB00097C500009385C5DB2685EFD08FD441011E
:10FFC0006F10FFD91306940297C500009385C5DA18
:10FFD0002685EFD00FD379D9DDB7EF127FD497679D
:10FFE000FF1F938767EE8043AE84B289368AAA8A60
:10FFF000EF80AF811316250081452285EF10FFD6D3
:020000040001F9
:100000009767FF1F238407EC9767FF1F938707DE1F
:1000100003A4070B13F714003E89230FE400CE85D9
:1000200025C713059408EFF07FF301C555556F10F0
:100030007FD28947A30FF4009767FF1F9387C711EB
:100040009C4303278900858093B717008607230008
:10005000F402231E54019767FF1F23A947D98588FF
:100060009377B7FF99C0936747001767FF1F232354
:10007000F7D82285930700061767FF1F2304F7DED2
:10008000EFF08FD3014565B713050403EFF01FEDC3
:1000900045D569BFEF127FCAFD572310F500231124
:1000A00005002312050023130500130620048145D3
:1000B0002105EF109FCB6F109FCAEF127FC6411131
:1000C000AA8401441769FF1F130989E09309A0045A
:1000D0002EC6EF80CF81B2456344A40061550DA0C8
:1000E00033053403832709003E9583572500639C1D
:1000F000B7008357050063989700EFF0BFF90145FB
:1001000041016F103FC50504E1B7EF127FC197674A
:10011000FF1F938727CC9C434111AA842E84B28968
:1001200003592500C1C39767FF1F83D7E7CE639BA1
:100130002707EF700F862A8903D524009305100244
:10014000B305B40285472302F10093578900A30247
:10015000F10093578500A303F10083D744002304E3
:10016000A100254613D787002305F10083D764003B
:10017000A304E1004E8513D78700A305E100230601
:10018000F1001387950093879501A105B386B4000C
:10019000A6974C00269723032101EFD0EF9C410145
:1001A0006F105FBBEF60FFFE51BFEF127FB74111D1
:1001B000AA8401441769FF1F130989D19309A00478
:1001C0003AC636C432C22EC0EF707FF28245124664
:1001D000A24632476344A400615599A0B307340393
:1001E00003250900AA9703D8070003D5C4016310AB
:1001F000A80495E91DEE91CA03C6E4019305100217
:100200003306B60225063E9690C2014511CB83C641
:10021000E40113061002B386C602E506B6971CC3B6
:1002200041016F103FB303D52700E305B5FC05047A
:1002300041BF83C5E40113051002B385A502BE9535
:1002400083C585002300B6007DB7EF127FAD5C410A
:1002500041112A8403DA2700C167FD17AE84328971
:10026000630CFA002685EF807F9A8D4763EDA70027
:100270007D5541016F101FAE2E85EF803F999D4740
:10028000E3E2A7FEF5B75C40268583D54700EF8003
:100290009F90835584002685EF80FF8F8D452685AE
:1002A000EF803F8EAA89EFF04FE09357050123803E
:1002B000F90093578500A380F9002381A9005840D5
:1002C000C167FD178345A7006314FA0093E505088D
:1002D0002685EF801F8F9767FF1F9387A7AF9C43EB
:1002E0000840D9CF8347B400858BD9CB7800340040
:1002F000130671008145EFF05FEB1DC98347B40021
:10030000184093069005F99BA305F4008347E70185
:10031000B387D702B306F70083C60604A303D10050
:100320009386170493879706BA96BA9736C43EC643
:100330001764FF1F130484AB1C440C40268589837B
:10034000858B9D8D834771009E05DD8D93F5F50F9F
:10035000EF803F871C44104022458983858BCA86E5
:100360001D8EA685EFC0DFCFE31505F01C440C40C1
:10037000324689838840858B9D8DEFC0DFC8D5BD0F
:100380008347B40013079005F99BA305F400834746
:10039000E501B387E7023307F50003470704A3032A
:1003A000E10013871704938797062A973E953AC46E
:1003B0002AC6BDBFEF12DF96032A45009307F00F50
:1003C000AA840347AA00AE89328436896316F700EF
:1003D000EFB06FAB2305AA00938AC9000146D6850A
:1003E0002685EFF09FE62A8A21E51767FF1F13078E
:1003F000A7D61843DC4039C383C6A7000547638FDF
:10040000E60283D547005685EF40102C05C9DC4035
:10041000839747006354F00201CC1C4089C74A8689
:100420008145014582975C4081C7CA850145829715
:100430004E85EF807FA352856F10DF91DC4003D59E
:100440004700EF60BFD501E9DC4003D54700EF600E
:10045000DFE181471DCD19C41C4089C74A8681450B
:10046000014582974E85EF807F9FAA851765FF1F04
:1004700013054599EF80DF9511C45C4081C7CA859B
:10048000014582971765FF1F13050597EF60F0364A
:100490008547D84085460346A700E30BD6F80317E7
:1004A00047006353E000C9F74A86A2854E85EF7086
:1004B0003F97BDBFEF12DF86AA8401441769FF1F73
:1004C000130909A19309A004130A9508EF703FC20C
:1004D0006344A400014535A0330534038327090094
:1004E0003E958357250099E30504CDB703570500D2
:1004F00083D7C401E31AF7FE52868545EFF0FFC0AB
:1005000065D56F103F85EF12BF81AA84014417693A
:10051000FF1F1309E99B9309A004EF705FBD6344BB
:10052000A4006F103F8333053403832709003E95F1
:100530008357250081CF8357050063999700930562
:100540009502130610022105EF80206A0504F1B719
:10055000EF12AFFE0347E5012A848347F5016307E5
:10056000B70089E781452E856F106FFF230FB40018
:10057000054781C9E398E7FE8947A30FF400854545
:10058000DDB7638BE7020947E39FE7FC2285EFF0C5
:100590002FA59767FF1F9387E7839C4399E797579A
:1005A000FF1F9387E76C9C4389C70355C401EFF095
:1005B0009FF5A30F0400E1B755D6C9BFEF124FF660
:1005C000EFA0FFEE85476312F508EF80EFCC1764CC
:1005D000FF1F130464B81C4081CBEFA03FFC894788
:1005E0006304F5001C4082979757FF1F9387877E0F
:1005F0009C43B9CF82979757FF1F938767679C43A8
:1006000091C382971754FF1F1304447E8327040B62
:1006100083D4C701EF60FFB78327040BAA8514407A
:1006200003C6E7011C448983858B99C313662600A2
:1006300026854169EF40C03D8144D9497D19EF705D
:100640005FB063CAA4006F10EFF0EF800FCA41B72C
:10065000EF705F884DB7B38734030327840ABA97D6
:1006600003D527006308250103C6470183D507008A
:10067000EF40A03B8504E1B7EF128FEA01449754A5
:10068000FF1F9384A4761309400EFD59EF70FF9865
:10069000634FA40401449754FF1F938424751309E6
:1006A0008002FD59EF707F98634CA4040144975475
:1006B000FF1F9384A4735949FD59EF709FA8634AA3
:1006C000A40497F5FFFF9385450A1755FF1F1305EF
:1006D000A579EF60D00797050000938585851755AC
:1006E000FF1F13056571EF6050056F10AFE633070C
:1006F000240383A7040B0504BA97239E370179B717
:100700003307240383A7C40A0504BA97239037014B
:1007100051BF3307240383A7840A0504BA972391A2
:10072000370161BFD4410387350085473356F50251
:100730006377E600A54899E7238006008280B387A7
:10074000E702EDB73358F502038735003375F5023C
:10075000B3D7E7021307000363DA080103C60500F5
:1007600013077003118A19E2130770058506429773
:10077000A38FE6FEC9B718451C416376F7005C41BC
:10078000BA972380B7001C4585071CC58280EF12ED
:10079000CFDA4111AA872E85B285368636C6829772
:1007A00063480500B246158D3335A0003305A040DF
:1007B00041016F10CFDAEF12AFD6056941112A8AD5
:1007C0002320060001448149975AFF1F938ACA7269
:1007D000056B7D1932C62EC4EF703F85AA84EF7079
:1007E000DF832695A24532466346A4004E8541012B
:1007F0006F104FD603A70A0093171400BA9703D7B8
:1008000007003377670101E71CC20504E1B703D78E
:1008100007009356D700858AE39946FF337727016F
:10082000E315B7FEBE89D5B7EF122FD101112EC641
:10083000B2843689EFB02FEE2A84615501C8B245E3
:1008400089E9232E040023200402014505616F106D
:100850000FD1A1463008CA852685EFF05FF37DF5FC
:10086000835781010357A101231EF4008357C1015F
:100870002310E4022311F4028357E101D207D1834C
:100880002312F4028357E1011397370163560700DF
:10089000FD57231FF4005DBF231F040045BFEF1267
:1008A0002FC81754FF1F130464548327040B03D766
:1008B000C701C167FD17630EF7109767FF1F938786
:1008C000E7899C4381C70545EF406077C1690149CD
:1008D000930A400EFD19176BFF1F130BEB87EF7088
:1008E000CFF3634BA90E1757FF1F0347A757930773
:1008F000F00563E4E702EF704FED93050006B3C522
:10090000A502B7F73600938707E81755FF1F1305B1
:10091000A555B385F502EF60A06F8145170500006E
:1009200013058520EF60DFF8EFB0EFDE01CD035750
:10093000C50109CB0357E50111C78347050299C3D8
:10094000EF60A06BEFB06FDE31C51757FF1F034795
:10095000275E9757FF1F9387A75D0DCF03C717002B
:100960002304E50003C72700A304E50003C73700FD
:100970002305E50003C74700A305E50003C75700AB
:100980002306E50003C7670083C77700A306E500D9
:100990002307F5001C4493E717001757FF1F232B6D
:1009A000F7445C4085E7EF708FEF0DC1EF702FEFDC
:1009B00044402A89EF70AFEE33F5A4025C40FD1786
:1009C000CA97898F1757FF1F2324F7420145EF70FD
:1009D000DF9F01456F100FB8B30459038327040B41
:1009E000BE9483D7C40163883703138A0403D28576
:1009F0005285EFF0AFD605E183C7F40199CF938517
:100A000094082E85EFF08FD509C91306900581450E
:100A10005285EF108FB50509D9B583270B002685C0
:100A200093B7170086072380F402EFE0FFB8E5B71D
:100A3000854763F8A7009307F5FFBE953305A040EF
:100A4000E98D2E8582809841C167BA9713D7070137
:100A50006304A7009CC182804207998FE5BFEF1213
:100A6000CFAD41112EC63284B684EFB00FCCE15722
:100A700001C9B24591E99757FF1F238B074A814768
:100A80003E8541016F10AFAD9D461756FF1F1306FF
:100A9000364AA6852285EFF09FCFAA8775F10547D4
:100AA0009756FF1F2386E648E1BFEF126FA741115B
:100AB00091E99757FF1F23AD073201442285410179
:100AC0006F104FA9B68532858D467000EFF03FCC90
:100AD0002A846DF58347D1000347E1001759FF1FB2
:100AE0001309C930A2074207D98F0347C100D98F24
:100AF0001757FF1F232EF72EEF706FDA61D1EF70BB
:100B00000FDA83244900AA89EF706FD933F5A40264
:100B100083274900FD17CE97898F1757FF1F232979
:100B2000F72C69BFEF126FA11C45AA8491CFD84B57
:100B300001CF83D7470089CBEF601F92AA8509C5F3
:100B400088446105EF60C04C9757FF1F9387872843
:100B50009C43014489EF6F108FA09C481317140029
:100B6000BA9703D5070019C1EFE0CFCF0504EF70A6
:100B7000CFC7E344A4FEC5B7EF122F9C011185E94E
:100B8000EF605FDA01449757FF1F23AD072E975799
:100B9000FF1F23AB072E9757FF1F23A9072E975739
:100BA000FF1F23A7072E228505616F104F9BB68775
:100BB0003285C9467000BE85EFF07FBD2A8465F599
:100BC00041469305E1001755FF1F1305A52BEF8044
:100BD000C0010355C100EF608FD7F1B78DE1975782
:100BE000FF1F23A507209757FF1F938727209C47A8
:100BF0000145ED9B1757FF1F232EF71E8280EF1232
:100C0000CF934111B685328595463000EFF03FB85D
:100C100015EDA2471757FF1F232AF71C9757FF1FF1
:100C20009387C71C9447B24713F7B6FF13F6170014
:100C300019C213E74600858393F7F7079756FF1FFE
:100C400023AAE61A1757FF1F230EF72041016F1042
:100C50000F91EF12EF8C03841500DC412A89AE84DA
:100C600085070387F7FF19C36340800C838724003F
:100C700091C7635580007D14620461849C403707EE
:100C800000FF0907F98F3707001009076392E70A89
:100C90006355800079146204618483C70400858BE6
:100CA00095E39379F40F4E8A93178A01E187634A9B
:100CB000F008A2876353040081473384F9407D1410
:100CC000620461848385240081C54A85EFF0BFAA50
:100CD0009C40370700FF0907F98F37070010090705
:100CE000639AE706930500034A85EFF0DFA883C700
:100CF000040093058005918B99E3930580074A854D
:100D0000EFF07FA783C70400858B81CB1374F40FAA
:100D100093178401E1876347F004C040050483050D
:100D2000F4FFA1E96F100F837D14620461840DBF8D
:100D3000370700080907E392E7F6E35080F67D14D1
:100D400099BF930500024A857D1AEFF0DFA2137A5E
:100D5000FA0F99BF370700080907E395E7FA9305EB
:100D6000000371BF930500034A85EFF0DFA07D14F7
:100D700071BF4A85EFF03FA055B7EF021FFCEF703F
:100D8000CFAA2A84EF706FA9229589450605EFE066
:100D90002FC6E55711C59757FF1F23AFA7148147EB
:100DA0003E856F00DFFB930700026306F5005D15CB
:100DB00013355500828005458280EF027FF6411190
:100DC000AA892A89130419008304F4FF32C62EC4A9
:100DD0002685EFF05FFDA245324659E19307D00228
:100DE0006392F408830404000548130429009377F0
:100DF000F6FEC9E793070003639FF40E8307040020
:100E00001307800593F7F7FD6399E7068304140041
:100E100041460904B70600806314080093C6F6FF34
:100E2000B3FEC6028147254F654EFD5F33D3C60230
:100E3000138704FD6368EF06BA8463D5C408630DA5
:100E4000F5017D55636AF3006394670063C69E00F5
:100E50000545B307F602A69705048304F4FFC9BF4E
:100E600022898DB79307B0020148E392F4F8830416
:100E700004002A88130429009DBF01CA8947E31B87
:100E8000F6F893070003E397F4F8830704001307C9
:100E9000200493F7F7FD639BE704830414000946DD
:100EA00009048DBF13E704021307F7F9636CEE0022
:100EB0009388F4FB1307700363741E011307700516
:100EC000998CA5BF7D576300E50263040800B30752
:100ED000F04091C519C19309F4FF23A035013E8567
:100EE00041016F003FE7B687FDF5D5BF93040003CE
:100EF00015F2214605B719FE294629BFEF025FE228
:100F0000011161540DC53284AE894146814536894F
:100F1000EFF0BFEA93140501C180639E09002685A6
:100F2000EF30102B014401C58145EF20501622857A
:100F300005616F003FE22285CD467000CA85EFF063
:100F40001F852A846DF52685EF30902809E9035620
:100F5000C1008345E1012685EF20500B01C94146C0
:100F60009305E1001105EF705048D1B75D54C1B74A
:100F7000EF021FDB0111E15401CDB284AE8941467D
:100F800081453689EFF07FE32A8463970900814425
:100F9000268505616F001FDC2685D1467000CA8555
:100FA000EFF0EFFEAA846DF58357C100EDD3EF702B
:100FB0000F8E4205931704014181C18363F9A70293
:100FC000EFB08FB64204E14741803304F40241465A
:100FD0000C082A9413054400EF7030418357E10058
:100FE0002311F4008357C1002310F40055B7E554D2
:100FF00045B7EF02FFD27971E15415C53284AE894D
:1010000041468145B684EFF05FDB131905011359A2
:101010000901639E09004A85EF401065814401C5BE
:101020008145EFB02FB1268545616F00BFD2A685FF
:101030009306300270002285EFF06FF5AA8465F503
:101040004A85EF4070622A8411E54A85EFB04F8CE3
:101050002A8431C58357C1002311240193096400F8
:101060002310F4008347E1009305F1004146230279
:10107000F4004E85EF7070371309740141469305F3
:10108000F1014A85EF707036930554004E85EFC02C
:101090004FBF930564014A85EFC0AFBE69B7DD5409
:1010A00059B7EF02FFC7797111E5E1542685456113
:1010B0006F005FCAB284AE89414681453689EFF040
:1010C000DFCF131A0501135A0A015285EFE06FCAE8
:1010D0002A846398090071D98145EFB02FB4814407
:1010E000F1B72685930610027000CA85EFF02FEA4B
:1010F000AA844DFD31C8B2479305D1004146858B86
:10110000230FF400B24713050403858393F7F70711
:10111000A30FF400EF70702D41469305D101130524
:101120009408EF70902C59B73304690383A70A0B16
:101130003E948357C401638337030509EF60FFEDD5
:10114000E344A9FEDD549DB7C1690149975AFF1FC9
:10115000938ACAC9130B400EFD19CDB7231E440153
:1011600059BF49CDEF02DFBB4111B289AE84414680
:101170008145368AEFF07FC4931A050193DA0A019C
:101180000149175BFF1F130B6BC6EF601FE1634A3A
:10119000A9000145ADCC81441759FF1F130909C5AA
:1011A00081A883274B0B131439003E948357040006
:1011B000638857050509D1BF8327490B1394340071
:1011C0003E948357040085E7231054019146700034
:1011D000D2854E85EFF0AFDB1DE9B247139787004C
:1011E000E1832183858B58C02301F4000DA0850481
:1011F000EF60BFDAE3C2A4FC5D5511A8615582809F
:10120000F1F4214681452285EF003FB601454101B9
:101210006F005FB41971D2C4130AC10686CEA2CC86
:10122000A6CACAC8CEC6D6C2B6D6BAD8BEDAC2DC3C
:10123000C6DE52C463810524FD151C102ACC2ECABB
:1012400002CE3EC89304B0021549A94983050600A1
:10125000130416009DE1F2465247E24763FBE62085
:10126000B697238007007245F6406644D644464947
:10127000B649264A964A09618280930750026386DE
:10128000F5004808EFF02FCFF5A88357C1002307DA
:101290000100014593F7C70F2316F100814501486E
:1012A0000147014681469308D00213030003130E41
:1012B000300205048307F4FF99C7638C970463C366
:1012C000F404638BC70501CA0346C100858A799A75
:1012D000D18E2306D100630908008346C100098B23
:1012E000F59A558F2306E10019C12307B100138732
:1012F00007FD1377F70FA54663E2E6068146A5458D
:10130000294535A0E38717FBE39F67FA0546FD569D
:101310004DB70545854571BF05487D5759BFB38613
:10132000A60205048307F4FFBA96E206E18613F7E6
:10133000F70F130607FD1376F60F63E5C500138755
:1013400007FDF1BF1306F7F91376F60F636EC902B6
:10135000138797FAE30537FDA306D100130790061C
:101360006385E704634BF706130780056384E70A88
:101370006345F702E38107EE13075002930550021D
:10138000E381E7F02286D9B51307F7FB1377F70F50
:10139000E364E9FC138797FC75BF13073006638687
:1013A000E70A13074006E39FE7FC03250A00A94765
:1013B000A307F100930A4A00635805009307D0027F
:1013C0003305A0402307F1006C00EFF0AFB56C00CF
:1013D0004808EFF01F88568A75B713073007638EE9
:1013E000E7066341F7021307F006638EE70413076D
:1013F0000007E399E7F80347C100136727002306B6
:10140000E10009A813075007638BE7021307800761
:10141000E39AE7F6938787FA414793B71700A30744
:10142000E100139727008347C100ED9BD98F230666
:10143000F100930A4A006C0003250A0079B7A94716
:10144000A307F100FDB7A147E5BF83050A004808DF
:10145000930A4A00EFF02FB2BDBF83270A006C0049
:1014600048083EC8EFF0EFFE1C10930A4A003EC841
:101470009DB7BA97FDB30145C5BBEF021F8C2A8803
:10148000368583464800BA8703475800A206D98E9E
:10149000328717B600001306669089E517B600007C
:1014A00013068690BE85EFF0FFD66F005F8B9757CF
:1014B000FF1F938767A79C4381CFEF021F88D84304
:1014C000B2862E861847AA853E8502976F003F890F
:1014D00061558280EF027F868357050039712A8427
:1014E000231EF1008347450093056500414613051F
:1014F000F101230FF100EF70406F93057401414635
:101500001305F102EF70606E8356240017B60000D9
:101510001306C691E5450A85EFF0DFCF6C08130688
:1015200030020A85EFF0BFF821616F005F83EF02A0
:10153000DF8039712A849305050341461305D101E3
:10154000EF70A06A9305940841461305D102EF702D
:10155000C0698347E4010347F4018356C401858BC6
:101560000607D98F17B600001306068DE5450A85D4
:10157000230EF100EFF01FCA6C08130610020A8553
:10158000EFF0FFF221616F008FFDEF026FF937047A
:101590000001B70400FF0111814A1759FF1F130909
:1015A000E9847D149389F4FF17BA0000130A4A8D69
:1015B000EF60BF9E63C5AA0005616F00AFF9832786
:1015C000490B13973A003E978347370095CF5C430A
:1015D000A30107005286B3F687008247E54548001D
:1015E000E58FD58F3EC083462700B3F73701858A44
:1015F000E206D58F835607003EC0EFF0BFC111460B
:101600008A854800EFF0BFEA850A5DB7EF02EFF286
:1016100001468145EFF0BFE96F006FF48357650025
:10162000638E071A1D71A2CCA6CACAC886CECEC6C2
:10163000D2C4D6C2DAC05EDE801013F7170032893A
:10164000AA8431CBF99B2313F500EF601F9906059F
:101650003D0541990A8BC16A3301A1408A8B8149BA
:10166000014AFD1AEF607F97634CAA0C79479306F5
:1016700004FB17A600001306A67FCA852685EFF097
:10168000DFDF638F090C13961900DE85130504FB59
:10169000EFF0FFE15A8183D7640013F7270021CBD5
:1016A000F59B2393F400EF605F9406053D05419997
:1016B0008A8A3301A1400A8B8149014AEF60FF9277
:1016C0006345AA0A6547930604FB17A600001306A4
:1016D000A67ACA852685EFF05FDA6387090A139632
:1016E0001900DA85130504FBEFF07FDC568183D700
:1016F000640013F7470005CBED9B2393F400654787
:10170000930604FB17A6000013064677CA852685B4
:10171000EFF0BFD69C4481C703D747003DEB1305CC
:1017200004FBEFF0BFEE130104FAF6406644D64422
:101730004649B649264A964A064BF25B25618280A5
:10174000DC4413171A00BA9703D707006308570140
:1017500093971900DE972390E7008509050A19B7CA
:10176000130504FBEFF09FEA35B79C4813171A00E6
:10177000BA9703D7070019C793971900DA972390F0
:10178000E7008509050A1DBF130504FBEFF01FE8FC
:10179000B1BF2314E4FA03D767008326C4FA2146B5
:1017A000520751832315E4FA370700F0758F9447E9
:1017B000930584FA130504FB92069182558F232624
:1017C000E4FA83C7770013F707018347F4FABD9B58
:1017D000D98FA307F4FAEFF09FCDB1B78280EF0263
:1017E0004FD31744FF1F130464600444797193F7C7
:1017F000F4FB1747FF1F232FF75E93F70404A1C7DD
:101800008588A1E097A9000093898967EF60EFF8C8
:1018100063DBA4028327440B139934003E9983565B
:10182000090091CE4E86E5454808EFF0BF9E480876
:10183000EFF0DFDD214681454A85EF000FD38504B7
:10184000F1B7EFF09FD41C4413F7F7F79746FF1F4B
:1018500023A2E65A93F707086397071E1C4413F761
:10186000F7EF9746FF1F23A7E65813F707106318F3
:10187000071E18449377F7DF9746FF1F23ACF656F1
:101880009376072095C6058B630A07201840898345
:10189000858B3ACA0347840715464C080607D98F3B
:1018A00017A500001305855A230CF100EFF03FC087
:1018B0001C4413F7F7BF9746FF1F23ADE65293F77B
:1018C00007408DC3835744000D464C08231AF1008E
:1018D0008357640017A5000013058557230BF100FB
:1018E000EFF0FFBC1844FD749387F47FF98F97469F
:1018F000FF1F23A1F6509317470163DF0700EFA0F6
:101900008FE119C98356C5016391061A17A5000016
:1019100013058554EFF09FCF1C447D777D177D8F95
:101920009746FF1F23A8E64C13973701635A070217
:10193000858B6388071CEFA04FDF1DC118458347C7
:10194000E5001D463ACA0357C5004C0817A500001C
:1019500013050551231CE100230DF100EFF03FB505
:101960001844F977FD17F98F9746FF1F23A4F6480F
:101970009317270163D90700814517050000130558
:1019800025CAEF50FFF21844E177FD17F98F97460B
:10199000FF1F23A1F6469317070163D30702EFA0A9
:1019A000BF982A84814417A900001309E94BEF600E
:1019B0000FEE939704014205C183418163EAA714A6
:1019C00045616F008FB883A70A0093141900BE9475
:1019D00083D7040033F767011DCF1396170133F740
:1019E0007701B3F637016352060417A60000130609
:1019F000E64309E717A6000013060644E545480834
:101A0000EFF05F814808EFF07FC083D70400B3F7A1
:101A100047012390F4000509EF602FE1AA84EF60ED
:101A2000CFDF2695E341A9FA15BD368519C7EF40EA
:101A3000A04361DDEFF01FAAC9BFEFD09FB371D5FE
:101A4000EFF0FFAED9B785697D7A0149974AFF1F4C
:101A5000938A8A4A056B896BFD197D1A75BF858B40
:101A60009DC7EF500FF3231AA10041469745FF1F72
:101A70009385454113056101EF70201749464C08D5
:101A800017A500001305053CEFF07FA2DDB317A5F5
:101A900000001305253BEFF07FB7E1BB17A5000061
:101AA0001305C53AEFF09FB621B50357E501C1779D
:101AB00085073E978357A101FD141337170032079E
:101AC000E58FD98F231DF100231AD100835605021B
:101AD000035725022146231BD100231CE100035795
:101AE00045028566FD16758FFD76F58FD98F4C08FA
:101AF00017A5000013054536231DF100EFF03F9BAD
:101B000021BD17A500001305A535EFF03FB089BD35
:101B10005C4813F7E7FF58C8858B89CFA6864A86AD
:101B2000C9450A85EFF00FEF8357040099E70A854E
:101B3000EFF0DFAD850461049DBD231AF1008357EA
:101B400024009305440041462808231BF100EF7050
:101B5000C00951464C080A85EFF07F95E1BFEF02BE
:101B6000CF9D85473395A7009747FF1F9387072889
:101B70009C47411181455D8D9747FF1F23ACA726E8
:101B80009377057085E393576500858BA1CBC1677B
:101B9000938707887D8D05EDEF606FD19305803EBB
:101BA000B305B5021745FF1F130545352EC6EF5087
:101BB000A03BB24519C16349B50085C51745FF1F54
:101BC0001305C533EF50C04441016F004F99EF60DA
:101BD0000FCE2A84EF60AFCEE360A4FCEF602FCE7F
:101BE00075BF0145EFF0BFBFC5B7EF020F95797123
:101BF000AA8601441749FF1F1309491F36C6EF6023
:101C0000CFB9B246635CA4028327490B9314340016
:101C1000BE9483D704006396D70285C617A600003A
:101C200013060626E5454808EFF0CFDE4808EFF03A
:101C3000FF9D214681452685EF002F9345616F006A
:101C40000F92050465BF19C223200600814701C514
:101C50009306D00389E53E85828085050505838747
:101C600005000307050099CF6394E700E397D7FECB
:101C70008147D5B79306D0038547E30ED7FC93374A
:101C80001700D1BF9307F002E316F7FE854761D630
:101C9000050508C2C9B799C123A0050081470DC138
:101CA0001308D0031306F0023307F500830607007C
:101CB00081CA638706016397C60099C1050798C169
:101CC0003E8582808507CDB731C9EF028F844111EF
:101CD0002E8A6C002A89368BB28A97A400009384DE
:101CE000E40DEFF05FFB2A8C0144A689B14B8840DC
:101CF0006286CA85EF70E01801ED0E044E945C40D8
:101D00003245DA865686D285829741016F00EF838D
:101D10000504A104E31D74FD6155C5BF7D55828096
:101D200099E561558280615505616F00AF82EFF2E0
:101D30003EFF2E8A2A8401118145B2845285414694
:101D4000BA893689EFF06F8793150501C181137643
:101D5000F50FA1812285EF507FB12A8469D5528584
:101D60004C08EFF05FF3524A2A8BE30E0AFA2A86F8
:101D700097A500009385C50F5285EF708010AA8A41
:101D80000DED7D5AEF606FA563C5AA0099E8014586
:101D900061BF5C4413971A00850ABA9723904701E4
:101DA000D5B74C442EC6EF604FA3B24513161500AD
:101DB0004E850299E34DA0FC85BF5A8697A5000089
:101DC0009385850B5285EF70C00B0DE1032A04014A
:101DD000EF60AFA11316150081455285EFF0FEF8B4
:101DE000DDD40C482EC6EF604FA0C1B75A8697A528
:101DF00000009385A5085285EF70A00841E11C44BE
:101E0000A5CF81ECD443370700E0758F9447D8C342
:101E10003707001F758F98C701BFA1463008CE85D0
:101E20004A85EFE0DF96E31105F0184483578101FE
:101E30007D762312F7008357A101939647018357BC
:101E40006700D182F18FD58FF2467D767D16F182C3
:101E5000858AB206F18FD58F2313F7008347E101FE
:101E60008356C1012305F7008347B7002314D70029
:101E7000FD8BA305F7004DBD7D557DB55A8697A511
:101E80000000938525F35285EF60B07FE31D05E8E0
:101E90001C4CE38A07E89C43E38707E8CE864A8622
:101EA000A6852285829749B5EFF23EE93687B2864C
:101EB0002E86AA850545EFF0BFE66FF05EEAEFF2E9
:101EC000DEE73687B2862E86AA850145EFF05FE50C
:101ED0006FF0FEE8EFF2DEE4411199C123A00500A6
:101EE0009747FF1F93874703804381441DC82E896E
:101EF000AA8931141DC40C4070004E85EFF0BFD488
:101F000019CD81E8A284630C0900B2472320F900AF
:101F100039A08C4008400146EFF0FFD265F54048FB
:101F200069F8268541016FF0FEE2184111CBEFF20E
:101F3000DEE0AE873E85B285368602976FF03EE2E0
:101F400035558280EFF27EDF8357C50013D7050138
:101F5000C205B387E7021841C1814849BA95BE95C9
:101F6000EFF0BFFC6FF0BEDF584111CBEFF2FEDCAB
:101F7000AE873E85B285368602976FF05EDE3555B8
:101F80008280184509CBEFF25EDBAE873E85B285D5
:101F900002976FF0DEDC355582805C4599C7EFF221
:101FA000DED92E8582976FF09EDB35558280EFF269
:101FB0003ED783290500035AC5002A844849AE84C8
:101FC0008145EFF09FFD2A890DE193D50401B3858A
:101FD00045030356C4004848CE95EFF09FFA2A897E
:101FE00009E548488545EFF05FFB4A856FF09ED6CE
:101FF000EFF21ED32A890441035BC5004849797179
:102000002E848145B28A368AEFF03FF941E1935937
:102010000401B3896903420441802694A2990344D0
:102020000901330480403374440111CC0325490174
:10203000A2865686CE85EFF03FF3AA8431E1330ABB
:102040008A40A299A29A8144630C0A025286D685DC
:10205000080803244901EF605039834609011C0830
:102060009305F00F338646413385470136C6EFF0BE
:10207000DECFB2461008CE852285EFF0FFEEAA84AF
:10208000032549018545EFF05FF1268545616FF035
:102090007ECCEFF29ECA2E864C41A1462A84EFF0F8
:1020A0003FF5AA8403450401A145EFE07F985C4019
:1020B0003385A74048C026856FF07ECA814797A622
:1020C00000009386A6CC6393C70082803387F50017
:1020D000034707008507398D135745003697034797
:1020E00007001205398D1375F50F13574500369704
:1020F000034707001205398D1375F50FE9B7EFF2A5
:10210000DEC32A84AA851D461305F00FEFF01FFBDE
:10211000834774003385A7403335A0006FF03EC479
:10212000EFF2BEC14111A1463000EFF0BFE109ED71
:1021300003578100C167FD1705456317F7002800A5
:10214000EFF0FFFB3335A00041016FF05EC1EFF20D
:102150003EBDAE848C414111A1462A89034405014C
:10216000EFF05FDEAA8939E9A1452285EFE05F8CB7
:102170009C400357C9002A8AAA97939607019CC0DE
:10218000C182098F639CE602C16513D70701B3853D
:10219000B74011E78355E900FD15C205BE958CC017
:1021A000A1460A864A85EFF0FFD9AA8901E90A8586
:1021B000EFF0FFF401C9832749009CC04E8541011F
:1021C0006FF05EB90357C900835721008040330781
:1021D000474163DBE70033FA470363170A0041779F
:1021E000798C3E9480C0D9BF03450901A145417A4D
:1021F000EFE01F84098CAA8A80C0337A4401417BB6
:1022000063648A0081495DBFA1463000A2854A858A
:10221000EFF05FD3AA895DF12800EFF05FEE11E9DE
:102220008357A1000357C100337A6A0180C0BA976F
:102230003E9A33045441E9B7EFF23EB02A84AA85AE
:102240001D461305F00FEFF07FE7A303A4006FF026
:102250001EB1EFF21EAC2A84034505015D71A14554
:10226000EFE00FFD5C402A8B0355E4004179B3F7A2
:1022700027016C003EC6EFE00FFD8355C400B24756
:10228000A1463008BE95B385654122852EC8EFF082
:102290007FCBAA84634B05002808EFF05FE611C9E5
:1022A000B2452285EFF0BFD0AA84268561616FF028
:1022B000DEA9C2470357A101417C338B6741B3F7C5
:1022C0002701BA973EC810100C082285C24BEFF0C8
:1022D0001FE8AA8479F90810EFF07FE22DE95C404D
:1022E0003ECA30104C0822855249EFF05FE6AA84BE
:1022F0004DFD03578102835701026316F700281032
:10230000EFF0FFDF09C55840D247E31CF7FC6390AC
:102310002B058357410285CF83572102B3FA8B01E6
:102320000810BE9A1C442311F102EFF0FFF083491C
:102330000401035A4102B309304193F90902631BB6
:102340000A000C102285EFF0DFD4AA8439FDE31CCB
:102350007BF7B9B74E8963733A015289CA86101860
:10236000D6852285EFF01FBEAA8421F163090900FA
:102370000C44CA8610182285EFF09FC7AA84034533
:102380000401CA85EFE0CFEA1C443E9508C4E39EF1
:1023900004F0330A2A41CA9A5DB7EFF27E984111E0
:1023A00091E5FD54268541016FF0DE9AC44983D73B
:1023B00025014CC904C12316F50003C705012A8471
:1023C0002317E50003C51501931607011307000243
:1023D0002308A400C182E366A7FCE1D7B3E4F402BA
:1023E000E9F08547E3FFD7FAA145EFE06FE4AA895A
:1023F000014A01498357C400931509012285BE95FE
:10240000B38535412EC2EFF0BFD119ED0355E4007D
:102410004C00050AEFE02FE39245420A2285135A49
:102420000A01EFF0FFCF09E905098357E4004209EB
:1024300013590901E360F9FC8357E40063944701F1
:10244000D1548DB7639427039245A1463000B385DC
:1024500035412285EFF01FAF35E12800EFF03FCA8C
:1024600011C50355E4004C00EFE0EFDD9247C17A5F
:102470003387374158C04177F98F1CC44C401C4406
:1024800063EEF500A14630002285EFF0BFAB1DE5FD
:102490002800EFF0DFC6032A44001DC15C4003554D
:1024A000E4004179B3F727014C003EC2EFE0AFD919
:1024B00092452285EFF0DFC6635C0502AA84DDB594
:1024C00012450359A100035BC10033F5AA002A9904
:1024D00003450401DA85EFE0AFD54A9508C46314DB
:1024E000450163130B04330A3A412322440179B7AF
:1024F00009C58547A308F40075B54C402285EFF067
:102500001FAB4DFD48408357C40086093375A900B1
:102510003E953305354148C03375250108C42285F1
:10252000EFF03FD379D559BF4D5549BF83471501CA
:10253000C9CFEFF20EFE2A840345050141112E8A10
:10254000A145BA893689328BEFE08FCE8357C4001C
:102550000605898F7D5563E727075C4081443EC2AD
:1025600030004C002285924AEFF07FBE21ED835B64
:10257000810063994B012800EFF07FB801E58504E5
:10258000C204C18058409247630BF702E3FA99FCFA
:102590008356C10061559DC663E63403C175B3FA25
:1025A000BA006373D900CA868355A1005A86228572
:1025B000D695EFF03F9919E50355C10021A061556B
:1025C000E3884BFD41016FF04EF849558280EFF2F0
:1025D000CEF60147EFF09FF56FF06EF8EFF2EEF5F3
:1025E0003284B2862E86835545000841EFF03FFEC7
:1025F000635385002A8422856FF06EF6EFF2EEF0C9
:10260000834715013971C954BDC7034B05012EC657
:102610002A84A1455A853689328AEFE06FC10D4779
:102620003307E5028357C400AA8DFD54998F63E4F4
:1026300027056304090063000A045C403ECA3008B1
:102640004C082285524DEFF09FB0AA8945ED835783
:10265000810132476397E7002808EFF05FAA63061D
:1026600005105840D247E31CF7FC8144631B090066
:1026700019A0814499E7268521616FF0CEECE35CD7
:10268000A0FE5A85CA85EFE0AFBA014B11C5330BE6
:10269000B501420B135B0B01014D7D5CC17B930CBB
:1026A00044008357E4006380A70D1C444440330773
:1026B000FB0063EBE40432472311F1020810FD57DD
:1026C0002310E102231221032303F102EFF0DFB60E
:1026D000630909000C44CA8652862285EFF05F9197
:1026E000AA8903450401CA85EFE08FB41C443E95D6
:1026F00008C4639909000C102285EFF09F99AA89FC
:10270000CA8435D9CE8485BF03450401A145EFE0D5
:102710002FB2B387A4002311F1028357C400B3F48E
:10272000740123108103BE94898C44C008102312C5
:102730000102EFF07FB00C102285EFF09F95AA8484
:102740000355E400E685EFE00FB05C40B3F7770196
:102750001CC4E39204F22285EFF0BFAFAA84E31C0D
:1027600005F0050D3DBFC15439B78357C101E302E0
:1027700009F0E39827F1C177034C0401B377FD001A
:10278000035DA101330C8041137C0C023E9DD28A73
:10279000CA8CE28B63F38C01E68BDE861010EA852F
:1027A0002285EFF02FFAAA84E31B05EC5E860C105D
:1027B0005685EF602041AA84E31505ECB38C7C417B
:1027C0005E9DDE9AE3970CFC7DB5EFF20ED7814655
:1027D0000146EFF0BFE26FF08ED8638C050EEFF28A
:1027E0004ED35D71054D19C213BD16000359050284
:1027F000B68B328B05094209135909012E8A2A84A6
:10280000CA89216C930A8500E15C9304F9FFC20434
:10281000C180638F84059306A0045000A685568569
:10282000EFF0FFDA6357050063139501A689268947
:10283000E9BF9C083E95230A05FA4C005285EFF04B
:102840004EDD75F563040D08835704026395970800
:102850009387F4FF2310F402894613060402A1654E
:102860005685EFF0BFD96358050661616FF0EECD74
:102870000145E31C0DFE0549B1675D55E387F9FE8F
:102880009165CE9593048400C205DE865A86C18187
:102890002685EFF0BFD6630D09005285EF60405DDD
:1028A000AA865286CE852685EFF05FD5E34F05FADE
:1028B0008357040263FF370323103403894613064A
:1028C0000402A1652685EFF07FD325A0A6890149E2
:1028D00065B77D558280A6855685EFF01FEFE346EC
:1028E00005F89165FD15CA95C205C1815685EFF0C1
:1028F000DFEDE35CA0F601458DBFEFF28EC103541E
:102900000502916A1D71050442042A89AE8941803D
:10291000A16B130A8500FD1A130B05029304F4FF43
:10292000C204C180639D7405916B2164130A890000
:10293000850B170C0000130CACCA835709029304D3
:102940001400C204C18085076383F40E5E9493066D
:10295000A0045008A68552854204EFF05FC741806D
:10296000AA8A854613067100A2855285EFF03FC6FC
:102970002A8B634750076347A00626847DBF569481
:102980009306A0045008A68552854204EFF03FC488
:1029900041802A8C854613067100A2855285EFF08E
:1029A0001FC3634C8003E351A0F883570902E39DE2
:1029B00097F69387F4FF2310F90289465A86A1659A
:1029C0005285EFF0BFC3A6855285EFF01FE0A285C8
:1029D0005285EFF09FDF268491B7E358A0FCA9B79A
:1029E000634BA000A6855285EFF03FDEA28552859D
:1029F000EFF0BFDD59B79C10BE9A238A0AFA6391A3
:102A000009022C004808EFF0EFCC25D91C452245DF
:102A100052C62318810074006286DA858297B1BF9E
:102A20000146CE854808EFF00FA261FDB9B7014518
:102A300025616FF08EB1EFF24EB09737FF1F93878D
:102A4000A74D8043814409C42A893114814401E49B
:102A500026856FF0CEB0631809005C4481EF4048D2
:102A600065D83114EDB708400146CA85EFF0AF9D37
:102A70006DF5F5B78297E5F4AA84D5B7EFF2EEAB22
:102A80009737FF1F9387C7498043AA8409EC26859F
:102A9000EFF07FFAAA840144EF502FD0636CA400BA
:102AA00026856FF0CEAB5C402285A6859C4382973D
:102AB0000040E9BF05041374F40FF9BFEFF2EEA76D
:102AC0000145EFF0BFFB6FF08EA99737FF1F93878B
:102AD000274523A0070023A207008280EFF2EEA57E
:102AE0009737FF1F9387474323A0070023A20700C0
:102AF000EFF0BFFD6FF0AEA6EFF22EA44111130967
:102B000085002A84EF50CFE5AA854A85EFF0FF883B
:102B1000AA8419ED89461306E100A1654A85EFF004
:102B20001FABE177634405008357E1002310F402F3
:102B3000268541016FF0AEA29737FF1F9387473E6E
:102B400090430147B28691EE05E3DC4310C117378D
:102B5000FF1F2327A73C85EF9737FF1F23A4A73C20
:102B6000828036879442C5B7144385E2DC43232034
:102B7000050091EB9737FF1F23A6A73A9737FF1F52
:102B800023A0A73A828088C3C1BF14C108C3828032
:102B9000EFF2AE9A1734FF1F1304C4332285EFF00F
:102BA000BFF5AA8405E51799000013092927228596
:102BB0009737FF1F23A22733EFF01FF89737FF1F28
:102BC00023AC27319737FF1F23A0873626856FF068
:102BD0000E999737FF1F83C76735795599EFEFF245
:102BE000CE95EFF0BFEFEFF0BFFA11E5854717374D
:102BF000FF1F230DF7326FF08E968280EFF2EE9377
